S01B00006275666665725F646973635F625F626F6172642E7372656365
S3150802000000000A20C56A020891520208995202089B
S31508020010A1520208A9520208B1520208156B020837
S31508020020000000000000000000000000B9520208AB
S31508020030C752020800000000D5520208E35202081D
S31508020040156B0208156B0208156B0208156B020878
S31508020050156B0208156B0208156B0208156B020868
S31508020060156B0208156B0208156B0208156B020858
S31508020070156B0208156B0208156B0208156B020848
S31508020080156B0208156B0208156B0208156B020838
S31508020090156B0208156B0208156B0208156B020828
S315080200A0156B0208156B0208156B0208156B020818
S315080200B0156B0208156B0208156B0208156B020808
S315080200C0156B0208156B0208156B0208156B0208F8
S315080200D000000000156B0208156B0208F1520208AF
S315080200E0156B0208156B0208156B0208156B0208D8
S315080200F0156B020805530208156B0208156B0208F0
S31508020100156B020819530208156B0208156B0208CB
S31508020110156B0208156B0208156B0208156B0208A7
S31508020120156B0208156B02082D530208156B020897
S31508020130156B0208156B0208156B0208156B020887
S31508020140156B0208156B0208156B0208156B020877
S31508020150156B0208156B0208156B0208156B020867
S31508020160156B0208156B0208156B0208156B020857
S31508020170156B0208156B0208156B0208156B020847
S31508020180156B0208156B0208156B0208156B020837
S31508020190156B0208156B0208156B0208156B020827
S315080201A0156B0208156B0208156B0208156B020817
S315080201B0156B0208156B0208156B0208156B020807
S315080201C0156B0208156B0208156B0208156B0208F7
S315080201D0156B0208156B0208156B0208156B0208E7
S315080201E0156B0208156B0208156B0208156B0208D7
S315080201F0156B0208156B0208156B0208156B0208C7
S31508020200156B0208156B0208156B02080000000040
S3150802021000000000156B020800000000156B0208BA
S31508020220156B0208156B0208156B0208156B020896
S31508020230156B0208156B0208156B0208156B020886
S31508020240156B0208156B0208156B02080000000000
S3150802025010B5054C237833B9044B13B10448AFF3F0
S3150802026000800123237010BD8407002000000000CF
S315080202702C95030808B5034B1BB103490348AFF392
S31508020280008008BD00000000880700202C9503089E
S31508020290034613F8012B002AFBD1181A01387047B6
S315080202A081F0004102E000BF83F0004330B54FEA17
S315080202B041044FEA430594EA050F08BF90EA020F84
S315080202C01FBF54EA000C55EA020C7FEA645C7FEA17
S315080202D0655C00F0E2804FEA5454D4EB5555B8BF3A
S315080202E06D420CDD2C4480EA020281EA030382EAAB
S315080202F0000083EA010180EA020281EA0303362D3D
S3150802030088BF30BD11F0004F4FEA01314FF4801C0F
S315080203104CEA113102D0404261EB410113F0004F21
S315080203204FEA03334CEA133302D0524263EB4303D8
S3150802033094EA050F00F0A780A4F10104D5F1200E76
S315080203400DDB02FA0EFC22FA05F2801841F10001D1
S3150802035003FA0EF2801843FA05F359410EE0A5F1A5
S3150802036020050EF1200E012A03FA0EFC28BF4CF0D6
S31508020370020C43FA05F3C01851EBE37101F000458C
S3150802038007D54FF0000EDCF1000C7EEB00006EEB99
S315080203900101B1F5801F1BD3B1F5001F0CD3490823
S315080203A05FEA30004FEA3C0C04F101044FEA44527A
S315080203B012F5800F80F09A80BCF1004F08BF5FEA01
S315080203C0500C50F1000041EB045141EA050130BDE1
S315080203D05FEA4C0C404141EB0101013C28BFB1F5F3
S315080203E0801FE9D291F0000F04BF01460020B1FA3E
S315080203F081F308BF2033A3F10B03B3F120020CDA11
S315080204000C3208DD02F1140CC2F10C0201FA0CF0EE
S3150802041021FA02F10CE002F11402D8BFC2F1200C53
S3150802042001FA02F120FA0CFCDCBF41EA0C01904009
S31508020430E41AA2BF01EB0451294330BD6FEA040452
S315080204401F3C1CDA0C340EDC04F11404C4F120023D
S3150802045020FA04F001FA02F340EA030021FA04F34F
S3150802046045EA030130BDC4F10C04C4F1200220FAA6
S3150802047002F001FA04F340EA0300294630BD21FAE4
S3150802048004F0294630BD94F0000F83F4801306BFAA
S3150802049081F480110134013D4EE77FEA645C18BF9E
S315080204A07FEA655C29D094EA050F08BF90EA020F35
S315080204B005D054EA000C04BF1946104630BD91EA2D
S315080204C0030F1EBF0021002030BD5FEA545C05D130
S315080204D04000494128BF41F0004130BD14F580046F
S315080204E03CBF01F5801130BD01F0004545F0FE41E3
S315080204F041F470014FF0000030BD7FEA645C1ABF18
S31508020500194610467FEA655C1CBF0B46024650EA4E
S31508020510013406BF52EA033591EA030F41F400217A
S3150802052030BD00BF90F0000F04BF0021704730B500
S315080205304FF4806404F132044FF000054FF00001D5
S3150802054050E700BF90F0000F04BF0021704730B596
S315080205504FF4806404F1320410F0004548BF40426B
S315080205604FF000013EE700BF42004FEAE2014FEAC0
S3150802057031014FEA02701FBF12F07F4393F07F4F9B
S3150802058081F06051704732F07F4208BF704793F09E
S315080205907F4F04BF41F40021704730B54FF46074B1
S315080205A001F0004521F000411CE700BF50EA0102B4
S315080205B008BF704730B54FF000050AE050EA01025D
S315080205C008BF704730B511F0004502D5404261EBCD
S315080205D041014FF4806404F132045FEA915C3FF40E
S315080205E0D8AE4FF003025FEADC0C18BF03325FEAAB
S315080205F0DC0C18BF033202EBDC02C2F1200300FA5C
S3150802060003FC20FA02F001FA03FE40EA0E0021FA80
S3150802061002F11444BDE600BF70B54FF0FF0C4CF46E
S31508020620E06C1CEA11541DBF1CEA135594EA0C0F20
S3150802063095EA0C0F00F0DEF82C4481EA030621EA5B
S315080206404C5123EA4C5350EA013518BF52EA033596
S3150802065041F4801143F4801338D0A0FB02CE4FF048
S315080206600005E1FB02E506F00042E0FB03E54FF078
S315080206700006E1FB03569CF0000F18BF4EF0010E70
S31508020680A4F1FF04B6F5007F64F5407404D25FEA6C
S315080206904E0E6D4146EB060642EAC62141EA55511F
S315080206A04FEAC52040EA5E504FEACE2EB4F1FD0C61
S315080206B088BFBCF5E06F1ED8BEF1004F08BF5FEADF
S315080206C0500E50F1000041EB045170BD06F0004691
S315080206D046EA010140EA020081EA0301B4EB5C043E
S315080206E0C2BFD4EB0C0541EA045170BD41F4801136
S315080206F04FF0000E013C00F3AB8014F1360FDEBF5B
S31508020700002001F0004170BDC4F10004203C35DA36
S315080207100C341BDC04F11404C4F1200500FA05F3B9
S3150802072020FA04F001FA05F240EA020001F000425A
S3150802073021F0004110EBD37021FA04F642EB0601D0
S315080207405EEA430E08BF20EAD37070BDC4F10C04FA
S31508020750C4F1200500FA04F320FA05F001FA04F2BE
S3150802076040EA020001F0004110EBD37041F10001AA
S315080207705EEA430E08BF20EAD37070BDC4F12005B5
S3150802078000FA05F24EEA020E20FA04F301FA05F21D
S3150802079043EA020321FA04F001F0004121FA04F2C5
S315080207A020EA020000EBD3705EEA430E08BF20EA95
S315080207B0D37070BD94F0000F0FD101F000464000CF
S315080207C041EB010111F4801F08BF013CF7D041EA51
S315080207D0060195F0000F18BF704703F00046520055
S315080207E043EB030313F4801F08BF013DF7D043EA26
S315080207F00603704794EA0C0F0CEA135518BF95EADC
S315080208000C0F0CD050EA410618BF52EA4306D1D162
S3150802081081EA030101F000414FF0000070BD50EA81
S31508020820410606BF1046194652EA430619D094EA0B
S315080208300C0F02D150EA013613D195EA0C0F05D1F5
S3150802084052EA03361CBF104619460AD181EA030149
S3150802085001F0004141F0FE4141F470014FF0000001
S3150802086070BD41F0FE4141F4780170BD70B54FF09C
S31508020870FF0C4CF4E06C1CEA11541DBF1CEA13551C
S3150802088094EA0C0F95EA0C0F00F0A7F8A4EB0504FE
S3150802089081EA030E52EA03354FEA013100F08880F5
S315080208A04FEA03334FF0805545EA131343EA1263BE
S315080208B04FEA022245EA111545EA10654FEA002673
S315080208C00EF000419D4208BF964244F1FD0404F52C
S315080208D0407402D25B084FEA3202B61A65EB030588
S315080208E05B084FEA32024FF480104FF4002CB6EB45
S315080208F0020E75EB030E22BFB61A754640EA0C00C5
S315080209005B084FEA3202B6EB020E75EB030E22BF04
S31508020910B61A754640EA5C005B084FEA3202B6EB45
S31508020920020E75EB030E22BFB61A754640EA9C0004
S315080209305B084FEA3202B6EB020E75EB030E22BFD4
S31508020940B61A754640EADC0055EA060E18D04FEA92
S31508020950051545EA16754FEA06164FEAC30343EA32
S3150802096052734FEAC2025FEA1C1CC0D111F4801FFF
S315080209700BD141EA00014FF000004FF0004CB6E7F8
S3150802098011F4801F04BF01430020B4F1FD0C88BF97
S31508020990BCF5E06F3FF6AFAEB5EB030C04BFB6EBA2
S315080209A0020C5FEA500C50F1000041EB045170BD95
S315080209B00EF0004E4EEA113114EB5C04C2BFD4EBC2
S315080209C00C0541EA045170BD41F480114FF0000E46
S315080209D0013C90E645EA060E8DE60CEA135594EAC2
S315080209E00C0F08BF95EA0C0F3FF43BAF94EA0C0FC5
S315080209F00AD150EA01347FF434AF95EA0C0F7FF43A
S31508020A0025AF104619462CE795EA0C0F06D152EA8D
S31508020A1003353FF4FDAE1046194622E750EA410671
S31508020A2018BF52EA43067FF4C5AE50EA41047FF482
S31508020A300DAF52EA43057FF4EBAE12E74FF0FF3CE7
S31508020A4006E000BF4FF0010C02E000BF4FF0010CB8
S31508020A504DF804CD4FEA410C7FEA6C5C4FEA430C31
S31508020A6018BF7FEA6C5C1BD001B050EA410C0CBF80
S31508020A7052EA430C91EA030F02BF90EA020F0020E2
S31508020A80704710F1000F91EA030F58BF994208BF49
S31508020A9090422CBFD8176FEAE37040F00100704706
S31508020AA04FEA410C7FEA6C5C02D150EA013C07D15D
S31508020AB04FEA430C7FEA6C5CD6D152EA033CD3D0A8
S31508020AC05DF8040B704700BF8446104662468C46A2
S31508020AD01946634600E000BF01B5FFF7B7FF0028D5
S31508020AE048BF10F1000F01BD4DF808EDFFF7F4FFFE
S31508020AF00CBF012000205DF808FB00BF4DF808ED89
S31508020B00FFF7EAFF34BF012000205DF808FB00BFAB
S31508020B104DF808EDFFF7E0FF94BF012000205DF8CD
S31508020B2008FB00BF4DF808EDFFF7CEFF94BF012082
S31508020B3000205DF808FB00BF4DF808EDFFF7C4FF7B
S31508020B4034BF012000205DF808FB00BF4FEA410CC4
S31508020B507FEA6C5C02D150EA013C0AD14FEA430CA7
S31508020B607FEA6C5C02D152EA033C02D14FF00000E4
S31508020B7070474FF0010070474FEA410212F5001222
S31508020B8015D211D56FF47873B3EB625212D94FEAC4
S31508020B90C12343F0004343EA505311F0004F23FAAE
S31508020BA002F018BF404270474FF00000704750EA03
S31508020BB0013005D111F0004008BF6FF000407047C0
S31508020BC04FF00000704700BF4A0011D212F500121A
S31508020BD011D20DD56FF47873B3EB62520ED44FEA85
S31508020BE0C12343F0004343EA505323FA02F0704705
S31508020BF04FF00000704750EA013002D14FF0FF3043
S31508020C0070474FF0000070474FEA4102B2F1E043E5
S31508020C1024BFB3F5001CDCF1FE5C0DD901F0004CD3
S31508020C204FEAC0024CEA5070B2F1004F40EB830023
S31508020C3008BF20F00100704711F0804F21D113F14F
S31508020C403872BCBF01F00040704741F480114FEA88
S31508020C505252C2F11802C2F1200C10FA0CF320FA11
S31508020C6002F018BF40F001004FEAC1234FEAD3232E
S31508020C7003FA0CFC40EA0C0023FA02F34FEA430398
S31508020C80CCE77FEA625307D150EA01331EBF4FF021
S31508020C90FE4040F44000704701F0004040F0FE403C
S31508020CA040F40000704700BF53B94AB9002908BF8B
S31508020CB000281CBF4FF0FF314FF0FF3000F0B4B9E7
S31508020CC0ADF1080C6DE904CE00F03CF8DDF804E05D
S31508020CD0DDE9022304B0704738B500220023044632
S31508020CE00D46FFF70BFF28B920462946BDE83840CE
S31508020CF000F00AB8204605F1004100F005F8404226
S31508020D0061EB410138BD00BFD0B500220B4B064648
S31508020D100F46FFF781FCFFF757FF0446FFF702FC71
S31508020D200022074BFFF778FC02460B463046394647
S31508020D30FFF7BAFAFFF748FF2146D0BD0000F03D9B
S31508020D400000F0412DE9F04F099D0C46002B4DD1CC
S31508020D508A420F4684469646B2FA82F360D94BB166
S31508020D6002FA03FEC3F120029F4000FA03FC20FAAE
S31508020D7002F217434FEA1E461FFA8EF44FEA1C4246
S31508020D80B7FBF6F106FB117701FB04F042EA0742CC
S31508020D90904208D91EEB020201F1FF3702D29042B5
S31508020DA000F22D813946121A1FFA8CFCB2FBF6F0B4
S31508020DB006FB102200FB04F44CEA024C644508D9EF
S31508020DC01EEB0C0C00F1FF3202D2644500F21A81C6
S31508020DD0104640EA0140ACEB040C002125B12CFA7E
S31508020DE003F30022C5E90032BDE8F08F8B4205D92C
S31508020DF00DB1C5E9000100210846F5E7B3FA83F10A
S31508020E0000294DD1A342C0F0F280904280F0EF80D3
S31508020E10064623460846002DE6D0C5E90063E3E701
S31508020E20002B40F0A2808A1A4FEA1E471FFA8EF656
S31508020E300121B2FBF7F407FB14204FEA1C4242EAEF
S31508020E40004206FB04F090420FD91EEB020204F19F
S31508020E50FF382CBF4FF001094FF00009904203D921
S31508020E60B9F1000F00F0C8804446121A1FFA8CFC2A
S31508020E70B2FBF7F007FB102200FB06F64CEA024C1F
S31508020E80664508D91EEB0C0C00F1FF3202D2664504
S31508020E9000F2BB801046ACEB060C40EA04409DE724
S31508020EA0C1F120068B4004FA01FE22FA06F720FA5F
S31508020EB006FCF4408A401F434EEA0C0300FA01FE80
S31508020EC04FEA17484FEA13491FFA87FCB4FBF8F0B2
S31508020ED008FB104449EA044400FB0CF9A1450ED963
S31508020EE03C1900F1FF3A2CBF4FF0010B4FF0000BF3
S31508020EF0A14503D9BBF1000F00F093805046A4EB3D
S31508020F0009041FFA83F9B4FBF8F308FB134403FB3D
S31508020F100CFC49EA0444A44506D93C1903F1FF38F6
S31508020F2001D2A4457AD8434643EA0040A4EB0C040E
S31508020F30A0FB02984445CC46434602D306D1CE4589
S31508020F4004D20138B9EB020C68EB07035DB1BEEBBC
S31508020F500C0264EB030404FA06F622FA01F3CC4007
S31508020F601E43C5E9006400213EE702FA03FEC3F107
S31508020F70200104FA03F200FA03FCCC404FEA1E47AA
S31508020F8020FA01F11FFA8EF6B4FBF7F00A4307FBC3
S31508020F901044110C41EA044100FB06F48C420ED9B6
S31508020FA01EEB010100F1FF382CBF4FF001094FF08B
S31508020FB000098C4202D9B9F1000F2CD04046091B10
S31508020FC092B2B1FBF7F407FB141142EA014204FBA1
S31508020FD006F1914207D91EEB020204F1FF3801D24B
S31508020FE0914215D84446521A44EA004121E7861A24
S31508020FF064EB030301200EE7023C724435E702392B
S315080210007244D0E6F4440238E3E6F444023842E78E
S31508021010023C7244E7E702387144D0E7023B3C449B
S3150802102082E702383C446AE7704700BF80B582B05F
S3150802103000AF04F015FA0346184604F05EFA786023
S3150802104024220021786814F0AFFF054805F0BEFC9B
S315080210507B68044A1A6000BF0837BD4680BD00BFD8
S31508021060509503080245434980B588B000AFF86039
S31508021070B9601346FB710023FB6100233B61BB6821
S315080210807B617B69BB610023FB6110E0FA69FB683F
S315080210901344184612F072FA03463B613A69BB6971
S315080210A01A60BB690433BB61FB690433FB61FB79D4
S315080210B0FA699A42EADB012318462037BD4680BD03
S315080210C080B58CB000AF002387F82F3004F0C8F93A
S315080210D00346184604F011FAB86224220021B86AB7
S315080210E014F062FF3B1D24220021184614F05CFF0F
S315080210F03B1D242219460F48FFF7B6FF7B680E4AA6
S31508021100934205D0FFF792FF002387F82F300BE0B2
S315080211103B1D24221946B86A14F0FDFF074805F05C
S3150802112055FC012387F82F3097F82F3018463037A9
S31508021130BD4680BD00C01F0802454349689503089D
S3150802114090B589B000AF0023FB6104F089F9034624
S31508021150184604F0D2F978617B69BB61FE2012F069
S315080211603CFA0023FB611CE03B1D102200211846B5
S3150802117014F01AFFBB693C1D186859689A68DB683F
S315080211800FC4FB6903F1016303F57C233A1D11467B
S31508021190184612F007FABB691033BB61FB691033B4
S315080211A0FB61FB69232BDFD9012318462437BD4689
S315080211B090BD000080B483B000AF0346FB71FB7993
S315080211C0002B02D1194B1B682AE0FB79012B02D1AD
S315080211D0174B1B6824E0FB79022B02D1154B1B68BF
S315080211E01EE0FB79032B02D1134B1B6818E0FB792F
S315080211F0042B02D1114B1B6812E0FB79052B02D195
S315080212000F4B1B680CE0FB79062B02D10D4B1B68B2
S3150802121006E0FB79072B02D10B4B1B6800E0002383
S3150802122018460C37BD465DF8047B7047A0070020B8
S31508021230A4070020A8070020AC070020B00700205A
S31508021240B4070020B8070020BC07002080B483B08A
S3150802125000AF03463960FB71FB79002B03D11D4AA7
S315080212603B6813602FE0FB79012B03D11A4A3B68CE
S31508021270136028E0FB79022B03D1184A3B681360F6
S3150802128021E0FB79032B03D1154A3B6813601AE068
S31508021290FB79042B03D1134A3B68136013E0FB79ED
S315080212A0052B03D1104A3B6813600CE0FB79062B29
S315080212B003D10E4A3B68136005E0FB79072B02D17E
S315080212C00B4A3B68136000BF0C37BD465DF8047BCA
S315080212D0704700BFA0070020A4070020A807002027
S315080212E0AC070020B0070020B4070020B80700208A
S315080212F0BC07002080B586B000AFF8600B467A605E
S31508021300FB720023FB752D4805F060FB0023FB7575
S315080213104CE0FB7D2A4A4FF48E7101FB03F313441A
S315080213201B78012B3FD1FB7D4FF48E7202FB03F330
S31508021330234A134402331946224805F047FB22483A
S3150802134005F044FBFB7D4FF48E7202FB03F3183360
S315080213501B4A1344043319461A4805F037FB1B483F
S3150802136005F034FBFB7D164A4FF48E7101FB03F33D
S3150802137013449C331B782D2B12D0154805F026FBF7
S31508021380FB7D4FF48E7202FB03F398330C4A134427
S31508021390043319460B4805F019FB0C4805F016FBF1
S315080213A00A4805F013FBFB7D0133FB75FB7D042B15
S315080213B0AFD900BF00BF1837BD4680BD7895030870
S315080213C000000020A0950308A4950308A895030821
S315080213D0AC95030880B586B000AFF8600B467A6014
S315080213E0FB7200237B617B6803F5007303221649AF
S315080213F0184614F0E1FD0346002B21D17B6803F55C
S3150802140000731846FEF744FF0346032B18D17B6880
S3150802141003F58063184613F0C5FC78617B69002BD7
S3150802142007D004F01DF803460121184604F036FBDE
S3150802143006E004F015F803460121184604F04BFBB2
S3150802144000BF1837BD4680BDB895030880B584B07D
S3150802145000AFF8600B467A60FB727B6803F500738F
S315080214600422A949184614F0A7FD0346002B08D101
S315080214707B6803F500731846FEF70AFF0346042B3A
S3150802148013D07B6803F500731A78A04B1B78D31A1E
S31508021490002B40F0D7807B6803F500731846FEF7E9
S315080214A0F7FE0346012B40F0CD807B6803F5806387
S315080214B01A78974B1B78D31A002B0FD17B6803F542
S315080214C080631846FEF7E4FE0346012B06D19148CF
S315080214D005F07CFA002000F077FFB2E07B6803F59E
S315080214E080631A788C4B1B78D31A002B0FD17B6832
S315080214F003F580631846FEF7CBFE0346012B06D199
S31508021500864805F063FA012000F05EFF99E07B68E1
S3150802151003F580631A78824B1B78D31A002B0FD1F6
S315080215207B6803F580631846FEF7B2FE0346012B75
S3150802153006D17C4805F04AFA022000F045FF80E011
S315080215407B6803F580631A78774B1B78D31A002BCE
S315080215500FD17B6803F580631846FEF799FE0346AA
S31508021560012B06D1714805F031FA032000F02CFF51
S3150802157067E07B6803F580631A786D4B1B78D31A8C
S31508021580002B0FD17B6803F580631846FEF780FEB1
S315080215900346012B06D1674805F018FA042000F025
S315080215A013FF4EE07B6803F580631A78624B1B785B
S315080215B0D31A002B0FD17B6803F580631846FEF712
S315080215C067FE0346012B06D15C4805F0FFF90520A4
S315080215D000F0FAFE35E07B6803F580631A78584B0B
S315080215E01B78D31A002B0FD17B6803F58063184644
S315080215F0FEF74EFE0346012B06D1524805F0E6F9E0
S31508021600062000F0E1FE1CE07B6803F580631A7889
S315080216104D4B1B78D31A002B0FD17B6803F58063D9
S315080216201846FEF735FE0346012B06D1474805F054
S31508021630CDF9072000F0C8FE03E0454805F0C6F9D3
S3150802164030E32FE37B6803F500730322414918460A
S3150802165014F0B2FC0346002B40F006817B6803F5C2
S3150802166000731846FEF714FE0346032B40F0FC806F
S315080216707B6803F580631A78254B1B78D31A002BEF
S315080216800FD17B6803F580631846FEF701FE034611
S31508021690012B06D1304805F099F9002001F0E4F84B
S315080216A0E1E07B6803F580631A781B4B1B78D31A33
S315080216B0002B0FD17B6803F580631846FEF7E8FD19
S315080216C00346012B06D1254805F080F9012001F0D1
S315080216D0CBF8C8E07B6803F580631A78104B1B7851
S315080216E0D31A002B3ED17B6803F580631846FEF7B2
S315080216F0CFFD0346012B35D1194805F067F90220BB
S3150802170001F0B2F8AFE000BFBC950308C495030820
S31508021710C8950308CC950308F0950308F4950308C1
S31508021720189603081C96030840960308449603086D
S31508021730689603086C96030890960308949603081D
S31508021740B8960308BC960308E0960308E4960308CD
S31508021750089703081C970308209703083C97030871
S315080217605C9703087B6803F580631A78AF4B1B788E
S31508021770D31A002B0FD17B6803F580631846FEF750
S3150802178087FD0346012B06D1A94805F01FF9032058
S3150802179001F06AF867E07B6803F580631A78A54B5F
S315080217A01B78D31A002B0FD17B6803F58063184682
S315080217B0FEF76EFD0346012B06D19F4805F006F992
S315080217C0042001F051F84EE07B6803F580631A782D
S315080217D09A4B1B78D31A002B0FD17B6803F58063CB
S315080217E01846FEF755FD0346012B06D1944805F027
S315080217F0EDF8052001F038F835E07B6803F58063DB
S315080218001A78904B1B78D31A002B0FD17B6803F5F5
S3150802181080631846FEF73CFD0346012B06D18A482B
S3150802182005F0D4F8062001F01FF81CE07B6803F5E2
S3150802183080631A78854B1B78D31A002B0FD17B68E5
S3150802184003F580631846FEF723FD0346012B06D1EE
S315080218507F4805F0BBF8072001F006F803E07D484B
S3150802186005F0B4F81EE21DE27B6803F50073042254
S315080218707949184614F0A0FB0346002B11D17B6860
S3150802188003F500731846FEF703FD0346042B08D139
S31508021890724805F09BF8FFF753FC714805F096F875
S315080218A000E27B6803F5007305226E49184614F0B8
S315080218B083FB0346002B40F05F817B6803F50073C8
S315080218C01846FEF7E5FC0346052B40F055817B6872
S315080218D003F580631A78644B1B78D31A002B19D147
S315080218E07B6803F580631846FEF7D2FC0346012B94
S315080218F010D15E4805F06AF8002000F0EFFD10EE00
S31508021900103A1846FEF730FE02460B46584805F0CE
S315080219105DF830E17B6803F580631A78554B1B78CE
S31508021920D31A002B19D17B6803F580631846FEF794
S31508021930AFFC0346012B10D14F4805F047F80120AA
S3150802194000F0CCFD10EE103A1846FEF70DFE0246E0
S315080219500B464A4805F03AF80DE17B6803F58063C1
S315080219601A78474B1B78D31A002B19D17B6803F5D3
S3150802197080631846FEF78CFC0346012B10D14148BA
S3150802198005F024F8022000F0A9FD10EE103A1846D8
S31508021990FEF7EAFD02460B463B4805F017F8EAE071
S315080219A07B6803F580631A78204B1B78D31A002BC1
S315080219B019D17B6803F580631846FEF769FC03466E
S315080219C0012B10D1314805F001F8032000F086FDFD
S315080219D010EE103A1846FEF7C7FD02460B462C488B
S315080219E004F0F4FFC7E07B6803F580631A78114BAD
S315080219F01B78D31A002B51D17B6803F580631846EE
S31508021A00FEF746FC0346012B48D1224804F0DEFFC6
S31508021A10042000F063FD10EE103A1846FEF7A4FD06
S31508021A2002460B461C4804F0D1FFA4E04096030880
S31508021A307C9703086896030820970308909603087C
S31508021A409C970308B8960308BC970308E096030810
S31508021A50DC97030808970308FC9703080498030809
S31508021A602098030840980308C8950308489803086D
S31508021A7068980308F095030884980308A49803084D
S31508021A8018960308C0980308E0980308FC98030808
S31508021A901C99030838990308589903087B6803F5C3
S31508021AA080631A78814B1B78D31A002B19D17B686D
S31508021AB003F580631846FEF7EBFB0346012B10D1AC
S31508021AC07B4804F083FF052000F008FD10EE103A6B
S31508021AD01846FEF749FD02460B46764804F076FF9D
S31508021AE049E07B6803F580631A78734B1B78D31A2F
S31508021AF0002B19D17B6803F580631846FEF7C8FBED
S31508021B000346012B10D16D4804F060FF062000F051
S31508021B10E5FC10EE103A1846FEF726FD02460B467D
S31508021B20674804F053FF26E07B6803F580631A785A
S31508021B30644B1B78D31A002B19D17B6803F5806393
S31508021B401846FEF7A5FB0346012B10D15E4804F0A2
S31508021B503DFF072000F0C2FC10EE103A1846FEF7C9
S31508021B6003FD02460B46594804F030FF03E0584885
S31508021B7004F02CFF96E095E07B6803F500730722D4
S31508021B805449184614F018FA0346002B40F086808A
S31508021B907B6803F500731846FEF77AFB0346072BA4
S31508021BA07CD17B6803F580631A784B4B1B78D31A72
S31508021BB0002B14D17B6803F580631846FEF768FB91
S31508021BC00346012B0BD1454804F000FF002000F024
S31508021BD0C5FA03461946424804F0F8FE5DE07B68FA
S31508021BE003F580631A783F4B1B78D31A002B14D15E
S31508021BF07B6803F580631846FEF74AFB0346012B0A
S31508021C000BD1394804F0E2FE012000F0A7FA034698
S31508021C101946364804F0DAFE3FE07B6803F580632E
S31508021C201A78334B1B78D31A002B14D17B6803F529
S31508021C3080631846FEF72CFB0346012B0BD12D4871
S31508021C4004F0C4FE022000F089FA034619462A481F
S31508021C5004F0BCFE21E07B6803F580631A78274B03
S31508021C601B78D31A002B14D17B6803F580631846B8
S31508021C70FEF70EFB0346012B0BD1214804F0A6FE04
S31508021C80032000F06BFA034619461E4804F09EFE2E
S31508021C9003E00F4804F09AFE04E003E00C4804F05F
S31508021CA095FE00BF1037BD4680BD00BF909603085B
S31508021CB07499030894990308B8960308B099030817
S31508021CC0D0990308E0960308EC9903080C9A0308CE
S31508021CD008970308289A0308C8950308309A030840
S31508021CE0509A0308F0950308689A0308889A030825
S31508021CF018960308A09A0308C09A03084096030890
S31508021D00D89A0308F89A030880B584B000AFF86039
S31508021D100B467A60FB7203F0A3FB0346184603F0F0
S31508021D20C3FB00BF1037BD4680BD000090B585B025
S31508021D3000AF78600023BB730023FB734FF4A052F5
S31508021D400021204814F030F907F10E030A221D4932
S31508021D5078680FF0D9FF0346012B2ED10023FB73B7
S31508021D6028E0FB7B4FF48E7202FB03F3164A1344F8
S31508021D709C1C1448FEF78CFA03461A46114920465B
S31508021D8014F01AF90346002B11D1FB7B0E4A4FF4C5
S31508021D908E7101FB03F3134418331B68B97B094A96
S31508021DA000209847094804F011FE012306E0FB7B50
S31508021DB00133FB73FB7B042BD3D900231846143754
S31508021DC0BD4690BDC007002000000020A895030864
S31508021DD080B582B000AF0346FB71FB790D2B24D187
S31508021DE04F4B00221A704F4804F0F0FD4E4B1B78F9
S31508021DF0002B16D04D48FFF799FF0346012B08D151
S31508021E00F02200214A4814F0CFF84849484814F00D
S31508021E106CF9454B00221A70F0220021434814F04F
S31508021E20C3F8444804F0D2FD76E0FB790A2B03D1C5
S31508021E303B4B00221A706FE0FB791B2B03D1384B00
S31508021E4001221A7068E0FB795B2B07D1344B1B78A9
S31508021E50012B03D1324B02221A705DE0FB79412B2A
S31508021E601FD12F4B1B78022B1BD12D4B00221A7028
S31508021E702D4B1B78002B4FD12D492F4804F0A6FD78
S31508021E802B48FEF705FA0346DAB2274B1A70F022F8
S31508021E900021264814F088F82549244814F025F923
S31508021EA03AE0FB79082B02D0FB797F2B16D11C4B23
S31508021EB000221A701C4B1B78002B2DD01A4B1B784C
S31508021EC0013BDAB2184B1A70174B1B781A46174B96
S31508021ED000219954194804F079FD1DE0124B1B782C
S31508021EE05A1CD1B2104A11701946104AFB7953543A
S31508021EF00D4B1A78124BA3FB0213D9090B461B0189
S31508021F005B1A1B01D31ADAB2074B1A70FB79194608
S31508021F100C4804F05BFDFFE700BF0837BD4680BDED
S31508021F20A11D0020A8950308A01D0020B01C0020B2
S31508021F30C01B0020109B0308A0950308149B0308E6
S31508021F4089888888189B030880B58CB004AF00235B
S31508021F50FB610023BB6100237B6100233B610023F5
S31508021F60FB600023BB6000237B6000233B6003F019
S31508021F7077FA0346184603F0C0FA0346184603F0F2
S31508021F80D7FAF86103F06CFA0346184603F0B5FA75
S31508021F900346184603F0E7FAB86103F061FA034606
S31508021FA0184603F0AAFA0346184603F0F7FA7861C8
S31508021FB003F056FA0346184603F09FFA03461846F4
S31508021FC003F007FB386103F04BFA0346184603F0A1
S31508021FD094FA0346184603F017FBF86003F040FA32
S31508021FE00346184603F089FA0346184603F027FB08
S31508021FF0B86003F035FA0346184603F07EFA03463C
S31508022000184603F037FB786003F02AFA03461846A7
S3150802201003F073FA0346184603F047FB38600020BC
S31508022020FFF7C8F80246FB69029301922023009340
S315080220303C4B10223B493C480FF0D8FB0120FFF7E6
S31508022040B9F80246BB69029301924FF40053009312
S31508022050364B4FF48052354935480FF0C7FB0220FC
S31508022060FFF7A8F802467B69029301924FF40073C0
S315080220700093304B4FF480722E492F480FF0B6FB6F
S315080220800320FFF797F802463B6902930192202341
S3150802209000932A4B1022294929480FF0A7FB04204E
S315080220A0FFF788F80246FB68029301924FF4006331
S315080220B00093224B4FF48062204922480FF096FB88
S315080220C00520FFF777F80246BB6802930192402380
S315080220D000931D4B20221C491C480FF087FB062043
S315080220E0FFF768F802467B6802930192022300937F
S315080220F0174B0122164917480FF078FB0720FFF7FE
S3150802210059F802463B68029301924FF48073009392
S315080221100F4B80220E4910480FF068FB00BF20378C
S31508022120BD4680BD00080242A41D002000100242DE
S31508022130C01D0020000C0242DC1D002000180242CD
S31508022140F81D0020141E002000040242301E002042
S31508022150001402424C1E0020681E002080B582B080
S3150802216000AF0346FB71FB79002B04D120480FF020
S3150802217071FB034638E0FB79012B04D11D480FF0A9
S3150802218069FB034630E0FB79022B04D11A480FF0AB
S3150802219061FB034628E0FB79032B04D117480FF0AD
S315080221A059FB034620E0FB79042B04D114480FF0AF
S315080221B051FB034618E0FB79052B04D111480FF0B1
S315080221C049FB034610E0FB79062B04D10E480FF0B3
S315080221D041FB034608E0FB79072B04D10B480FF0B5
S315080221E039FB034600E0002318460837BD4680BD82
S315080221F0A41D0020C01D0020DC1D0020F81D0020A3
S31508022200141E0020301E00204C1E0020681E0020CE
S3150802221080B582B000AF03460A46FB711346BB710E
S31508022220FB79002B06D1BB79194628480FF064FBC7
S31508022230034646E0FB79012B06D1BB7919462448A9
S315080222400FF05AFB03463CE0FB79022B06D1BB7919
S31508022250194620480FF050FB034632E0FB79032B60
S3150802226006D1BB7919461C480FF046FB034628E0FF
S31508022270FB79042B06D1BB79194618480FF03CFBAB
S3150802228003461EE0FB79052B06D1BB79194614488D
S315080222900FF032FB034614E0FB79062B06D1BB7915
S315080222A0194610480FF028FB03460AE0FB79072B6C
S315080222B006D1BB7919460C480FF01EFB034600E00F
S315080222C0002318460837BD4680BD00BFA41D00205E
S315080222D0C01D0020DC1D0020F81D0020141E002051
S315080222E0301E00204C1E0020681E002080B582B0D9
S315080222F000AF0346FB71FB79002B08D10020FEF7DD
S3150802230059FF0346194629480FF019FB49E0FB799C
S31508022310012B08D10120FEF74DFF03461946244832
S315080223200FF00DFB3DE0FB79022B08D10220FEF7E8
S3150802233041FF034619461F480FF001FB31E0FB79BE
S31508022340032B08D10320FEF735FF034619461A4820
S315080223500FF0F5FA25E0FB79042B08D10420FEF7E5
S3150802236029FF0346194615480FF0E9FA19E0FB79E1
S31508022370052B16D0FB79062B08D10620FEF71AFF85
S31508022380034619460E480FF0DAFA0AE0FB79072BDC
S3150802239007D10720FEF70EFF0346194609480FF034
S315080223A0CEFA00BF0837BD4680BD00BFA41D002077
S315080223B0C01D0020DC1D0020F81D0020141E002070
S315080223C04C1E0020681E002080B584B000AF03466C
S315080223D0FB710023FB60FB79002B0CD10521002041
S315080223E0FFF716FFF860F9680020FEF72FFF0020B6
S315080223F0FFF77CFF6EE0FB79012B0CD1052101204A
S31508022400FFF706FFF860F9680120FEF71FFF0120B3
S31508022410FFF76CFF5EE0FB79022B0CD10521022047
S31508022420FFF7F6FEF860F9680220FEF70FFF0220B2
S31508022430FFF75CFF4EE0FB79032B0CD10521032045
S31508022440FFF7E6FEF860F9680320FEF7FFFE0320B1
S31508022450FFF74CFF3EE0FB79042B0CD10521042043
S31508022460FFF7D6FEF860F9680420FEF7EFFE0420AF
S31508022470FFF73CFF2EE0FB79052B0CD10521052041
S31508022480FFF7C6FEF860F9680520FEF7DFFE0520AD
S31508022490FFF72CFF1EE0FB79062B0CD1052106203F
S315080224A0FFF7B6FEF860F9680620FEF7CFFE0620AB
S315080224B0FFF71CFF0EE0FB79072B0BD1052107203E
S315080224C0FFF7A6FEF860F9680720FEF7BFFE0720A9
S315080224D0FFF70CFF00BF1037BD4680BD80B586B03A
S315080224E000AF0346FB714FF000037B614FF0000318
S315080224F03B614FF00003FB604FF00003BB60FB79C2
S31508022500002B2ED10020FFF729FE07EE900AF8EEDF
S31508022510E77AC7ED047A0020FEF74CFE07EE900A2A
S31508022520F8EEE77AC7ED037A02F09AFF03461846F1
S3150802253002F0E3FF0346184602F0FAFF07EE900A96
S31508022540F8EEE77AC7ED027A02F08AFF0346D7ED7C
S31508022550047AFCEEE77A17EE901A184603F0A9F900
S315080225605CE1FB79012B2ED10120FFF7F7FD07EE7F
S31508022570900AF8EEE77AC7ED047A0120FEF71AFE0A
S3150802258007EE900AF8EEE77AC7ED037A02F068FFDB
S315080225900346184602F0B1FF0346184602F0E3FF67
S315080225A007EE900AF8EEE77AC7ED027A02F058FFCC
S315080225B00346D7ED047AFCEEE77A17EE901A184628
S315080225C003F092F92AE1FB79022B2ED10220FFF7BA
S315080225D0C5FD07EE900AF8EEE77AC7ED047A0220FF
S315080225E0FEF7E8FD07EE900AF8EEE77AC7ED037AFA
S315080225F002F036FF0346184602F07FFF03461846E6
S3150802260002F0CCFF07EE900AF8EEE77AC7ED027AF7
S3150802261002F026FF0346D7ED047AFCEEE77A17EEB8
S31508022620901A184603F07BF9F8E0FB79032B2ED1B2
S315080226300320FFF793FD07EE900AF8EEE77AC7ED57
S31508022640047A0320FEF7B6FD07EE900AF8EEE77A5B
S31508022650C7ED037A02F004FF0346184602F04DFF5F
S315080226600346184602F0B5FF07EE900AF8EEE77A37
S31508022670C7ED027A02F0F4FE0346D7ED047AFCEEC1
S31508022680E77A17EE901A184603F064F9C6E0FB7962
S31508022690042B2ED10420FFF761FD07EE900AF8EE0F
S315080226A0E77AC7ED047A0420FEF784FD07EE900A5E
S315080226B0F8EEE77AC7ED037A02F0D2FE0346184629
S315080226C002F01BFF0346184602F09EFF07EE900A29
S315080226D0F8EEE77AC7ED027A02F0C2FE0346D7EDB4
S315080226E0047AFCEEE77A17EE901A184603F04DF9CB
S315080226F094E0FB79052B2ED10520FFF72FFD07EE77
S31508022700900AF8EEE77AC7ED047A0520FEF752FD3D
S3150802271007EE900AF8EEE77AC7ED037A02F0A0FE12
S315080227200346184602F0E9FE0346184602F087FFFA
S3150802273007EE900AF8EEE77AC7ED027A02F090FE03
S315080227400346D7ED047AFCEEE77A17EE901A184696
S3150802275003F036F962E0FB79062B2ED10620FFF745
S31508022760FDFC07EE900AF8EEE77AC7ED047A062032
S31508022770FEF720FD07EE900AF8EEE77AC7ED037A30
S3150802278002F06EFE0346184602F0B7FE03461846E6
S3150802279002F070FF07EE900AF8EEE77AC7ED027AC2
S315080227A002F05EFE0346D7ED047AFCEEE77A17EEF0
S315080227B0901A184603F01FF930E0FB79072B2DD142
S315080227C00720FFF7CBFC07EE900AF8EEE77AC7ED8B
S315080227D0047A0720FEF7EEFC07EE900AF8EEE77A8F
S315080227E0C7ED037A02F03CFE0346184602F085FE60
S315080227F00346184602F059FF07EE900AF8EEE77A02
S31508022800C7ED027A02F02CFE0346D7ED047AFCEEF7
S31508022810E77A17EE901A184603F008F9D7ED027A06
S31508022820F5EE407AF1EE10FA10D097ED047AD7ED6C
S31508022830037A77EE676A97ED027AC6EE877A9FED94
S31508022840097A67EE877AC7ED057A02E04FF0000348
S315080228507B617B6907EE903AB0EE670A1837BD4688
S3150802286080BD00BF0000484390B585B000AF03465F
S31508022870FB710023FB60FB79002B25D11E2100206A
S31508022880FFF7C6FC04460020FEF794FC0346E31A4B
S31508022890FB6002F0E5FD0346184602F02EFE0346EB
S315080228A0F968184602F035FE02F0DAFD0346012100
S315080228B0184603F0D6F80346002B00F01F81F96884
S315080228C0904804F083F819E1FB79012B25D11E21E2
S315080228D00120FFF79DFC04460120FEF76BFC034628
S315080228E0E31AFB6002F0BCFD0346184602F005FE39
S315080228F00346F968184602F027FE02F0B1FD0346C0
S315080229000121184603F0ADF80346002B00F0F680C5
S31508022910F9687C4804F05AF8F0E0FB79022B25D1D5
S315080229201E210220FFF774FC04460220FEF742FC31
S315080229300346E31AFB6002F093FD0346184602F0CB
S31508022940DCFD0346F968184602F019FE02F088FD16
S3150802295003460121184603F084F80346002B00F0CB
S31508022960CD80F968674804F031F8C7E0FB79032B94
S3150802297025D11E210320FFF74BFC04460320FEF750
S3150802298019FC0346E31AFB6002F06AFD0346184681
S3150802299002F0B3FD0346F968184602F00BFE02F090
S315080229A05FFD03460121184603F05BF80346002B38
S315080229B000F0A480F968534804F008F89EE0FB7911
S315080229C0042B24D11E210420FFF722FC04460420EE
S315080229D0FEF7F0FB0346E31AFB6002F041FD0346ED
S315080229E0184602F08AFD0346F968184602F0FDFD0C
S315080229F002F036FD03460121184603F032F8034673
S31508022A00002B7BD0F9683F4803F0E0FF76E0FB79BC
S31508022A10052B24D11E210520FFF7FAFB04460520C3
S31508022A20FEF7C8FB0346E31AFB6002F019FD0346EC
S31508022A30184602F062FD0346F968184602F0F0FDF0
S31508022A4002F00EFD03460121184603F00AF8034672
S31508022A50002B53D0F9682B4803F0B8FF4EE0FB79F8
S31508022A60062B24D11E210620FFF7D2FB0446062098
S31508022A70FEF7A0FB0346E31AFB6002F0F1FC0346ED
S31508022A80184602F03AFD0346F968184602F0E3FDD5
S31508022A9002F0E6FC03460121184602F0E2FF03466D
S31508022AA0002B2BD0F968174803F090FF26E0FB7934
S31508022AB0072B23D11E210720FFF7AAFB044607206E
S31508022AC0FEF778FB0346E31AFB6002F0C9FC0346ED
S31508022AD0184602F012FD0346F968184602F0D6FDBA
S31508022AE002F0BEFC03460121184602F0BAFF03466D
S31508022AF0002B03D0F968034803F068FF00BF1437B8
S31508022B00BD4690BD249B030880B400AF034B1B68E7
S31508022B101846BD465DF8047B704700BF841E002038
S31508022B2080B500AF4FF400620E490F480FF056F910
S31508022B304FF400620D490E480FF050F94FF4007237
S31508022B400C490D480FF04AF94FF400620B490C483C
S31508022B500FF044F94FF400620A490B480FF03EF9A8
S31508022B6000BF80BD981E0020881E0020A8260020CF
S31508022B7098260020DC2E0020CC2E00201C310020B6
S31508022B80DC3000205C3900201C39002080B483B078
S31508022B9000AF78607B68002B01D1002346E07B6892
S31508022BA0012B01D1012341E07B68022B01D10223CB
S31508022BB03CE07B68032B01D1032337E07B68042BB7
S31508022BC001D1042332E07B68052B01D105232DE0D0
S31508022BD07B68062B01D1062328E07B68072B01D1E7
S31508022BE0072323E07B68082B01D108231EE07B68B4
S31508022BF0092B01D80C2319E07B680A2B01D810236C
S31508022C0014E07B680B2B01D814230FE07B680C2B8E
S31508022C1001D818230AE07B680D2B01D8202305E08A
S31508022C207B680E2B01D8302300E0402318460C3768
S31508022C30BD465DF8047B704780B483B000AF034697
S31508022C40FB80FB88002B01D1002346E0FB88012B81
S31508022C5001D1012341E0FB88022B01D102233CE08A
S31508022C60FB88032B01D1032337E0FB88042B01D110
S31508022C70042332E0FB88052B01D105232DE0FB88CE
S31508022C80062B01D1062328E0FB88072B01D107234F
S31508022C9023E0FB88082B01D108231EE0FB880C2BB6
S31508022CA001D8092319E0FB88102B01D80A2314E05E
S31508022CB0FB88142B01D80B230FE0FB88182B01D8AD
S31508022CC00C230AE0FB88202B01D80D2305E0FB889C
S31508022CD0302B01D80E2300E00F2318460C37BD46C9
S31508022CE05DF8047B7047000084B0B0B400AF07F10A
S31508022CF00C0484E80F00074B1D4607F10C040FCCA1
S31508022D000FC50FCC0FC523682B6000BFBD46B0BCEC
S31508022D1004B07047A82E002080B586B000AF786050
S31508022D200B467B800023FB7500233B610023FB6077
S31508022D300023BB6000F0F6FC0346002B0BD0444B85
S31508022D40D3F844323B61424BD3F8843AFB607B6842
S31508022D501B68BB600AE03E4BD3F844323B613C4BEE
S31508022D60D3F8843AFB607B681B68BB603A69BB6828
S31508022D709A4227D1364B93F86832002B0AD1344B44
S31508022D80D3F850227B881344314AC2F850320123C1
S31508022D90FB7558E02E4BB3F86C321A467B881344FF
S31508022DA0B3F5006F0BDA2A4BB3F86C227B8813440F
S31508022DB09AB2274BA3F86C220123FB7543E0002342
S31508022DC0FB7540E0FA68BB689A4227D1204B93F814
S31508022DD0A83A002B0AD11E4BD3F850227B881344FB
S31508022DE01B4AC2F850320223FB752CE0184BB3F883
S31508022DF0AC3A1A467B881344B3F5006F0BDA144BC8
S31508022E00B3F8AC2A7B8813449AB2114BA3F8AC2ABE
S31508022E100223FB7517E00023FB7514E03B69002BC0
S31508022E2007D1242279680B4813F075F90123FB753B
S31508022E3009E0FB68002B06D124227968064813F0BC
S31508022E406AF90223FB75FB7D18461837BD4680BD15
S31508022E50A82E0020EC3000202C39002080B584B042
S31508022E6000AF03463960FB711346BB800023FB8122
S31508022E70FB79012B12D10023FB810AE0FB893A6810
S31508022E8013440122194612480FF04EF8FB89013302
S31508022E90FB81FA89BB889A42F0D314E0FB79022BAC
S31508022EA011D10023FB810AE0FB893A681344012207
S31508022EB0194608480FF038F8FB890133FB81FA896D
S31508022EC0BB889A42F0D300BF1037BD4680BD00BF0B
S31508022ED0DC3000201C39002080B582B000AF0346E2
S31508022EE0FB71FB1D0122194603480FF01DF800BFAE
S31508022EF00837BD4680BD00BFCC2E0020B0B5B4B0A1
S31508022F0000AFF860B9607A60002387F8CB300023F7
S31508022F1087F8CA30F86804F04EFAC7F8CC000023DE
S31508022F2087F8CB3004E097F8CB30013387F8CB30FB
S31508022F300721F86804F054FB0346002BF3D17A689C
S31508022F40B968F86804F0F3F90346002B3AD097F803
S31508022F50CA30013387F8CA3002F082FA03460121E1
S31508022F60184602F07EFD0346002B02D06A4803F09B
S31508022F702DFD6A4B1B78012B24D0684B01221A704F
S31508022F8007F1C803012118460FF031FF07F1840241
S31508022F9007F1C8031146184610F0F4F910F076FA4C
S31508022FA0044607F1840318460FF081FF054607F128
S31508022FB0840318460FF087FF03461A462946204619
S31508022FC011F004FE97F8CA30002B28D1534B1B7810
S31508022FD0002B24D0514B00221A7007F1C803002196
S31508022FE018460FF004FF07F1840207F1C8031146D9
S31508022FF0184610F0C7F910F049FA044607F1840397
S3150802300018460FF054FF054607F1840318460FF0D9
S315080230105AFF03461A462946204611F0D7FDF86894
S3150802302000F0ECFA03461A463D4B9A60F86800F03F
S31508023030AFFA03463A4A1360F86800F0C1FA034643
S31508023040374A5360364B9B68002B1CD002F008FAAD
S3150802305003460121184602F004FD0346002B12D04E
S315080230602F4B1A682E4B5B6807F110002D4912F098
S3150802307007FF07F11003184603F0A8FC284B9B68C4
S31508023080184600F003FB0C222549274812F07CFF5C
S315080230900346002B36D0224B1B68DAB207F15403DB
S315080230A0114618460FF052FE1D4B5B68DAB207F15D
S315080230B05403114618460FF064FE194B9B68DAB2A0
S315080230C007F15403114618460FF076FE07F110026F
S315080230D007F154031146184610F025F910F0D6F9EF
S315080230E0044607F1100318460FF0E1FE054607F1FC
S315080230F0100318460FF0E7FE03461A4629462046ED
S3150802310011F064FD084B064A07CA83E8070000BFA8
S31508023110D037BD46B0BD00BF489B030874410020A6
S315080231205C4100206C9B03086841002080B592B080
S3150802313000AF3B4640220021184612F035FF002315
S31508023140A7F8423000237B649C480EF0D1FE034662
S3150802315083F00103DBB2002B00F0C480984B93F88E
S315080231606832002B50D1964BD3F850329AB2944B10
S31508023170A3F86C22924B0F22C3F8502210233B70FD
S315080231803B785AB28E4BB3F86C321B0A9BB25BB2CF
S3150802319003F00F035BB213435BB2DBB23B70884B9F
S315080231A0B3F86C32DBB27B703B4602333E221946D9
S315080231B082480EF0F4FE0346002B00F0FC80FFF76F
S315080231C0A3FC3B461A467F49FFF798FE7C4BB3F8A9
S315080231D06C323E3B9AB27A4BA3F86C22784BB3F820
S315080231E06A3201339AB2764BA3F86A22744B0122E9
S315080231F083F86822724BFF2283F86E22704B4FF4D3
S31508023200FA62C3F87022D6E06D4B93F86E32002B41
S3150802321005D06B4B93F86E32012B40F0CC80684B8D
S31508023220B3F86C323E2B02D940237B6404E0644B2C
S31508023230B3F86C3201337B6420233B703B785AB275
S315080232405F4BB3F86A325BB203F00F035BB2134308
S315080232505BB2DBB23B707B6C5A1E3B4601331946A6
S3150802326056480EF09CFE0346002B00F0A4807B6CA9
S315080232709BB21846FFF7E0FC0346514AC2F85032A1
S31508023280FFF742FC3B461A464E49FFF737FE4C4BC0
S31508023290B3F86C227B6C9BB2D31A9BB201339AB2F7
S315080232A0474BA3F86C22464BB3F86A3201339AB2FB
S315080232B0434BA3F86A22424BB3F86C32002B7AD1FD
S315080232C0242200213F4812F06FFE3D4B002283F86C
S315080232D068223B4B0022A3F86A22394BFF2283F865
S315080232E06E2268E038480EF003FE034683F00103B7
S315080232F0DBB2002B5FD03B460122194632480EF05C
S315080233004EFE0346002B53D03B781B09DBB2032B38
S3150802331014D13B460133022219462B480EF03FFED2
S315080233200346002B47D0264B0322DA60FFF7ECFB55
S315080233303B461A462249FFF7E1FD3CE03B781B096A
S31508023340DBB2002B37D13B460133012219461E4810
S315080233500EF025FE0346002B2CD03B781B029BB2AF
S3150802336003F47063A7F842307B781A46B7F84230FE
S315080233701343A7F84230B7F842203B4602331946B0
S3150802338011480EF00CFE0346002B14D0B7F8423053
S3150802339002339BB21846FFF74FFC0346084AD3602E
S315080233A0FFF7B2FB3B461A460549FFF7A7FD02E0BF
S315080233B000BF00E000BF4837BD4680BDDC300020B4
S315080233C0A82E0020EC300020CC2E002080B59AB022
S315080233D000AF3B4668220021184612F0E5FD0E486A
S315080233E00EF086FD034683F00103DBB2002B0ED0F6
S315080233F004E03B466821184600F010F83B4668226E
S31508023400194605480EF0CBFD0346002BF1D100BF45
S315080234106837BD4680BD00BF9826002080B582B0B9
S3150802342000AF78600B467B80786800F0F1FB00BF3E
S315080234300837BD4680BD000080B500AF194B93F82A
S315080234406832002B2BD0174B93F86E32FF2B26D1FE
S31508023450144BD3F87032002B07D0124BD3F87032C4
S31508023460013B104AC2F8703219E0242200210E48A4
S3150802347012F09AFD4FF400620C490D480EF0AEFCAC
S31508023480084B002283F86822064B0022A3F86A2218
S31508023490044BFF2283F86E22064803F097FA00BF10
S315080234A080BD00BFA82E0020EC3000201C31002071
S315080234B0DC300020909B030880B582B000AF7860AC
S315080234C00B467B80786800F0B1FA00BF0837BD4624
S315080234D080BD000080B582B000AF78600B467B8065
S315080234E07B881A46796803480EF01EFD00BF083726
S315080234F0BD4680BD881E002080B59AB000AF3B4607
S3150802350068220021184612F04FFD0E480EF0F0FC14
S31508023510034683F00103DBB2002B0ED004E03B46E0
S3150802352068211846FFF7C8FF3B4668221946054830
S315080235300EF035FD0346002BF1D100BF6837BD46B4
S3150802354080BD00BF881E002080B582B000AF7860BB
S315080235500B4A7B681360FFF7E3FA24220021094825
S3150802356012F022FD24220021074812F01DFD242212
S315080235700021064812F018FD00BF0837BD4680BD77
S31508023580841E0020A82E0020EC3000202C390020B2
S3150802359080B485B000AF78607B681B681B6CBB6023
S315080235A00023FB60BB68DBB2002B02D0BB68DBB230
S315080235B0FB60FB6818461437BD465DF8047B704706
S315080235C080B485B000AF78607B681B681B6CBB60F3
S315080235D00023FB60BB6803F4FE43002B06D0BB68DE
S315080235E003F4FE43FB60FB681B0AFB60FB68184694
S315080235F01437BD465DF8047B7047000080B485B079
S3150802360000AF78607B681B685B6CBB600023FB605D
S31508023610BB6803F00703002B2FD0BB6803F0070330
S31508023620013B052B20D801A252F823F045360208A1
S315080236304B36020851360208573602085D3602082A
S31508023640633602080123FB600FE00223FB600CE0ED
S315080236500323FB6009E00423FB6006E00523FB6005
S3150802366003E00623FB6000E000BF7B681B685A6C18
S315080236707B681B6822F007025A64FB68DBB21846AD
S315080236801437BD465DF8047B704700BF80B582B02B
S3150802369000AF786001F0E4FE03460121184602F005
S315080236A0E0F9034683F00103DBB2002B2AD17B68DB
S315080236B0013B052B27D801A252F823F0D53602087A
S315080236C0DD360208E5360208ED360208F536020846
S315080236D0FD3602080D4803F079F914E00C4803F0A8
S315080236E075F910E00B4803F071F90CE00A4803F08B
S315080236F06DF908E0094803F069F904E0084803F09F
S3150802370065F900E000BF0837BD4680BDA09B0308E7
S31508023710B09B0308C09B0308D89B0308F09B0308C9
S31508023720089C030880B400AF034B1B781846BD46B5
S315080237305DF8047B704700BF8C05002080B500AF9A
S31508023740FFF7F0FF0346002B02D04FF4807301E027
S315080237504FF48073184680BD80B500AFFFF7E2FFCD
S315080237600346002B02D04FF4803300E000231846AC
S3150802377080BD80B500AFFFF7D5FF0346002B02D008
S315080237804FF4847300E00023184680BDB0B5A4B098
S3150802379006AFF860B9601346FB800023A7F87630B7
S315080237A0FB683B65FFF7BEFF0346002B03D04FF0CD
S315080237B080437B6501E000237B650023BB65FB88AC
S315080237C002339BB21846FFF737FA0346FB65002316
S315080237D03B664FF480137B664FF40013BB660023E7
S315080237E0FB6600233B6700233B743B7C5AB2FB888B
S315080237F01B0A9BB25BB203F00F035BB213435BB2C5
S31508023800DBB23B74FB88DBB27B740223A7F8763003
S3150802381010E0B7F87630023BBA681A44B7F8763041
S31508023820127878333B4403F8682CB7F876300133BC
S31508023830A7F87630B7F87620FB8801339A42E8DD96
S315080238400023A7F876300DE0B7F8763078333B4494
S3150802385013F8683C1846FFF73FFBB7F87630013392
S31508023860A7F87630B7F87620FB8801339A42EBDD63
S315080238706D4607F160040FCC0FC523682B6007F16C
S3150802388050030FCBFFF730FA00BF7837BD46B0BDFD
S3150802389080B58EB000AFF860B9601346FB8000238E
S315080238A087F83730FB683B61FFF73CFF0346002B7E
S315080238B003D04FF080437B6101E000237B61002344
S315080238C0BB61FB88FB6100233B624FF480137B627A
S315080238D04FF40013BB620023FB6200233B63FA88A2
S315080238E007F1100311461846FFF716FA034687F83A
S315080238F0373097F83730002B06D0FA8897F83730E2
S31508023900B9681846FFF7AAFA00BF3837BD4680BD20
S31508023910B0B5A2B006AF7860084611461A46034605
S31508023920FB700B46BB7013467B70002387F86F301B
S315080239307B68BB64FFF7F6FE0346002B03D04FF005
S315080239408043FB6401E00023FB6400233B650323F9
S315080239507B650023BB654FF48013FB654FF40013A8
S315080239603B6600237B660023BB6630233B723B7AA9
S315080239705AB297F9033003F00F035BB213435BB2F3
S31508023980DBB23B72BB787B727B78BB72002387F80B
S315080239906F300DE097F86F3070333B4413F8683C8C
S315080239A01846FFF799FA97F86F30013387F86F30A0
S315080239B097F86F30022BEDD96D4607F158040FCCF4
S315080239C00FC523682B6007F148030FCBFFF78CF965
S315080239D000BF7037BD46B0BD80B582B000AF786013
S315080239E00023002200217868FFF792FF00BF0837FC
S315080239F0BD4680BD80B584B000AFF860B960134695
S31508023A00FB80FB883E2B06D8FB881A46B968F868FD
S31508023A10FFF7BCFE05E0FB881A46B968F868FFF7A7
S31508023A2037FF00BF1037BD4680BD000080B588B09D
S31508023A3000AF7860FF23FB7600237B610023FB61DE
S31508023A4000237B827B68FB60FB6893F828301B099E
S31508023A50FB76FB681B687B61FFF77EFE02467B6985
S31508023A60934202D1FFF785FEF861FB7E032B00F233
S31508023A70B98001A252F823F0893A0208CB3A020821
S31508023A802D3B0208813B0208FB6893F8283003F0B5
S31508023A900F039AB2554B1A80544B1B881B029AB2D3
S31508023AA0524B1A80FB6893F829301A464F4B1B88EB
S31508023AB013439AB24D4B1A80FB682A334B4A128833
S31508023AC01146184600F0F2FB8CE0FB6893F82830A2
S31508023AD003F00F039AB2454B1A80444B1B881B020C
S31508023AE09AB2424B1A80FB6893F829301A463F4B22
S31508023AF01B8813439AB23D4B1A803D4B01221A701A
S31508023B003C4B1B78002B04D03B4802F05FFF00F0C9
S31508023B10DFFBFB682A333E21184600F0C7FBF8692B
S31508023B20FFF75AFF334B01221A705BE0314B002232
S31508023B301A702F4B1B781A46FB6893F8283003F045
S31508023B400F039A424BD1FB68DB681846FFF71EF84B
S31508023B500346013B7B82FB6829337A8A114618465B
S31508023B6000F0A4FB224B1B780133DAB2204B1A7001
S31508023B701F4B1B780F2B32D91D4B00221A702EE0D1
S31508023B801E4BD3F84432FA699A4212D1FB6893F86B
S31508023B90283003F00F03DAB2184B83F86E22FB685B
S31508023BA093F82920154B83F86F22154802F00EFF69
S31508023BB017E0124BD3F8843AFA699A4211D1FB6894
S31508023BC093F8283003F00F03DAB20C4B83F8AE2AC7
S31508023BD0FB6893F82920094B83F8AF2A01E000BF56
S31508023BE000E000BF00BF2037BD4680BD76410020F9
S31508023BF07841002079410020149C0308A82E002051
S31508023C00209C030880B500AF10F028FB00BF80BDDA
S31508023C1080B584B000AF78607B68FB60FFF782FDF1
S31508023C200346002B0AD0FB681B68B3F5806F10D1D8
S31508023C30FB6893F82830002B0BD10AE0FB681B6857
S31508023C40B3F5806F05D1FB6893F82830002B00D1B5
S31508023C5000BF00BF1037BD4680BD000080B500AF6B
S31508023C604022034903480EF0B9F80123184680BDDD
S31508023C708C4100207C41002080B500AF05480EF03B
S31508023C8037F90346002B01D0012300E0002318462A
S31508023C9080BD00BF7C41002080B582B000AF78604D
S31508023CA00B46FB70FB781A46796804480EF0ABFAA5
S31508023CB0012318460837BD4680BD00BF7C41002057
S31508023CC080B584B000AF78600023FB737968054835
S31508023CD00EF0AAFA0346FB73FB7B18461037BD465D
S31508023CE080BD00BF7C41002090B593B000AF002391
S31508023CF087F84730FFF7C0FF0346002B40F0C6811E
S31508023D0001F0AEFB03460121184601F0AAFE03465E
S31508023D10002B02D0BE4802F059FE3B1D402200216C
S31508023D20184612F041F93B1D1846FFF7C9FF03462C
S31508023D3087F847303B79012B40F0A88197F847303E
S31508023D40002B00F0A3817B79082B17DC022BC0F22B
S31508023D509681023B062B00F2928101A252F823F0C9
S31508023D60973D02087F400208233F0208093E0208DF
S31508023D70F93E02087F40020839400208FF2B40F04C
S31508023D807E81A44802F022FE01F06AFB0346184629
S31508023D9001F08AFB7AE13B1D02339F4918460FF070
S31508023DA0F1F99D480EF0C7FE034619469B4802F0F4
S31508023DB00DFE99480EF0BFFE0346012B07D101F00E
S31508023DC04FFB03460121184601F088FB0CE0924896
S31508023DD00EF0B1FE0346022B06D101F041FB034663
S31508023DE00021184601F07AFB10F072F903461846CC
S31508023DF010F084F9044688480EF09DFE03461946DB
S31508023E0020460EF0BDFC41E13B1D023384491846AB
S31508023E100FF00FFA82480EF0D0FE03461946814883
S31508023E2002F0D4FD10F054F90346184610F066F96C
S31508023E300346142118460EF045FC00F0D9FA7848D4
S31508023E400EF0BBFE0346012B03D10020FEF7BCFA97
S31508023E5044E073480EF0B1FE0346022B03D101205B
S31508023E60FEF7B2FA3AE06E480EF0A7FE0346032BB7
S31508023E7003D10220FEF7A8FA30E069480EF09DFE4B
S31508023E800346042B03D10320FEF79EFA26E0644874
S31508023E900EF093FE0346052B03D10420FEF794FA8F
S31508023EA01CE05F480EF089FE0346062B03D1052067
S31508023EB0FEF78AFA12E05A480EF07FFE0346072BEF
S31508023EC003D10620FEF780FA08E055480EF075FE83
S31508023ED00346082B02D10720FEF776FA00F088FA85
S31508023EE010F0F6F80346184610F008F903461521AD
S31508023EF018460EF0E7FBC9E03B1D02334A4918464D
S31508023F000FF05FFA48480EF081FF03461C46464802
S31508023F100EF097FF03461A462146444802F056FD1C
S31508023F20B4E03B1D0233424918460FF066F9404891
S31508023F300EF028FE034619463E4802F047FD10F0E9
S31508023F40C7F80346184610F0D9F80346162118464C
S31508023F500EF0B8FB36480EF015FE0346012B03D1C8
S31508023F600020FEF781FC44E031480EF00BFE0346C2
S31508023F70022B03D10120FEF777FC3AE02C480EF01B
S31508023F8001FE0346032B03D10220FEF76DFC30E047
S31508023F9027480EF0F7FD0346042B03D10320FEF74C
S31508023FA063FC26E022480EF0EDFD0346052B03D1FD
S31508023FB00420FEF759FC1CE01D480EF0E3FD0346FB
S31508023FC0062B03D10520FEF74FFC12E018480EF027
S31508023FD0D9FD0346072B03D10620FEF745FC08E068
S31508023FE013480EF0CFFD0346082B02D10720FEF731
S31508023FF03BFCFDF7A5F810F06BF80346184610F0DF
S315080240007DF80346172118460EF05CFB3EE000BF1A
S315080240102C9C0308589C0308CC410020749C030876
S31508024020D4410020C09C0308D8410020149D0308EF
S31508024030D04100206C9D03083B1D023315491846E2
S315080240400FF0E6F913480EF017FF03461946124811
S3150802405002F0BCFC0F480EF00FFF0346002B14D1EA
S3150802406010F036F80346184610F048F803460021C1
S3150802407018460EF042FB094802F0A8FC05E07B79D7
S315080240801946074802F0A2FC00E000BF00BF4C3701
S31508024090BD4690BDDC410020BC9D0308009E030876
S315080240A0209E030880B582B000AF78600B467B80FD
S315080240B009480DF0BFFE02467B889A4207D37B88E1
S315080240C01A46796804480EF09EF8012300E0002398
S315080240D018460837BD4680BDE041002080B5C4B009
S315080240E000AF024607F58873A3F209131A70002374
S315080240F087F80F3123E007F10C034FF48072002191
S31508024100184611F051FF07F10C03194615480EF02F
S31508024110F1F8034687F80F3107F10C0319461148DF
S315080241200EF082F8034687F80F31FFF722FB97F85D
S315080241300F319AB207F10C031946FFF75BFC0948DF
S315080241400DF0D6FE034683F00103DBB2002B03D043
S31508024150054B1B78002BCED000BF07F58877BD46E6
S3150802416080BD00BFE0410020F041002080B483B04A
S3150802417000AF78600B467B8000BF00BF0C37BD4698
S315080241805DF8047B7047000080B582B000AF00235B
S31508024190FB712A4B1B78002B48D0294B1B7801331D
S315080241A0DAB2274B1A70264B1B78092B41D9244BB6
S315080241B000221A70214B5B78012B17D81F4B5B78AC
S315080241C00133DAB21D4B5A70FFF7D3FA03461B4A7C
S315080241D092F883201B491846FFF70CFC01F040F9B8
S315080241E003460121184601F03CFC22E001F038F9A9
S315080241F003460121184601F034FC0346002B0BD076
S315080242000023FB7102E0FB790133FB710B4B93F838
S315080242108330FA799A42F6D30A490B480EF004F823
S3150802422084220021054811F0BFFE02E0044B002259
S315080242301A7000BF0837BD4680BD00BFF041002096
S3150802424074420020F3410020E041002080B582B08C
S3150802425000AF786039603968786800F04BF800BFBB
S315080242600837BD4680BD80B582B000AF7860396038
S315080242703B689BB219467868FFF714FF00BF0837F8
S31508024280BD4680BD80B582B000AF78603960064B06
S315080242901B683A6892B2796818460DF099FB00BF16
S315080242A00837BD4680BD00BF9005002080B582B0A4
S315080242B000AF78603960054B1B683A68796818461A
S315080242C00DF020FC00BF0837BD4680BD90050020D2
S315080242D080B500AF044B1868044B054A00210DF05F
S315080242E03CFB00BF80BD00BF900500206742020864
S315080242F04D42020890B583B000AF786039603B68DA
S315080243009BB219467868FFF731FF7B681B780F2B3B
S3150802431023D00F2B48DC012B02D0052B31D043E0EA
S31508024320244B9B78194624480FF05DFA214BDB781B
S31508024330194621480FF073FA20491F480FF0E1F990
S315080243401E480FF02CFA04461C480FF034FA0346AE
S3150802435019462046FFF796FF27E0194B01221A70E5
S31508024360164917480FF0F0F914480FF018FA0446E0
S3150802437012480FF020FA034619462046FFF782FF35
S3150802438013E0104802F022FB0C480FF0F6F90B482E
S315080243900FF005FA044609480FF00DFA03461946C6
S315080243A02046FFF76FFF00E000BF00BF0C37BD468F
S315080243B090BD00BFE0BF1F08AC530020A4520020E6
S315080243C0A85300204C9E030880B500AF03480BF0A3
S315080243D025FA02480BF0E2F800BF80BD74540020AB
S315080243E080B500AF00F0EAF902F0E0FA00BF80BD3E
S315080243F080B500AF01F034F80346184601F048F8D4
S315080244000346002B02D1024804F0FEF900BF80BD24
S315080244101454002080B582B000AF3E4B3E4A9A60E3
S3150802442062B600BF02F078FB00F09EF800F012FABE
S3150802443000F004F900F04AF900F06AF900F0BEF952
S3150802444000F06EF935480AF04BFA02F0AFFA344832
S31508024450FFF77AF800F0C0FCFFF73AFF10F034FBDA
S31508024460FFF7FCFBFCF72CFE0346FB71FDF76CFD20
S31508024470FB79002B47D02B4802F0A8FA0020FDF75B
S31508024480A3FF294802F0A2FA284802F09FFA01205F
S31508024490FDF79AFF264802F099FA264802F096FA9C
S315080244A00220FDF791FF244802F090FA234802F011
S315080244B08DFA0320FDF788FF214802F087FA214882
S315080244C002F084FA0420FDF77FFF1F4802F07EFA05
S315080244D01E4802F07BFA0520FDF776FF1C4802F01B
S315080244E075FA1C4802F072FA0620FDF76DFF1A48A3
S315080244F002F06CFA194802F069FA0720FDF764FF20
S31508024500174802F063FA174802F060FA01F0B4FCA1
S31508024510FCE700BF00ED00E0000002082854002076
S31508024520B0530020689E0308889E0308A89E0308C5
S31508024530C89E0308E89E0308089F0308289F0308E5
S31508024540489F0308689F0308889F0308A89F0308D3
S31508024550C89F0308E89F030808A0030828A00308C1
S3150802456048A0030868A0030880B59CB000AF07F10D
S31508024570200350220021184611F016FD07F1080300
S3150802458000221A605A609A60DA601A615A612A4BE6
S315080245901B69294A43F030031361274B1B6903F051
S315080245A030037B607B6800BF234B5B6903F008031B
S315080245B0082BF9D109233B624FF480337B624FF013
S315080245C08063BB630223BB640323FB6403233B654B
S315080245D07D237B650223BB650223FB6502233B66BB
S315080245E008237B660023BB660023FB6607F12003CC
S315080245F0184604F019F90346002B01D000F0A6FA72
S315080246001F23BB600323FB6000233B6100237B61FE
S315080246100023BB610023FB6107F108030521184645
S3150802462004F03AFD0346002B01D000F08FFA00BFD2
S315080246307037BD4680BD00BF0008024480B500AF92
S31508024640204B214A1A601F4B00225A601D4B4FF419
S3150802465040729A601B4B0022DA601A4B00221A74C7
S31508024660184B00225A74174B00229A74154B0522CE
S315080246705A61144B0A229A61124B2722DA61114BAC
S315080246800A221A620F4B05225A620E4B02229A62BC
S315080246900C4B0722DA620B4B02221A63094B0122E0
S315080246A05A63084B01229A63064B0022DA630548CD
S315080246B002F030FC0346002B01D000F047FA00BF97
S315080246C080BD00BFB053002000A4004080B500AFF3
S315080246D00D4B0E4A1A600C4B05225A600A4B40F2E1
S315080246E0EE22DA60084B40F2EE229A60064B00226E
S315080246F01A61054804F000F80346002B01D000F0C1
S3150802470025FA00BF80BD00BF1454002000300040C7
S3150802471080B400AF00BFBD465DF8047B7047000059
S3150802472080B588B000AF07F1100300221A605A60FC
S315080247309A60DA603B1D00221A605A609A601E4B24
S315080247404FF080421A601C4B40F6C3125A601A4B4D
S3150802475000229A60184B6322DA60174B00221A610C
S31508024760154B00229A6114480AF062F80346002B98
S3150802477001D000F0EBF94FF480533B6107F11003C7
S3150802478019460D480AF0A4FA0346002B01D000F098
S31508024790DDF900237B600023FB603B1D19460648B2
S315080247A00AF096FD0346002B01D000F0CFF900BFB0
S315080247B02037BD4680BD00BF2854002080B500AF13
S315080247C0224B234A1A60214B4FF4E1325A601F4B9F
S315080247D000229A601D4B0022DA601C4B00221A61E5
S315080247E01A4B0C225A61194B00229A61174B002266
S315080247F0DA61164B00221A62144B00225A62134BD4
S3150802480000229A6211480AF079FE0346002B01D06B
S3150802481000F09CF900210D480CF0E9FE0346002B36
S3150802482001D000F093F9002108480CF01EFF034658
S31508024830002B01D000F08AF904480CF09FFE0346CB
S31508024840002B01D000F082F900BF80BD745400200D
S315080248500038014080B58EB000AF07F1240300226C
S315080248601A605A609A60DA601A61A44BD3F88C30DF
S31508024870A24A43F02003C2F88C30A04BD3F88C30FE
S3150802488003F020033B623B6A9C4BD3F88C309B4A6D
S3150802489043F08003C2F88C30984BD3F88C3003F07F
S315080248A08003FB61FB69954BD3F88C30934A43F03E
S315080248B00403C2F88C30914BD3F88C3003F004030E
S315080248C0BB61BB698D4BD3F88C308C4A43F04003ED
S315080248D0C2F88C30894BD3F88C3003F040037B61E5
S315080248E07B69864BD3F88C30844A43F01003C2F8AE
S315080248F08C30824BD3F88C3003F010033B613B6952
S315080249007E4BD3F88C307D4A43F00803C2F88C30CC
S315080249107A4BD3F88C3003F00803FB60FB68774BBD
S31508024920D3F88C30754A43F00103C2F88C30734BC6
S31508024930D3F88C3003F00103BB60BB686F4BD3F826
S315080249408C306E4A43F00203C2F88C306B4BD3F8B4
S315080249508C3003F002037B607B6800224FF481717E
S31508024960674803F097FE00222021664803F092FE6C
S31508024970002240F62101644803F08CFE00224FF41F
S315080249800051624803F086FE00224FF40071604827
S3150802499003F080FE002240215E4803F07BFE81235D
S315080249A07B620023BB620023FB6207F124031946DC
S315080249B0534803F049FC4FF481737B620123BB62BF
S315080249C00023FB6203233B6307F1240319464C4881
S315080249D003F03AFC10237B620023BB620023FB62CE
S315080249E007F124031946474803F02EFC20237B626D
S315080249F00123BB620023FB6203233B6307F1240303
S31508024A001946404803F020FC40F621037B62012345
S31508024A10BB620023FB6203233B6307F124031946A7
S31508024A20394803F011FC4FF480537B620023BB62C2
S31508024A300023FB6207F124031946344803F004FCF9
S31508024A404FF400537B620123BB620023FB620323FC
S31508024A503B6307F1240319462C4803F0F5FB4FF490
S31508024A6080737B620023BB620023FB6207F1240387
S31508024A701946274803F0E8FB4FF400737B620123CB
S31508024A80BB620023FB6203233B6307F12403194637
S31508024A901F4803F0D9FB4FF482637B620023BB6293
S31508024AA00023FB6207F124031946174803F0CCFBDF
S31508024AB020237B620023BB620023FB6207F12403E7
S31508024AC01946144803F0C0FB40237B620123BB62EC
S31508024AD00023FB6203233B6307F1240319460D48AF
S31508024AE003F0B2FB0C4BD3F800310B4A43F4803384
S31508024AF0C2F8003100BF3837BD4680BD000C0244FB
S31508024B000014024200080242001802420010024241
S31508024B10000C0242000402420004004480B582B03E
S31508024B2000AF78607B681B68074A934201D102F09E
S31508024B3019F87B681B68B3F1804F01D101F0A0F820
S31508024B4000BF0837BD4680BD0010004080B400AFE4
S31508024B5072B600BF00BFFDE7B0B596B000AF786089
S31508024B60396000237B6548E0654B664A40217868D0
S31508024B7002F02EFC0346002B0DD000F071FC034612
S31508024B800121184600F06DFF0346002B35D05E481A
S31508024B9001F01CFF31E0FEF7C5FD0346002B03D0EA
S31508024BA0584B1B687B6502E0564B1B687B65796D23
S31508024BB0564801F00BFFFEF7CFFD02467B6D934286
S31508024BC004D168214F48FEF785FC16E00EF03CFC3E
S31508024BD002467B6D934205D00EF044FC02467B6D7D
S31508024BE093420AD1474BDB681846FDF7CFFF0346C7
S31508024BF01A464349786D0FF0B1FF4021786802F0F2
S31508024C0005FD0346002BAFD17868FEF7F7FC03468D
S31508024C101A463F4B9A607868FEF7BAFC03463C4A46
S31508024C2013607868FEF7CCFC0346394A5360384B62
S31508024C309B68002B1CD000F013FC03460121184682
S31508024C4000F00FFF0346002B12D0314B1A68304B87
S31508024C505B6807F10C002F4911F012F907F10C03F2
S31508024C60184601F0B3FE2A4B9B681846FEF70EFD5E
S31508024C700C222749284811F087F90346002B36D01B
S31508024C80234B1B68DAB207F15003114618460DF09A
S31508024C90A0FB1F4B5B68DAB207F1500311461846B0
S31508024CA00DF0B2FB1A4B9B68DAB207F150031146B4
S31508024CB018460DF0C4FB07F10C0207F15003114622
S31508024CC018460DF082FC0EF0E1FB044607F10C03D0
S31508024CD018460DF0C3FB054607F10C0318460DF0FE
S31508024CE0C9FB03461A46294620460FF06FFF0A4BB0
S31508024CF0074A07CA83E8070000BF5837BD46B0BD52
S31508024D00305500200855002094A00308B4A00308D3
S31508024D105C410020D4A003086841002080B58AB00F
S31508024D2002AF78600B467B8013463B800023BB604C
S31508024D300023FB607B683B6101237B617B88BB6147
S31508024D403B88FB6107F108031946074802F03CFA5B
S31508024D5001230093012302220221034802F08EFA5C
S31508024D6000BF2037BD4680BDB053002080B58CB049
S31508024D7002AFF860B9607A604FF080433B61002366
S31508024D807B61FB68BB610123FB61BB683B627B6895
S31508024D907B6207F110031946074802F015FA012348
S31508024DA00093012302220221034802F067FA00BF98
S31508024DB02837BD4680BD00BFB053002080B500AF7E
S31508024DC0044802F08CFA00220121024802F03CFC57
S31508024DD000BF80BDB053002080B500AFFEF7A2FC2D
S31508024DE00346002B09D0FEF7B7FC03461A466FF0B6
S31508024DF060410220FFF7BAFF09E0FEF7ADFC034661
S31508024E009BB21A464FF6FF710220FFF787FFFFF79C
S31508024E10D5FF00BF80BD000080B58EB000AFF86038
S31508024E20B9601346FB80FB88002B02D0FB88402B17
S31508024E3001D900232FE007F1140324220021184682
S31508024E4011F0B2F8FB687B61FEF76CFC0346002B97
S31508024E5003D04FF08043BB6101E00023BB6100230E
S31508024E60FB61FB881846FDF7E7FE03463B62002313
S31508024E707B624FF48013BB624FF40013FB6200237C
S31508024E803B6300237B6307F11403BA681946044897
S31508024E90FEF734F8012318463837BD4680BD00BFF1
S31508024EA0B053002080B400AF00BFBD465DF8047B56
S31508024EB07047000080B5CCB000AF07F59873A3F52C
S31508024EC09673186007F58E7300221A605A609A6004
S31508024ED0DA601A6107F59873A3F5907318464FF4CA
S31508024EE084731A46002111F05FF807F59873A3F543
S31508024EF096731B681B68384A934267D107F59873FD
S31508024F00A3F590714FF000024FF00403C1E90023A4
S31508024F1007F59873A3F590734FF48072C3F8BC2013
S31508024F2007F11003184604F031FC0346002B01D0A2
S31508024F30FFF70CFE294BD3F8A030284A43F4007336
S31508024F40C2F8A030254BD3F8A03003F4007207F557
S31508024F509873A3F592731A6007F59873A3F592737B
S31508024F601B681E4BD3F88C301C4A43F00103C2F867
S31508024F708C301A4BD3F88C3003F0010207F598737C
S31508024F80A3F594731A6007F59873A3F594731B68CF
S31508024F904FF4C053C7F81C310223C7F82031002347
S31508024FA0C7F824310323C7F828310923C7F82C3157
S31508024FB007F58E7319460A4803F046F900220021BE
S31508024FC0272001F0CBFE272001F0E2FE00BF07F5FD
S31508024FD09877BD4680BD00BF00A40040000C02447D
S31508024FE00000024280B584B000AF78607B681B6817
S31508024FF0B3F1804F16D10D4BD3F89C300B4A43F0D0
S315080250000103C2F89C30094BD3F89C3003F0010324
S31508025010FB60FB68002200212D2001F09FFE2D2057
S3150802502001F0B6FE00BF1037BD4680BD000C024433
S3150802503080B5CCB000AF07F59873A3F596731860E0
S3150802504007F58E7300221A605A609A60DA601A614E
S3150802505007F59873A3F5907318464FF484731A46A6
S31508025060002110F0A1FF07F59873A3F596731B6844
S315080250701B68374A934265D107F59873A3F5907171
S315080250804FF001024FF00003C1E9002307F59873B8
S31508025090A3F590730022DA6507F11003184604F0A7
S315080250A075FB0346002B01D0FFF750FD294BD3F8B9
S315080250B0A430284A43F48043C2F8A430254BD3F8D7
S315080250C0A43003F4804207F59873A3F592731A6025
S315080250D007F59873A3F592731B681E4BD3F88C30A9
S315080250E01C4A43F00103C2F88C301A4BD3F88C30B1
S315080250F003F0010207F59873A3F594731A6007F58E
S315080251009873A3F594731B684FF4C063C7F81C31F0
S315080251100223C7F820310023C7F824310323C7F82E
S3150802512028310723C7F82C3107F58E7319460A4822
S3150802513003F08AF8002200213A2001F00FFE3A20F5
S3150802514001F026FE00BF07F59877BD4680BD00BF71
S3150802515000380140000C02440000024280B582B0C9
S3150802516000AF78607B681B680B4A93420FD10B4BE2
S31508025170D3F8A430094A23F48043C2F8A4304FF482
S31508025180C061074803F0B2F93A2001F00FFE00BFEA
S315080251900837BD4680BD00BF00380140000C0244F6
S315080251A00000024280B58EB000AF7860334BD3F868
S315080251B09C30324A43F01003C2F89C302F4BD3F886
S315080251C09C3003F01003BB60BB6807F10C0207F1C1
S315080251D010031146184604F0A1FAFB69FB62FB6A42
S315080251E0002B03D104F058FA786304E004F054FA69
S315080251F003465B007B637B6B5B09214AA2FB0323A5
S31508025200DB09013BBB621F4B1F4A1A601D4B632217
S31508025210DA601C4ABB6A53601A4B00221A61194BA0
S3150802522000229A60174809F003FB034687F83330D1
S3150802523097F83330002B18D1124809F051FB034670
S3150802524087F8333097F83330002B0ED17B680F2B53
S3150802525008D800227968312001F080FD0B4A7B6864
S31508025260136002E0012387F83330312001F090FD04
S3150802527097F8333018463837BD4680BD000C0244CD
S31508025280C55A7C0A70550020001000409805002077
S3150802529080B400AF00BFFDE780B400AF00BFFDE7F2
S315080252A080B400AF00BFFDE780B400AF00BFFDE7E2
S315080252B080B400AF00BFFDE780B400AF00BFBD46B3
S315080252C05DF8047B704780B400AF00BFBD465DF849
S315080252D0047B704780B400AF00BFBD465DF8047B0F
S315080252E0704780B400AF00BFBD465DF8047B7047C7
S315080252F080B500AF024802F08DFA00BF80BD00BF3C
S31508025300B053002080B500AF024809F097FB00BFF2
S3150802531080BD00BF2854002080B500AF024809F0BE
S315080253208DFB00BF80BD00BF7055002080B500AF61
S3150802533002480AF027FB00BF80BD00BF7454002054
S3150802534080B400AF01231846BD465DF8047B70475A
S3150802535080B582B000AF7860396010F099FE0346D6
S3150802536016221A604FF0FF3318460837BD4680BD2D
S3150802537080B582B000AF78604FF0FF317868FFF7EA
S31508025380E7FF00BFFDE780B586B000AFF860B960F9
S315080253907A6000237B610AE0AFF300800146BB68AE
S315080253A05A1CBA60CAB21A707B6901337B617A6980
S315080253B07B689A42F0DB7B6818461837BD4680BD83
S315080253C080B586B000AFF860B9607A6000237B6169
S315080253D009E0BB685A1CBA601B781846AFF300800E
S315080253E07B6901337B617A697B689A42F1DB7B6868
S315080253F018461837BD4680BD80B483B000AF7860C2
S315080254004FF0FF3318460C37BD465DF8047B7047EC
S3150802541080B483B000AF786039603B684FF40052BD
S315080254205A60002318460C37BD465DF8047B704760
S3150802543080B483B000AF7860012318460C37BD46A6
S315080254405DF8047B704780B485B000AFF860B96038
S315080254507A60002318461437BD465DF8047B704708
S3150802546080B500AF084B1B78DBB2002B09D1064B7F
S3150802547001221A706C220021044810F095FD0EF0E4
S3150802548019F9024B184680BD28560020BC55002043
S3150802549080B483B000AF78607B681B7818460C37F7
S315080254A0BD465DF8047B704780B483B000AF786070
S315080254B07B6801221A70012318460C37BD465DF82F
S315080254C0047B704780B483B000AF78607B685B78F2
S315080254D018460C37BD465DF8047B704780B483B026
S315080254E000AF78600B46FB707B68FA785A7000BF8B
S315080254F00C37BD465DF8047B704780B483B000AFB5
S3150802550078607B68043318460C37BD465DF8047B21
S31508025510704780B483B000AF786039607B683A68B8
S315080255205A60012318460C37BD465DF8047B70475E
S3150802553080B483B000AF78607B685B6818460C3726
S31508025540BD465DF8047B704780B483B000AF7860CF
S3150802555039607B683A689A60012318460C37BD465B
S315080255605DF8047B704780B483B000AF78607B68CF
S315080255709B6818460C37BD465DF8047B704780B4B5
S3150802558083B000AF786039607B683A68DA600123D5
S3150802559018460C37BD465DF8047B704780B483B065
S315080255A000AF78607B68DB6818460C37BD465DF845
S315080255B0047B704780B483B000AF786039607B683B
S315080255C03A681A61012318460C37BD465DF8047B12
S315080255D0704780B483B000AF78607B681B69184651
S315080255E00C37BD465DF8047B704780B483B000AFC4
S315080255F0786039607B683A685A61012318460C3725
S31508025600BD465DF8047B704780B483B000AF78600E
S315080256107B685B6918460C37BD465DF8047B7047A4
S3150802562080B483B000AF786039607B683A689A6163
S31508025630012318460C37BD465DF8047B704780B4D3
S3150802564083B000AF78607B689B6918460C37BD4605
S315080256505DF8047B704780B483B000AF7860396028
S315080256607B683A68DA61012318460C37BD465DF84D
S31508025670047B704780B483B000AF78607B68DB69CF
S3150802568018460C37BD465DF8047B704780B483B074
S3150802569000AF786039607B683A681A620123184657
S315080256A00C37BD465DF8047B704780B483B000AF03
S315080256B078607B681B6A18460C37BD465DF8047B22
S315080256C0704780B483B000AF786087ED000A7B68C4
S315080256D03A689A62012318460C37BD465DF8047B80
S315080256E0704780B483B000AF78607B689B6A07EE28
S315080256F0903AB0EE670A0C37BD465DF8047B7047F0
S3150802570080B483B000AF786087ED000A7B683A6898
S31508025710DA62012318460C37BD465DF8047B7047EA
S3150802572080B483B000AF78607B68DB6A07EE903A94
S31508025730B0EE670A0C37BD465DF8047B704780B445
S3150802574083B000AF786087ED000A7B683A681A630F
S31508025750012318460C37BD465DF8047B704780B4B2
S3150802576083B000AF78607B681B6B07EE903AB0EEA9
S31508025770670A0C37BD465DF8047B704780B483B070
S3150802578000AF786087ED000A7B683A685A6301239E
S3150802579018460C37BD465DF8047B704780B483B063
S315080257A000AF78607B685B6B07EE903AB0EE670AEB
S315080257B00C37BD465DF8047B704780B483B000AFF2
S315080257C0786087ED000A7B683A689A63012318466F
S315080257D00C37BD465DF8047B704780B483B000AFD2
S315080257E078607B689B6B07EE903AB0EE670A0C37D7
S315080257F0BD465DF8047B704780B483B000AF78601D
S3150802580087ED000A7B683A68DA63012318460C3783
S31508025810BD465DF8047B704780B483B000AF7860FC
S315080258207B68DB6B07EE903AB0EE670A0C37BD462B
S315080258305DF8047B704780B483B000AF786087ED6B
S31508025840000A7B683A681A64012318460C37BD4673
S315080258505DF8047B704780B483B000AF78607B68DC
S315080258601B6C07EE903AB0EE670A0C37BD465DF838
S31508025870047B704780B483B000AF786087ED000A76
S315080258807B683A685A64012318460C37BD465DF8A8
S31508025890047B704780B483B000AF78607B685B6C2A
S315080258A007EE903AB0EE670A0C37BD465DF8047B00
S315080258B0704780B483B000AF786039607B683A6815
S315080258C09A64012318460C37BD465DF8047B704777
S315080258D080B483B000AF78607B689B6C18460C373F
S315080258E0BD465DF8047B704780B483B000AF78602C
S315080258F039607B683A68DA64012318460C37BD4674
S315080259005DF8047B704780B483B000AF78607B682B
S31508025910DB6C18460C37BD465DF8047B704780B4CD
S3150802592083B000AF786039607B683A681A650123EC
S3150802593018460C37BD465DF8047B704780B483B0C1
S3150802594000AF78607B681B6D18460C37BD465DF85C
S31508025950047B704780B483B000AF786039607B6897
S315080259603A685A65012318460C37BD465DF8047B2A
S31508025970704780B483B000AF78607B685B6D184669
S315080259800C37BD465DF8047B704780B483B000AF20
S31508025990786039607B683A689A65012318460C373D
S315080259A0BD465DF8047B704780B483B000AF78606B
S315080259B07B689B6D18460C37BD465DF8047B7047BD
S315080259C080B483B000AF786039607B683A68DA657C
S315080259D0012318460C37BD465DF8047B704780B430
S315080259E083B000AF78607B68DB6D18460C37BD461E
S315080259F05DF8047B704780B483B000AF7860396085
S31508025A007B683A681A66012318460C37BD465DF864
S31508025A10047B704780B483B000AF78607B681B6EE6
S31508025A2018460C37BD465DF8047B704780B483B0D0
S31508025A3000AF786039607B683A685A66012318466F
S31508025A400C37BD465DF8047B704780B483B000AF5F
S31508025A5078607B685B6E18460C37BD465DF8047B3A
S31508025A60704780B485B000AF78600B46FB70FB7850
S31508025A70002B01D100230BE07B6893F86820FB78A2
S31508025A801340DBB2002B14BF01230023FB73FB7BFD
S31508025A9018461437BD465DF8047B704780B483B058
S31508025AA000AF78600B46FB70FB78002B01D1002310
S31508025AB00BE07B6893F86820FB781343DAB27B68BD
S31508025AC083F868207B6893F8683018460C37BD4619
S31508025AD05DF8047B704780B483B000AF78600B46EC
S31508025AE0FB70FB78002B01D1002310E07B6893F84A
S31508025AF068305AB297F90330DB435BB213405BB2A4
S31508025B00DAB27B6883F868207B6893F868301846AF
S31508025B100C37BD465DF8047B7047000080B586B039
S31508025B2000AF7860144A154BD31A7B617B693B61D7
S31508025B30134B1B68002B02D1114B124A1A60104BE9
S31508025B401A687B6813443A699A4207D210F0A0FA97
S31508025B5003460C221A604FF0FF3309E0084B1B6814
S31508025B60FB60074B1A687B681344054A1360FB6897
S31508025B7018461837BD4680BD00000A2000040000FA
S31508025B802C5600205860002080B483B000AF354BF5
S31508025B90D3F88830334A43F47003C2F88830324B5C
S31508025BA001221A60304B0022DA612F4B00221A6258
S31508025BB02D4B1A682C492D4B13400B602A4B002299
S31508025BC09A62294B0022DA62274B00221A63264B75
S31508025BD0274A5A63244B00229A63234B244ADA63E0
S31508025BE0214B00221A64204B214A5A641E4B00227A
S31508025BF09A641D4B1B681C4A23F4802313601A4BB4
S31508025C0000221A65174B4FF000629A60194B9B697E
S31508025C1003F060437B607B68B3F1604F03D07B6817
S31508025C20B3F1404F17D1134BDB6903F00103002B85
S31508025C3005D0104B104ADA600E4B104ADA600D4B4B
S31508025C40DB690C4A43F00203D3610A4BDB69094A52
S31508025C5043F00103D36100BF0C37BD465DF8047BF0
S31508025C60704700BF00ED00E0000C0244E3EAE2EAF6
S31508025C7080020101002002403B2A19087F6E5D4C12
S31508025C8080B400AF214B1B8801339AB21F4B1A808E
S31508025C901F4B01221A701D4B1A881E4BA3FB0213B7
S31508025CA0D9080B469B000B445B00D31A9BB2002B08
S31508025CB002D1194B01221A70144B1B88174AA2FBF0
S31508025CC003125209642101FB02F29B1A9BB2002BB2
S31508025CD002D1134B01221A700C4B1B88114AA2FBE4
S31508025CE0031292094FF47A7101FB02F29B1A9BB2D4
S31508025CF0002B05D10C4B01221A70044B00221A8084
S31508025D0000BFBD465DF8047B704700BF30560020D1
S31508025D1032560020CDCCCCCC335600201F85EB5111
S31508025D2034560020D34D62103556002098B500AF80
S31508025D30FEF75EFBFFF794FB04460020FCF7CEFB5A
S31508025D40F0EE407AB0EE670A2046FFF7BAFCFEF795
S31508025D504FFBFFF785FB04460120FCF7BFFBF0EE7D
S31508025D60407AB0EE670A2046FFF7CAFCFEF740FB08
S31508025D70FFF776FB04460220FCF7B0FBF0EE407A0A
S31508025D80B0EE670A2046FFF7DAFCFEF731FBFFF7AB
S31508025D9067FB04460320FCF7A1FBF0EE407AB0EE5F
S31508025DA0670A2046FFF7EAFCFEF722FBFFF758FBD5
S31508025DB004460420FCF792FBF0EE407AB0EE670A3E
S31508025DC02046FFF7FAFCFEF713FBFFF749FB0446EA
S31508025DD00520FCF783FBF0EE407AB0EE670A204610
S31508025DE0FFF70AFDFEF704FBFFF73AFB0446062017
S31508025DF0FCF774FBF0EE407AB0EE670A2046FFF72E
S31508025E001AFDFEF7F5FAFFF72BFB04460720FCF707
S31508025E1065FBF0EE407AB0EE670A2046FFF72AFDE8
S31508025E20FEF7E6FA00BF98BDB0B592B000AF114BC7
S31508025E301A883B46114618460CF06DFF3A1D3B463A
S31508025E40114618460DF050FA0DF020FB04463B1D8C
S31508025E5018460DF02CF805463B1D18460DF033F88A
S31508025E6003461A46294620460EF0B0FE00BF4837BA
S31508025E70BD46B0BD3E560020B0B592B000AFC24B8B
S31508025E801B78002B13D0C04B00221A70FDF72CFF8B
S31508025E90FDF732FBFDF79AFAFDF748F9FDF7CCFA5A
S31508025EA00EF032FA0EF042FC0020FEF717F9B74B55
S31508025EB01B78002B08D0B54B00221A70B44B1B78FE
S31508025EC00133DAB2B24B1A70B14B1B78042B02D9E2
S31508025ED0AF4B00221A70AF4B1B78002B60D0AD4B2C
S31508025EE000221A70AC4B1B780133DAB2AA4B1A702D
S31508025EF00EF0AAFB0EF0BAFD0EF0EEFA0EF0FEFC5C
S31508025F00FEF742F9A54800F0D1FCFFF7A9FA0346C5
S31508025F101846FFF7D7FA0346012B03D1FFF706FF08
S31508025F2000F0DBFA0EF0D4F8034618460EF0E6F84F
S31508025F300346012118460CF0FBFB0346002B29D128
S31508025F400EF0C6F8034618460EF0D8F803460221A4
S31508025F5018460CF0EDFB0346002B1BD10EF0B8F8E1
S31508025F60034618460EF0CAF80346042118460CF0F2
S31508025F70DFFB0346002B0DD10EF0AAF8034618469E
S31508025F800EF0BCF80346082118460CF0D1FB03466E
S31508025F90002B03D00421824802F094FBFEF728FA6C
S31508025FA07D4B1B78012B11D97B4B00221A7000F00E
S31508025FB06FFAFFF755FA03461846FFF783FA0346C0
S31508025FC0002B03D1FFF7B2FE00F087FA754B1B7858
S31508025FD0002B00F0F481734B00221A70724B1B7867
S31508025FE00133DAB2704B1A70704B1B780133DAB28E
S31508025FF06E4B1A706E4B1B780133DAB26C4B1A7001
S315080260006C4B1B780133DAB26A4B1A706A4B1B78EF
S315080260100133DAB2684B1A70684B1B8801339AB29D
S31508026020664B1A800EF054F8034618460EF066F8C8
S315080260300346012118460CF07BFB034683F0010355
S31508026040DBB2002B36D00EF043F8034618460EF0A4
S3150802605055F80346022118460CF06AFB034683F0FC
S315080260600103DBB2002B25D00EF032F803461846A0
S315080260700EF044F80346042118460CF059FB034671
S3150802608083F00103DBB2002B14D00EF021F803468D
S3150802609018460EF033F80346082118460CF048FB5A
S315080260A0034683F00103DBB2002B03D004213C48EC
S315080260B002F008FBFFF7D4F9034601211846FFF759
S315080260C0D0FC0346002B0FD0FFF7CAF90346184641
S315080260D0FFF707FB10EE103A1846FAF745FA02469A
S315080260E00B46374800F072FCFFF7BAF9034601215E
S315080260F01846FFF7B6FC0346002B0FD0FFF7B0F998
S3150802610003461846FFF70CFB10EE103A1846FAF744
S315080261102BFA02460B462B4800F058FCFFF7A0F96B
S31508026120034601211846FFF79CFC0346002B0FD0B5
S31508026130FFF796F903461846FFF711FB10EE103AD9
S315080261401846FAF711FA02460B461F4800F03EFCBB
S31508026150FFF786F9034601211846FFF782FC034634
S31508026160002B35D0FFF77CF903461846FFF716FBD6
S3150802617010EE103A1846FAF7F7F902460B46134894
S3150802618000F024FC24E000BF3256002033560020DB
S315080261903C560020345600203B560020F1430208A4
S315080261A00004024235560020365600203756002093
S315080261B038560020395600203D5600203E5600200B
S315080261C0F8A0030808A1030818A1030828A10308D0
S315080261D0FFF746F9034601211846FFF742FC034634
S315080261E0002B0FD0FFF73CF903461846FFF7F5FADE
S315080261F010EE103A1846FAF7B7F902460B469748D0
S3150802620000F0E4FBFFF72CF9034601211846FFF7D5
S3150802621028FC0346002B0FD0FFF722F9034618463F
S31508026220FFF7FAFA10EE103A1846FAF79DF90246FF
S315080262300B468B4800F0CAFBFFF712F90346012109
S315080262401846FFF70EFC0346002B0FD0FFF708F996
S3150802625003461846FFF7FFFA10EE103A1846FAF701
S3150802626083F902460B467F4800F0B0FBFFF7F8F8C1
S31508026270034601211846FFF7F4FB0346002B0FD00D
S31508026280FFF7EEF803461846FFF704FB10EE103A3E
S315080262901846FAF769F902460B46734800F096FB68
S315080262A0FFF7DEF8034601211846FFF7DAFB034635
S315080262B0002B02D06D4800F089FBFFF7D1F80346A0
S315080262C001211846FFF7CDFB0346002B02D068488A
S315080262D000F07CFBFFF7C4F8034601211846FFF7D6
S315080262E0C0FB0346002B0FD00DF0F2FE03461846FC
S315080262F00DF004FF0346012118460CF019FA03466D
S3150802630019465C4800F062FBFFF7AAF8034601212A
S315080263101846FFF7A6FB0346002B0FD00DF0D8FE52
S31508026320034618460DF0EAFE0346022118460CF00B
S31508026330FFF9034619464F4800F048FBFFF790F865
S31508026340034601211846FFF78CFB0346002B0FD0A4
S315080263500DF0BEFE034618460DF0D0FE0346042194
S3150802636018460CF0E5F903461946424800F02EFB9A
S31508026370FFF776F8034601211846FFF772FB034634
S31508026380002B0FD00DF0A4FE034618460DF0B6FEFC
S315080263900346082118460CF0CBF903461946354838
S315080263A000F014FBFFF75CF8034601211846FFF7D5
S315080263B058FB0346002B02D02C4800F007FB2E4B55
S315080263C01B78012B02D92C4B00221A702B4B1B78F7
S315080263D0022B25D9294B00221A70294B1B78002B30
S315080263E01ED1274B01221A7000F07EF901233B7059
S315080263F03A1D3B46114618460CF0E0FE0DF046F8EB
S3150802640004463B1D18460CF052FD05463B1D184630
S315080264100CF059FD03461A46294620460EF0D6FBCD
S31508026420184B1B78042B02D9164B00221A70164BEE
S315080264301B780E2B04D9144B00221A70FDF7E2FBC7
S31508026440124B1B783B2B04D9104B00221A70FFF70C
S31508026450EBFC00BF4837BD46B0BD00BF38A10308F4
S3150802646048A1030858A1030868A1030878A10308EC
S315080264707CA1030888A10308365600203756002057
S315080264803A56002038560020395600203D5600203C
S31508026490B0B592B000AF0DF01BFE034618460DF0DC
S315080264A02DFE02463B1D194610460CF094FD0CF0D3
S315080264B0FBFF04463B1D18460CF0F9FC05463B1D3E
S315080264C018460CF000FD03461A46294620460EF0E9
S315080264D07DFB00BF4837BD46B0BDB0B5A2B000AF20
S315080264E007F148034022002118460FF05DFDFEF72A
S315080264F0B7FF03461846FFF7F4F8F0EE407A07F1BD
S315080265004803B0EE670A18460CF064F9FEF7A8FFCE
S3150802651003461846FFF704F9F0EE407A07F14803F6
S31508026520B0EE670A18460CF073F9FEF799FF0346B0
S315080265301846FFF714F9F0EE407A07F14803B0EE71
S31508026540670A18460CF082F9FEF78AFF03461846D0
S31508026550FFF724F9F0EE407A07F14803B0EE670A2E
S3150802656018460CF091F9FEF77BFF03461846FFF72B
S3150802657034F9F0EE407A07F14803B0EE670A184696
S315080265800CF0A0F9FEF76CFF03461846FFF744F92C
S31508026590F0EE407A07F14803B0EE670A18460CF0A7
S315080265A0AFF9FEF75DFF03461846FFF754F9F0EE1A
S315080265B0407A07F14803B0EE670A18460CF0BEF9AE
S315080265C0FEF74EFF03461846FFF764F9F0EE407AE7
S315080265D007F14803B0EE670A18460CF0CDF9FEF744
S315080265E03FFF03461846FFF773F9024607F14803C9
S315080265F0114618460CF0DBF9FEF732FF0346184639
S31508026600FFF781F9024607F14803114618460CF0CE
S31508026610E8F9FEF725FF03461846FFF78FF9024603
S3150802662007F14803114618460CF0F5F9FEF718FF6C
S3150802663003461846FFF79DF9024607F14803114635
S3150802664018460CF002FAFEF70BFF03461846FFF748
S31508026650ABF9024607F14803114618460CF00FFA41
S31508026660FEF7FEFE03461846FFF7B9F9024607F19A
S315080266704803114618460CF01CFAFEF7F1FE0346CB
S315080266801846FFF7C7F9024607F1480311461846A6
S315080266900CF029FAFEF7E4FE03461846FFF7D5F989
S315080266A0024607F14803114618460CF036FA3A1D17
S315080266B007F14803114618460CF0C5FC0CF002FF18
S315080266C004463B1D18460CF0F2FB05463B1D1846D0
S315080266D00CF0F9FB03461A46294620460EF076FACE
S315080266E000BF8837BD46B0BDB0B594B000AF5C4BAD
S315080266F0D3F8F430002B09DA5A4800F067F907F1A3
S315080267004803062118460CF07FFA5DE0544BD3F88D
S31508026710F43003F08043002B09D0534800F056F9B1
S3150802672007F14803052118460CF06EFA4CE04C4B6B
S31508026730D3F8F43003F00053002B09D04B4800F08D
S3150802674045F907F14803042118460CF05DFA3BE0C7
S31508026750434BD3F8F43003F08053002B09D0444856
S3150802676000F034F907F14803032118460CF04CFAF5
S315080267702AE03B4BD3F8F43003F00063002B09D030
S315080267803C4800F023F907F14803022118460CF0A9
S315080267903BFA19E0324BD3F8F43003F08063002B4E
S315080267A009D0354800F012F907F1480301211846C5
S315080267B00CF02AFA08E0314800F008F907F1480314
S315080267C0002118460CF020FA254BD3F8F430244A57
S315080267D043F40003C2F8F43029480CF0BAFE034623
S315080267E01B0ADAB207F14803114618460CF027FAD3
S315080267F023480CF0AEFE0346DAB207F14803114607
S3150802680018460CF037FA1F4B9A7807F148031146D7
S3150802681018460CF04AFA1B4BDA7807F14803114678
S3150802682018460CF05DFA3A1D07F148031146184658
S315080268300CF01BFD0CF02AFE04463B1D18460CF014
S3150802684036FB05463B1D18460CF03DFB03461A4629
S31508026850294620460EF0BAF900BF5037BD46B0BDEC
S31508026860000C024490A10308ACA10308C8A10308BE
S31508026870E4A1030804A203081CA2030834A203081D
S3150802688000E00108E0BF1F0880B582B000AF0346EA
S31508026890FB71FB1D0122194603480BF045FB00BF9D
S315080268A00837BD4680BD00BF4056002080B584B07B
S315080268B000AF78600023FB730023BB7324480BF0F8
S315080268C017FB034683F00103DBB2002B19D00DE058
S315080268D07B689847BB7B1846FBF77AFA0023BB739B
S315080268E0FB7B0133FB73FB7B3F2B2CD807F10E0393
S315080268F00122194616480BF052FB0346002BE7D134
S3150802690022E0144809F032FB0346202B0DD1114B25
S315080269100122A3F85C200F4B0122A3F85E20012274
S315080269200D490C4808F018FF0EE00A4BB3F85C2034
S31508026930084BB3F85E309BB29A4205D0FDF744FD88
S31508026940FDF74EFD00E000BF00BF1037BD4680BD13
S3150802695040560020745400209056002080B582B01C
S3150802696000AF78600B467B807A884FF47A73796831
S31508026970034808F052FE012318460837BD4680BD73
S315080269807454002080B500AF4022064906480BF031
S3150802699025FAFEF765FD034680211846FFF77EF8BD
S315080269A000BF80BD505600204056002080B500AF7B
S315080269B0FFF7E8FF01220349034808F0CDFE00BFAE
S315080269C080BD00BF90560020745400200FB480B5D5
S315080269D082B000AFFEF744FD034680211846FFF752
S315080269E040F8034683F00103DBB2002B01D00023F3
S315080269F01FE04FF48072002111480FF0D5FA07F113
S31508026A0014033B603A6839690D480FF0B3FA7860A7
S31508026A100B4A0C490C480FF033FA0B48F9F738FCC5
S31508026A2003469BB219460848FFF798FF03467B6060
S31508026A307B6818460837BD46BDE8804004B07047F3
S31508026A409856002050A203089857002080B582B0B5
S31508026A5000AF78607B681B68094A93420CD1094BE0
S31508026A601B781846FFF710FF064B00221A70012200
S31508026A700449054808F070FE00BF0837BD4680BDC8
S31508026A8000380140905600207454002080B582B028
S31508026A9000AF7860786809F07EFA0346074A136001
S31508026AA07B681B68064A934203D1FDF78DFCFDF706
S31508026AB097FC00BF0837BD4680BD00BF945600202C
S31508026AC0003801400D488546FFF75EF80C480D4927
S31508026AD00D4A002302E0D458C4500433C4188C4229
S31508026AE0F9D30A4A0A4C002301E013600432A2428F
S31508026AF0FBD30FF0D3FAFDF78DFCFEE700000A2060
S31508026B000000002084070020B0B60308840700208E
S31508026B1058600020FEE7000080B500AF032000F0B1
S31508026B2012F902F071FC02460B4B1B6A03F00F03C3
S31508026B300A49CB5C22FA03F3094A13600F20FEF7CF
S31508026B4031FB0346002B01D0012302E0FEF7AAF926
S31508026B500023184680BD00BF000C0244F8B10308A2
S31508026B609405002080B400AF064B1B781A46064BE4
S31508026B701B681344044A136000BFBD465DF8047BD4
S31508026B80704700BF9C050020A858002080B400AFBB
S31508026B90034B1B681846BD465DF8047B704700BF69
S31508026BA0A858002080B485B000AF78607B6803F0EF
S31508026BB00703FB600C4BDB68BB60BA684FF6FF0342
S31508026BC01340BB60FB681A02BB68134343F0BF63FA
S31508026BD043F40033BB60044ABB68D36000BF143772
S31508026BE0BD465DF8047B704700ED00E080B400AF57
S31508026BF0044BDB681B0A03F007031846BD465DF81B
S31508026C00047B704700ED00E080B483B000AF034612
S31508026C10FB80B7F90630002B0BDBFB8803F01F025B
S31508026C200749B7F906305B09012000FA02F241F872
S31508026C30232000BF0C37BD465DF8047B704700BFB2
S31508026C4000E100E080B483B000AF0346FB80B7F9E9
S31508026C500630002B12DBFB8803F01F020A49B7F93C
S31508026C6006305B09012000FA02F2203341F823209C
S31508026C70BFF34F8F00BFBFF36F8F00BF00BF0C3744
S31508026C80BD465DF8047B704700E100E080B483B03E
S31508026C9000AF03463960FB80B7F90630002B0ADBE2
S31508026CA03B68DAB20C49B7F906301201D2B20B4484
S31508026CB083F800230AE03B68DAB20849FB8803F046
S31508026CC00F03043B1201D2B20B441A7600BF0C37EB
S31508026CD0BD465DF8047B704700E100E000ED00E088
S31508026CE080B489B000AFF860B9607A60FB6803F0D7
S31508026CF00703FB61FB69C3F10703042B28BF0423BF
S31508026D00BB61FB690433062B02D9FB69033B00E02E
S31508026D1000237B614FF0FF32BB6902FA03F3DA43C1
S31508026D20BB681A407B699A404FF0FF317B6901FACA
S31508026D3003F3D9437B680B40134318462437BD46F1
S31508026D405DF8047B704780B582B000AF78607868DA
S31508026D50FFF728FF00BF0837BD4680BD80B586B05D
S31508026D6000AF0346B9607A60FB81FFF73FFF78619F
S31508026D707A68B9687869FFF7B3FF0246B7F90E3041
S31508026D8011461846FFF782FF00BF1837BD4680BD79
S31508026D9080B582B000AF0346FB80B7F906301846C5
S31508026DA0FFF732FF00BF0837BD4680BD80B582B007
S31508026DB000AF0346FB80B7F906301846FFF742FFD5
S31508026DC000BF0837BD4680BD80B584B000AF786085
S31508026DD0FFF7DCFEF8607B68002B01D101236BE02C
S31508026DE07B6893F85430DBB2022B08D07B682022EA
S31508026DF09A657B68002283F84C2001235CE07B6855
S31508026E001B685A697B681B6842F004025A617B68F0
S31508026E10052283F8542020E0FFF7B8FE0246FB68F5
S31508026E20D31A052B19D97B689B6D43F010027B6830
S31508026E309A657B68032283F854207B681B6D03F0EE
S31508026E408003002B03D07B685B6F01221A737B6871
S31508026E50002283F84C2001232EE07B681B681B69FD
S31508026E6003F40053002BD7D07B681B685A697B68EA
S31508026E701B6842F002025A617B68042283F8542096
S31508026E807B681B684FF4FE42DA607B68012283F84E
S31508026E9054207B681B6D03F08003002B07D07B68A8
S31508026EA05B6F01221A737B681B6800229A647B68EF
S31508026EB0002283F84C20002318461037BD4680BDB1
S31508026EC080B483B000AF78607B68002B01D10123C0
S31508026ED019E07B6893F85430DBB2022B04D07B6846
S31508026EE020229A6501230EE07B68042283F8542047
S31508026EF07B681B685B697A68126843F4005343F03F
S31508026F0004035361002318460C37BD465DF8047B1B
S31508026F107047000080B584B000AF78607B68002BAC
S31508026F2001D1012347E17B6893F85C30DBB2002B81
S31508026F3006D17B68002283F85D207868FDF7BAFFE0
S31508026F407B681B689A697B681B6822F010029A6143
S31508026F50FFF71CFEF86012E0FFF718FE0246FB6810
S31508026F60D31A0A2B0BD97B681B6E43F001027B6886
S31508026F701A667B68032283F85C2001231BE17B687F
S31508026F801B689B6903F00803082BE5D07B681B681E
S31508026F909A697B681B6842F001029A61FFF7F6FD5F
S31508026FA0F86012E0FFF7F2FD0246FB68D31A0A2BD5
S31508026FB00BD97B681B6E43F001027B681A667B68F5
S31508026FC0032283F85C200123F5E07B681B689B6932
S31508026FD003F00103002BE5D07B681B689A697B687E
S31508026FE01B6842F002029A617B681B68744A9342E4
S31508026FF003D1744A7B685B6813607B681B7C012B30
S3150802700008D17B681B689A697B681B6822F0400274
S315080270109A6107E07B681B689A697B681B6842F07D
S3150802702040029A617B685B7C012B08D17B681B68EE
S315080270309A697B681B6842F480429A6107E07B681A
S315080270401B689A697B681B6822F480429A617B688E
S315080270509B7C012B08D17B681B689A697B681B6835
S3150802706022F480529A6107E07B681B689A697B68FA
S315080270701B6842F480529A617B681B689B6923F4F9
S3150802708040717B689A687B681B680A439A617B68C9
S315080270901B689A697B681B6822F0A4029A617B685E
S315080270A01B681A697B681B6822F010021A617B68E2
S315080270B0DB68012B08D17B681B689A697B681B68A9
S315080270C042F004029A612CE07B68DB68002B28D028
S315080270D07B68DB68022B1CD07B681B689A697B6815
S315080270E01B6842F080029A617B681B681A697B6892
S315080270F01B6842F010021A617B68DB68032B10D109
S315080271007B681B689A697B681B6842F020029A6151
S3150802711007E07B681B689A697B681B6842F0200255
S315080271209A617B689B69013B5A067B68DB69013B6E
S315080271301B021A437B681B6A013B42EA03017B680E
S315080271405B69013B1A047B681B680A43DA617B6840
S315080271509B68B3F5407F15D17B689B6A5A1E7B688C
S31508027160DB6A013B1B021A437B681B6B013B1B0153
S3150802717042EA03017B685B6A013B1A047B681B6867
S315080271800A43DA607B681B68D3F8C0107B68DA6B3F
S315080271907B681B680A43C3F8C020786800F0C8FCFD
S315080271A07B6800229A657B6800221A667B68012240
S315080271B083F85C20002318461037BD4680BD00BF01
S315080271C000A4004000A5004080B487B000AF7860F4
S315080271D039607B6893F85C30FB75FB7D012B02D026
S315080271E0FB7D022B3DD13B681B68002B19D13B68FE
S315080271F09B689A073B68DB68DB061A433B681B6990
S315080272001B041A433B685B6913433B617B681A6C30
S315080272103B685B689B001344BB60BB683A691A60AB
S315080272201DE03B68DB685A073B681B6913433B61F1
S315080272303B689B689A073B685B691343FB607B68FC
S315080272405A6C3B685B68DB001344BB60BB683A69EF
S315080272501A60BB680433BB60BB68FA681A6000230D
S3150802726006E07B681B6E43F002027B681A660123FE
S3150802727018461C37BD465DF8047B704780B485B056
S3150802728000AFF860B9607A603B60FB6893F85C30DF
S31508027290DBB2012B16D1FB681B68D3F8803023F0CA
S315080272A03F01BB681A017B689B001A433B685B0077
S315080272B01A43BB691A43FB681B680A43C3F8802052
S315080272C0002306E0FB681B6E43F00402FB681A669D
S315080272D0012318461437BD465DF8047B704780B40F
S315080272E083B000AF78607B6893F85C30DBB2012B21
S315080272F010D17B68022283F85C207B681B689A6936
S315080273007B681B6822F001029A617B6800221A6672
S31508027310002306E07B681B6E43F004027B681A664C
S31508027320012318460C37BD465DF8047B704780B5C5
S3150802733086B000AFF860B9607A60FB6893F85C3093
S31508027340DBB2022B2CD1FB681B68D3F8C43003F4DA
S315080273500013002B07D0FB681B6E43F40072FB6810
S315080273601A66012323E0FB681B68D3F8C4301B0C9A
S3150802737003F003037B617B697A68B968F86800F0F1
S3150802738039FCFB681B6801217A6901FA02F2C3F823
S31508027390CC2001227B699A40FB689A65002306E0A5
S315080273A0FB681B6E43F00802FB681A66012318463F
S315080273B01837BD4680BD80B483B000AF78607B685D
S315080273C09B6D18460C37BD465DF8047B7047000076
S315080273D080B48BB000AFF860B9607A603B60002376
S315080273E0FB61FB6893F85C30FB76FB7E022B40F070
S315080273F0E880BB68402B37D1FB681B68D3F890300E
S3150802740003F00F03002B07D1FB681B6E43F480724F
S31508027410FB681A660123DBE0FB681B68D3F8903029
S315080274201B0E03F00103012B0AD1FB681B68D3F874
S3150802743080305B0A03F00103012B01D10123FB61B2
S31508027440FB681B68D3F890301B0A03F00303FA693A
S315080274501344FB61FB68996CFA691346DB00134413
S31508027460DB000B447B6236E0FB681B68D3F8983076
S3150802747003F00F03002B07D1FB681B6E43F48072DF
S31508027480FB681A660123A3E0FB681B68D3F89830E9
S315080274901B0E03F00103012B0AD1FB681B68D3F804
S315080274A080301B0A03F00103012B01D10123FB6182
S315080274B0FB681B68D3F898301B0A03F00303FA69C2
S315080274C01344FB61FB68D96CFA691346DB00134463
S315080274D0DB000B447B627B6A1B6803F080427B6895
S315080274E05A607B685B68002B07D17B6A1B689B0C1A
S315080274F0C3F30A027B681A6005E07B6A1B6823F0FD
S3150802750060427B681A607B6A1B6803F000527B68DC
S315080275109A607B6A1B6803F000427B681A617B6A81
S3150802752004337B627B6A1B689AB27B68DA617B6A80
S315080275301B681B0C03F00F027B68DA607B6A1B6808
S3150802754003F480127B685A617B6A1B6803F4001293
S315080275507B689A617B6A1B681B0E03F07F027B6855
S315080275601A627B6A1B68DA0F7B685A627B6A043383
S315080275707B627B6A7B6100233B620AE07A693B6A2B
S315080275801A4439683B6A0B4412781A703B6A01330B
S315080275903B627B68DB68114AD35C1A463B6A9342B4
S315080275A0ECD3BB68402B05D1FB681B68FA69C3F8A4
S315080275B0942004E0FB681B68FA69C3F89C20002340
S315080275C006E0FB681B6E43F00802FB681A66012395
S315080275D018462C37BD465DF8047B704710B203087F
S315080275E080B483B000AF786039607B681B68D3F8D3
S315080275F0C8203B681340002B01D1002300E0012379
S3150802760018460C37BD465DF8047B704780B485B0D2
S3150802761000AF786039603B68402B07D17B681B68EE
S31508027620D3F8903003F00F03FB6006E07B681B6813
S31508027630D3F8983003F00F03FB60FB68184614373B
S31508027640BD465DF8047B704780B487B000AFF8602A
S31508027650B9607A60FB6893F85C30FB75FB7D012B99
S3150802766003D0FB7D022B40F0C880FB681B689B6D2C
S315080276703B61BB6803F00703002B04D03B6903F0A8
S315080276800103002B3BD0BB6803F03803002B04D060
S315080276903B6903F00203002B31D0BB6803F4E073A5
S315080276A0002B04D03B6903F00403002B27D0BB68E8
S315080276B003F4F053002B04D03B6903F00803002BB4
S315080276C01DD0BB6803F46043002B04D03B6903F06A
S315080276D01003002B13D0BB6803F44033002B04D0ED
S315080276E03B6903F02003002B09D0BB6803F47C0333
S315080276F0002B0CD03B6903F04003002B07D1FB6833
S315080277001B68DA6DFB681B6842F00102DA65BB6822
S3150802771003F00703002B04D03B6903F00103002B97
S315080277203BD1BB6803F03803002B04D03B6903F056
S315080277300203002B31D1BB6803F4E073002B04D09B
S315080277403B6903F00403002B27D1BB6803F4F0530B
S31508027750002B04D03B6903F00803002B1DD1BB683C
S3150802776003F46043002B04D03B6903F01003002B9B
S3150802777013D1BB6803F44033002B04D03B6903F0F2
S315080277802003002B09D1BB6803F47C03002B0CD021
S315080277903B6903F04003002B07D0FB681B68DA6DD0
S315080277A0FB681B6842F00202DA65BB6803F08003D5
S315080277B0002B09D0FB681B68D3F8DC10FB681B6832
S315080277C07A680A43C3F8DC20BB6803F48073002B8B
S315080277D009D0FB681B68D3F8E010FB681B687A6857
S315080277E00A43C3F8E020FB681B68596DFB681B68EF
S315080277F0BA680A435A65002306E0FB681B6E43F023
S315080278000202FB681A66012318461C37BD465DF854
S31508027810047B704780B58CB000AF78607B681B68C4
S315080278201B6D03F4E053FB627B681B685B6DFA6AA7
S315080278301340FB627B681B681B6D03F00703BB6280
S315080278407B681B685B6DBA6A1340BB627B681B6800
S315080278501B6D03F038037B627B681B685B6D7A6A73
S3150802786013407B627B681B681B6D03F471033B62E2
S315080278707B681B685B6D3A6A13403B627B681B68D0
S315080278801B6D03F46023FB617B681B685B6DFA69F9
S315080278901340FB617B681B685B6DBB617B681B6879
S315080278A01B6D7B617B6903F04003002B0BD0BB6920
S315080278B003F04003002B06D07B681B6840221A653A
S315080278C0786800F016F97B6903F48073002B19D0E7
S315080278D0BB6903F48073002B14D07B681B68D3F84A
S315080278E0D8303B617B681B68D3F8E0303A691340AD
S315080278F03B617B681B684FF480721A653969786840
S3150802790000F0D8F8FB6A002B07D07B681B68FA6A76
S315080279101A65F96A786800F0A2F8BB6A002B07D0E4
S315080279207B681B68BA6A1A65B96A7868FDF714F93A
S315080279307B6A002B07D07B681B687A6A1A65796AA4
S31508027940786800F097F87B6903F40073002B0CD073
S31508027950BB6903F40073002B07D07B681B684FF4DE
S3150802796000721A65786800F090F87B6903F0800364
S31508027970002B18D0BB6903F08003002B13D07B6859
S315080279801B68D3F8D430FB607B681B68D3F8DC30FD
S31508027990FA681340FB607B681B6880221A65F968DF
S315080279A0786800F07CF87B6903F40053002B0CD04E
S315080279B0BB6903F40053002B07D07B681B684FF49E
S315080279C000521A65786800F080F87B6903F4004370
S315080279D0002B0CD0BB6903F40043002B07D07B684D
S315080279E01B684FF400421A65786800F078F87B69DC
S315080279F003F48043002B0FD0BB6903F48043002BAA
S31508027A000AD07B681B684FF480421A657B681B6E36
S31508027A1043F080027B681A66FB69002B07D07B68F5
S31508027A201B68FA691A65F969786800F076F83B6A9C
S31508027A30002B09D07B681B683A6A1A657B681A6E3E
S31508027A403B6A1A437B681A667B681B6E002B02D058
S31508027A50786800F058F800BF3037BD4680BD80B45C
S31508027A6083B000AF7860396000BF0C37BD465DF859
S31508027A70047B704780B483B000AF7860396000BF7A
S31508027A800C37BD465DF8047B704780B483B000AFFF
S31508027A90786000BF0C37BD465DF8047B704780B43A
S31508027AA083B000AF7860396000BF0C37BD465DF819
S31508027AB0047B704780B483B000AF7860396000BF3A
S31508027AC00C37BD465DF8047B704780B483B000AFBF
S31508027AD0786000BF0C37BD465DF8047B704780B4FA
S31508027AE083B000AF786000BF0C37BD465DF8047BF3
S31508027AF0704780B483B000AF786000BF0C37BD46CC
S31508027B005DF8047B704780B483B000AF786000BF2D
S31508027B100C37BD465DF8047B704780B483B000AF6E
S31508027B207860396000BF0C37BD465DF8047B704744
S31508027B3080B485B000AF78602C4BBB607B681B684D
S31508027B402B4A934203D1BB6803F55473BB607B6827
S31508027B50BA681A647B681B68D3F8803023F4F81174
S31508027B607B685B6B1A047B681B680A43C3F8802030
S31508027B70BB6803F170027B685A647B681B68D3F89A
S31508027B80803023F070617B689B6B1A067B681B68E2
S31508027B900A43C3F88020BB6803F1B0027B689A6483
S31508027BA0BB6803F5C4727B68DA64BB6803F51872AE
S31508027BB07B681A65BB6803F51E727B685A65BB68E3
S31508027BC0FB6005E0FB6800221A60FB680433FB6071
S31508027BD0BB6803F55473FA689A42F3D300BF00BF31
S31508027BE01437BD465DF8047B704700BF00AC004001
S31508027BF000A8004080B489B000AFF860B9607A6026
S31508027C003B60BB685B68002B0AD1BB681A69BB6814
S31508027C109B681A43BB681B689B041343FB610AE013
S31508027C20BB681A69BB689B681A43BB681B6813431F
S31508027C3043F08043FB61BB681B6A1A06BB68DB69B3
S31508027C401A43BB689B691A43BB685B691A43BB68DC
S31508027C50DB681B0413433B61FB68596D3A6813469C
S31508027C60DB001344DB000B44BB61BB69FA691A608B
S31508027C70BB690433BB61BB693A691A60BB690433E1
S31508027C80BB6100237B6120E07B6903337A68134476
S31508027C901B781A067B69023379680B441B781B0426
S31508027CA01A437B69013379680B441B781B02134319
S31508027CB079687A690A4412781A43BB691A60BB69F9
S31508027CC00433BB617B6904337B61BB68DB68064AA4
S31508027CD0D35C1A467B699342D6D300BF00BF2437CA
S31508027CE0BD465DF8047B704710B2030880B588B0BC
S31508027CF000AFF860B9607A60324B1B78012B01D16C
S31508027D0002235AE02F4B01221A702E4B00225A6088
S31508027D104FF47A7000F0A4F80346FB77FB7F002B3A
S31508027D2047D1284AFB689360274BBB61FB6823F05F
S31508027D300043022B04D17968B86800F0DFF81BE02B
S31508027D40FB68224A934203D0FB68214A934204D134
S31508027D507968B86800F00EF90EE0FB6823F0004374
S31508027D601C4A934204D17968B86800F04FF903E0D7
S31508027D707968B86800F04AF94FF47A7000F070F83A
S31508027D800346FB77BB691A68FB6823F0304323F086
S31508027D900403DB431A40BB691A60FB680C4A934228
S31508027DA007D10D4B7B617B691B6823F004027B6953
S31508027DB01A60044B00221A70FB7F18462037BD460C
S31508027DC080BD00BFA0050020282002400200001046
S31508027DD006000010020000404020024080B483B032
S31508027DE000AF0023FB710D4B9B6A03F00103002BC6
S31508027DF00DD00A4B0A4A5A60084B0A4A5A60074B80
S31508027E009B6A03F00103002B01D00123FB71FB7966
S31508027E1018460C37BD465DF8047B704700200240C1
S31508027E2023016745AB89EFCD80B483B000AF002349
S31508027E30FB710A4B9B6A094A43F001039362074B9B
S31508027E409B6A03F00103002B01D10123FB71FB7925
S31508027E5018460C37BD465DF8047B70470020024081
S31508027E6080B586B000AF7860FEF790FE7861204B49
S31508027E703B6110E07B68B3F1FF3F0CD0FEF786FE4C
S31508027E8002467B69D31A7A689A4202D37B68002B28
S31508027E9001D1032327E03B691B6803F00B03002B80
S31508027EA0E8D1144BFB603B691B6803F47E03BB6095
S31508027EB0BB68002B0CD0104B5A68BB6813430E4A9A
S31508027EC05360BB6803F47E02FB681A6001230AE06A
S31508027ED03B691B6803F48033002B03D0FB684FF41D
S31508027EE080321A60002318461837BD4680BD00BF87
S31508027EF02020024030200240A005002080B48BB02A
S31508027F0000AF78603960042387F827307B683B62C4
S31508027F103B68FB61164BBB61BB691B6843F00202F7
S31508027F20BB691A60EFF310833B613B697B6172B6EA
S31508027F3000BFFB691A683B6A1A603B6A04333B62F4
S31508027F40FB690433FB6197F82730013B87F8273032
S31508027F5097F82730002BECD17B69FB60FB6883F32B
S31508027F60108800BF00BF2C37BD465DF8047B7047FA
S31508027F702820024080B48BB000AF786039600423B1
S31508027F8087F827307B683B623B68FB611C4BBB6109
S31508027F901C4B7B61BB691B6843F00202BB691A6012
S31508027FA07B691A68184B9B6803F004031A437B69BA
S31508027FB01A60EFF31083FB60FB683B6172B600BF81
S31508027FC0FB691A683B6A1A603B6A04333B62FB69BF
S31508027FD00433FB6197F82730013B87F8273097F877
S31508027FE02730002BECD13B69BB60BB6883F3108852
S31508027FF000BF00BF2C37BD465DF8047B704700BF43
S315080280002820024040200240A005002080B485B006
S3150802801000AF78603960094BFB60FB681B6843F068
S315080280200202FB681A603A687B68128892B21A8062
S3150802803000BF1437BD465DF8047B7047282002400E
S3150802804080B586B000AF786039603A4B1B78012B51
S3150802805001D102236AE0374B01221A70354B0022FE
S315080280605A604FF47A70FFF7FBFE0346FB75FB7DF9
S31508028070002B57D17B681B682E4A93602E4BFB60F8
S315080280807B681B6823F0004348F2080293420BD12F
S315080280907B685B68184600F053F84FF47A70FFF76E
S315080280A0DFFE0346FB7533E07B681B68234A93426F
S315080280B008D100F0B5F84FF47A70FFF7D1FE0346FF
S315080280C0FB7525E03B684FF0FF321A607B689B68B8
S315080280D03B6115E07B685B681946386900F068F809
S315080280E04FF47A70FFF7BCFE0346FB75FB7D002B47
S315080280F003D03B683A691A600AE03B6901333B617F
S315080281007B68DA687B689B6813443A699A42E1D3CA
S31508028110FB681A687B681B6823F00043DB431A4036
S31508028120FB681A60034B00221A70FB7D1846183743
S31508028130BD4680BDA0050020282002400800008018
S3150802814080B485B000AF7860184BFB607B6803F09B
S315080281500303032B08D1FB681B6843F4004343F06F
S315080281602003FA6813601BE07B6803F00103002B07
S3150802817009D0FB681B6823F0004323F0280343F069
S315080281802802FB681A607B6803F00203002B07D0FB
S31508028190FB681B6843F0004343F02803FA68136040
S315080281A000BF1437BD465DF8047B7047282002409D
S315080281B080B485B000AF78603960184BFB603B68C5
S315080281C003F00103002B11D0FB681B6823F0004360
S315080281D023F4FE53FA681360FB681A687B689B01EE
S315080281E0134343F02402FB681A6010E0FB681B681D
S315080281F023F4FE52FB681A60FB681A687B689B01C7
S31508028200134343F0004343F02403FA68136000BFA4
S315080282101437BD465DF8047B704700BF282002402C
S3150802822080B483B000AF074B7B607B681B6843F062
S3150802823008027B681A6000BF0C37BD465DF8047BEE
S31508028240704700BF4020024080B487B000AF786014
S31508028250396000233B6136E13B681A6801213B69B4
S3150802826001FA03F31340FB60FB68002B00F0288138
S315080282703B685B68022B03D03B685B68122B25D1EF
S315080282803B69DA087B68083253F822307B613B691E
S3150802829003F007039B000F2202FA03F3DB437A6912
S315080282A013407B613B681B6903F00F023B6903F0CD
S315080282B007039B0002FA03F37A6913437B613B695E
S315080282C0DA087B680832796943F822107B681B68EA
S315080282D07B613B695B00032202FA03F3DB437A699B
S315080282E013407B613B685B6803F003023B695B00F2
S315080282F002FA03F37A6913437B617B687A691A6027
S315080283003B685B68012B0BD03B685B68022B07D086
S315080283103B685B68112B03D03B685B68122B30D134
S315080283207B689B687B613B695B00032202FA03F365
S31508028330DB437A6913407B613B68DA683B695B0019
S3150802834002FA03F37A6913437B617B687A699A6056
S315080283507B685B687B6101223B6902FA03F3DB43B4
S315080283607A6913407B613B685B681B0903F001026B
S315080283703B6902FA03F37A6913437B617B687A697C
S315080283805A603B685B68032B17D07B68DB687B61A6
S315080283903B695B00032202FA03F3DB437A69134063
S315080283A07B613B689A683B695B0002FA03F37A6968
S315080283B013437B617B687A69DA603B685B6803F022
S315080283C08053002B7CD0474A3B699B08183352F8E6
S315080283D023307B613B6903F00303DB000F2202FAB9
S315080283E003F3DB437A6913407B617B689A0A3E4B47
S315080283F013403A6902F00302D20093407A691343A2
S315080284007B6138493B699B0818337A6941F823200E
S31508028410344B1B687B61FB68DB437A6913407B61DB
S315080284203B685B6803F48013002B03D07A69FB6808
S3150802843013437B612B4A7B6913602A4B5B687B611A
S31508028440FB68DB437A6913407B613B685B6803F42C
S315080284500013002B03D07A69FB6813437B61214A18
S315080284607B6953601F4BD3F884307B61FB68DB431F
S315080284707A6913407B613B685B6803F40033002B1F
S3150802848003D07A69FB6813437B61164A7B69C2F893
S315080284908430144BD3F880307B61FB68DB437A69FE
S315080284A013407B613B685B6803F48033002B03D07F
S315080284B07A69FB6813437B610A4A7B69C2F8803092
S315080284C03B6901333B613B681A683B6922FA03F34D
S315080284D0002B7FF4C1AE00BF00BF1C37BD465DF856
S315080284E0047B7047002002447F7F2F0080B487B048
S315080284F000AF7860396000237B61A0E001227B69C6
S3150802850002FA03F33A6813403B613B69002B00F019
S315080285109380524A7B699B08183352F82330FB60D2
S315080285207B6903F00303DB000F2202FA03F3FA68FE
S315080285301340FB607B689A0A494B13407A6902F03A
S315080285400302D2009340FA689A4236D1434BD3F8D3
S3150802855080203B69DB4341491340C1F880303F4BD9
S31508028560D3F884203B69DB433C491340C1F8843085
S315080285703A4B1A683B69DB43384913400B60374B61
S315080285805A683B69DB43354913404B607B6903F004
S315080285900303DB000F2202FA03F3FB602F4A7B690F
S315080285A09B08183352F82310FB68DA432B487B6979
S315080285B09B080A40183340F823207B681A687B69AF
S315080285C05B00032101FA03F31A437B681A607B698D
S315080285D0DA087B68083253F822107B6903F007032E
S315080285E09B000F2202FA03F3DB437A69D208194089
S315080285F07B68083243F822107B689A687B695B00BD
S31508028600032101FA03F3DB431A407B689A607B680D
S315080286105A6801217B6901FA03F3DB431A407B6836
S315080286205A607B68DA687B695B00032101FA03F307
S31508028630DB431A407B68DA607B6901337B613A68FF
S315080286407B6922FA03F3002B7FF458AF00BF00BF01
S315080286501C37BD465DF8047B704700BF0020024404
S315080286607F7F2F0080B485B000AF78600B467B8091
S315080286707B681A697B881340002B02D00123FB739F
S3150802868001E00023FB73FB7B18461437BD465DF8F1
S31508028690047B704780B483B000AF78600B467B805A
S315080286A013467B707B78002B03D07A887B689A61A5
S315080286B002E07A887B689A6200BF0C37BD465DF88D
S315080286C0047B704780B485B000AF78600B467B8028
S315080286D07B685B69FB607A88FB6813401A04FB684F
S315080286E0D9437B880B401A437B689A6100BF1437CB
S315080286F0BD465DF8047B704780B584B000AF7860EC
S315080287007B68002B01D1012370E0786800F072F8CB
S315080287107B681B684CF6CC421A607B681B6845F27C
S3150802872055521A607B681B687A6852685A607B6879
S315080287301B687A6892689A60FEF728FAF8600FE072
S31508028740FEF724FA0246FB68D31A212B08D97B685E
S315080287501B68DB6803F00203002B01D0032345E004
S315080287607B681B68DB6803F00203002BE8D17B6891
S315080287701B69002B05D17B681B684FF480425A613E
S3150802878006E07B681A697B681B6842F440425A61B4
S31508028790FEF7FCF9F8600FE0FEF7F8F90246FB6807
S315080287A0D31A212B08D97B681B68DB6803F00F03F1
S315080287B0002B01D0032319E07B681B68DB6803F0F2
S315080287C00F03002BE8D17B681B681A697B68DB6894
S315080287D09A4205D07B681B687A68D2681A6104E0F7
S315080287E07B681B684AF6AA221A60002318461037C5
S315080287F0BD4680BD80B483B000AF786000BF0C3739
S31508028800BD465DF8047B704780B483B000AF7860DC
S315080288107B681B684AF6AA221A60002318460C3798
S31508028820BD465DF8047B704780B588B000AF7860B6
S315080288307B68002B02D1012300F028BC944BDB692C
S3150802884003F01803FB61924B9B6A03F00303BB61B7
S315080288507B681B6803F01003002B5BD0FB69082BAF
S3150802886005D0FB69182B14D1BB69022B11D17B6881
S31508028870DB69002B02D1012300F008BC844B9B69FB
S3150802888023F47C127B681B6A1B04814913438B61A0
S3150802889040E07B68DB69002B23D07D4B1B687C4A52
S315080288A043F480731360FEF771F9786108E0FEF706
S315080288B06DF902467B69D31A022B01D90323E5E334
S315080288C0734B1B6803F40073002BF0D0704B9B6943
S315080288D023F47C127B681B6A1B046D4913438B6164
S315080288E018E06B4B1B686A4A23F480731360FEF721
S315080288F04DF9786108E0FEF749F902467B69D31A11
S31508028900022B01D90323C1E3614B1B6803F40073ED
S31508028910002BF0D17B681B6803F00103002B00F0E3
S31508028920A080FB69102B05D0FB69182B09D1BB69FE
S31508028930032B06D17B685B68002B40F092800123EB
S31508028940A4E37B685B68B3F5803F06D1504B1B688E
S315080289504F4A43F48033136058E07B685B68002B08
S3150802896012D14B4B1B684A4A23F480331360484B97
S315080289701B68474A23F480131360454B1B68444A15
S3150802898023F48023136041E07B685B68B3F5A02F6C
S3150802899012D13F4B1B683E4A43F4802313603C4B7B
S315080289A01B683B4A23F480131360394B1B68384A09
S315080289B043F48033136029E07B685B68B3F5A81F2C
S315080289C012D1334B1B68324A43F480231360304B6F
S315080289D01B682F4A43F4801313602D4B1B682C4ADD
S315080289E043F48033136011E0294B1B68284A23F4A9
S315080289F080331360264B1B68254A23F480231360B1
S31508028A00234B1B68224A23F4801313607B685B6836
S31508028A10002B13D0FEF7BAF8786108E0FEF7B6F82D
S31508028A2002467B69D31A642B01D903232EE3184B1A
S31508028A301B6803F40033002BF0D012E0FEF7A6F809
S31508028A40786108E0FEF7A2F802467B69D31A642B1E
S31508028A5001D903231AE30E4B1B6803F40033002BD8
S31508028A60F0D17B681B6803F00203002B00F09A80A2
S31508028A70FB69002B05D0FB69182B49D1BB69012B71
S31508028A8046D17B68DB68002B04D10123FEE200BFD6
S31508028A90000C0244FB69002B1CD19A4B1B6803F09D
S31508028AA018027B681B699A4214D0964B1B6823F0FE
S31508028AB018027B681B69934913430B6000F0D0FDCB
S31508028AC0914B1B681846FCF76DFB0346002B01D039
S31508028AD00123DBE2FEF75AF8786108E0FEF756F85A
S31508028AE002467B69D31A022B01D90323CEE2854BB0
S31508028AF01B6803F00203002BF0D0824B1B6923F498
S31508028B00FE027B685B691B047E4913430B6149E0DD
S31508028B107B68DB68002B2CD07A4B1B6823F0180283
S31508028B207B681B69774913430B60764B1B68754A4A
S31508028B3043F001031360FEF729F8786108E0FEF7AF
S31508028B4025F802467B69D31A022B01D903239DE233
S31508028B506C4B1B6803F00203002BF0D0694B1B69B0
S31508028B6023F4FE027B685B691B04664913430B61A7
S31508028B7018E0644B1B68634A23F001031360FEF78F
S31508028B8005F8786108E0FEF701F802467B69D31A10
S31508028B90022B01D9032379E25A4B1B6803F002031D
S31508028BA0002BF0D17B681B6803F00803002B3CD02E
S31508028BB07B689B69002B1CD0524BD3F8F030514A84
S31508028BC043F08063C2F8F030FDF7E0FF786108E011
S31508028BD0FDF7DCFF02467B69D31A022B01D9032370
S31508028BE054E2484BD3F8F03003F00063002BEFD081
S31508028BF01BE0444BD3F8F030424A23F08063C2F8B4
S31508028C00F030FDF7C3FF786108E0FDF7BFFF0246C3
S31508028C107B69D31A022B01D9032337E2394BD3F8DE
S31508028C20F03003F00063002BEFD17B681B6803F07A
S31508028C300403002B00F0D280344B5B6A03F0010375
S31508028C40002B18D1314B5B6A304A43F00103536259
S31508028C50FDF79CFF786108E0FDF798FF02467B69FD
S31508028C60D31A022B01D9032310E2284B5B6A03F0BD
S31508028C700103002BF0D07B689B68012B08D1214B9E
S31508028C80D3F8F0301F4A43F00103C2F8F03074E01B
S31508028C907B689B68002B18D11A4BD3F8F030194A17
S31508028CA023F00103C2F8F030164BD3F8F030154A18
S31508028CB023F08003C2F8F030124BD3F8F030114A91
S31508028CC023F00403C2F8F03057E07B689B68052B53
S31508028CD01ED10C4BD3F8F0300A4A43F00403C2F80B
S31508028CE0F030084BD3F8F030064A23F08003C2F876
S31508028CF0F030044BD3F8F030024A43F00103C2F8CD
S31508028D00F0303AE0000C02449805002000080244BC
S31508028D107B689B68852B18D1A24BD3F8F030A14A01
S31508028D2043F00403C2F8F0309E4BD3F8F0309D4A64
S31508028D3043F08003C2F8F0309A4BD3F8F030994AE0
S31508028D4043F00103C2F8F03017E0964BD3F8F0303F
S31508028D50944A23F00103C2F8F030924BD3F8F0306C
S31508028D60904A23F00403C2F8F0308E4BD3F8F03061
S31508028D708C4A23F08003C2F8F0307B689B68002B8C
S31508028D8016D0FDF703FF78610AE0FDF7FFFE0246FB
S31508028D907B69D31A41F28832934201D9032375E1DA
S31508028DA0804BD3F8F03003F00203002BEDD015E028
S31508028DB0FDF7ECFE78610AE0FDF7E8FE02467B69FC
S31508028DC0D31A41F28832934201D903235EE1754BE5
S31508028DD0D3F8F03003F00203002BEDD17B681B6851
S31508028DE003F02003002B36D07B685B6A002B19D070
S31508028DF06C4B1B686B4A43F480531360FDF7C6FE3F
S31508028E00786108E0FDF7C2FE02467B69D31A022B97
S31508028E1001D903233AE1634B1B6803F40053002B81
S31508028E20F0D018E05F4B1B685E4A23F48053136048
S31508028E30FDF7ACFE786108E0FDF7A8FE02467B69FD
S31508028E40D31A022B01D9032320E1564B1B6803F4DC
S31508028E500053002BF0D17B689B6A002B00F015812A
S31508028E60FB69182B00F0AF807B689B6A022B40F0E7
S31508028E7086804C4B1B684B4A23F080731360FDF7C0
S31508028E8085FE786108E0FDF781FE02467B69D31A02
S31508028E90022B01D90323F9E0424B1B6803F0007346
S31508028EA0002BF0D13F4B9B6A23F47C5323F0030338
S31508028EB07A68D16A7A68126B12020A4339491343ED
S31508028EC08B627B685B6B013BC3F308027B689B6B17
S31508028ED0013B5B029BB21A437B68DB6B013B1B04BB
S31508028EE003F4FE031A437B681B6C013B1B0603F063
S31508028EF0FE432C4913434B632A4B9B6A294A23F0A8
S31508028F00100393627B68DB6C264ADB009363254B6E
S31508028F109B6A244A43F010039362224B9B6A23F00E
S31508028F200C027B685B6C1F4913438B621D4B9B6A61
S31508028F3023F020027B689B6C1A4913438B62194BF8
S31508028F409B6A184A43F480339362164B1B68154A88
S31508028F5043F080731360FDF719FE786108E0FDF7A8
S31508028F6015FE02467B69D31A022B01D903238DE02B
S31508028F700C4B1B6803F00073002BF0D085E0094BFD
S31508028F801B68084A23F080731360FDF7FFFD7861BA
S31508028F900AE0FDF7FBFD02467B69D31A022B03D9C9
S31508028FA0032373E0000C02443A4B1B6803F0007378
S31508028FB0002BEED1374B9B6A364A23F4E02323F083
S31508028FC00303936261E0334B9B6A3B61314B5B6BF4
S31508028FD0FB607B689B6A012B31D03B6903F0030275
S31508028FE07B68DB6A9A422AD13B691B0A03F03F0275
S31508028FF07B681B6B9A4222D1FB68C3F308027B6823
S315080290005B6B013B9A421AD1FB685B0A03F07F024B
S315080290107B689B6B013B9A4211D1FB681B0C03F0E0
S315080290207F027B68DB6B013B9A4208D1FB681B0E09
S3150802903003F07F027B681B6C013B9A4201D0012335
S3150802904024E0144B9B6BDB08C3F30C027B68DB6CD6
S315080290509A421AD00F4B9B6A0E4A23F01003936268
S31508029060FDF794FD786100BFFDF790FD02467B6926
S315080290709342F9D07B68DB6C064ADB009363054BA7
S315080290809B6A044A43F0100393620023184620376A
S31508029090BD4680BD000C024480B584B000AF78603E
S315080290A039607B68002B01D101239EE1834B1B6843
S315080290B003F00F033A689A4210D9804B1B6823F0D3
S315080290C00F027E493B6813430B607C4B1B6803F017
S315080290D00F033A689A4201D0012386E17B681B682E
S315080290E003F01003002B12D07B685A69744B1B6A73
S315080290F01B0A03F070039A4209D9714B1B6A23F4BF
S31508029100E0427B685B691B026D4913430B627B680D
S315080291101B6803F00803002B12D07B681A69684B98
S315080291201B6A1B0903F070039A4209D9644B1B6A2E
S3150802913023F4E0627B681B691B01614913430B62D6
S315080291407B681B6803F00403002B10D07B68DA687F
S315080291505B4B1B6A03F070039A4208D9584B1B6A89
S3150802916023F070027B68DB68554913430B627B6800
S315080291701B6803F00203002B10D07B689A68504BD9
S315080291801B6A03F00F039A4208D94D4B1B6A23F058
S315080291900F027B689B684A4913430B627B681B680C
S315080291A003F00103002B00F093807B685B68032BB6
S315080291B007D1434B1B6803F00073002B21D101230F
S315080291C013E17B685B68022B07D13D4B1B6803F4EE
S315080291D00033002B15D1012307E17B685B68012B5D
S315080291E007D1374B1B6803F40073002B09D10123FF
S315080291F0FBE0334B1B6803F00203002B01D101236A
S31508029200F3E02F4BDB6923F003027B685B682C498A
S315080292101343CB61FDF7BAFCF8607B685B68032BE6
S3150802922012D10AE0FDF7B2FC0246FB68D31A41F2F4
S315080292308832934201D90323D7E0214BDB6903F035
S315080292401803182BEED143E07B685B68022B12D118
S315080292500AE0FDF79BFC0246FB68D31A41F2883204
S31508029260934201D90323C0E0154BDB6903F01803C7
S31508029270102BEED12CE07B685B68012B22D10AE029
S31508029280FDF784FC0246FB68D31A41F28832934200
S3150802929001D90323A9E00A4BDB6903F01803082B5B
S315080292A0EED115E0FDF772FC0246FB68D31A41F2CD
S315080292B08832934206D9032397E000BF0020024072
S315080292C0000C02444B4BDB6903F01803002BE9D16F
S315080292D07B681B6803F00203002B10D07B689A6830
S315080292E0444B1B6A03F00F039A4208D2414B1B6A8E
S315080292F023F00F027B689B683E4913430B623E4B81
S315080293001B6803F00F033A689A4210D23A4B1B685D
S3150802931023F00F0238493B6813430B60364B1B6830
S3150802932003F00F033A689A4201D001235DE07B6895
S315080293301B6803F00403002B10D07B68DA682D4BF8
S315080293401B6A03F070039A4208D22A4B1B6A23F05F
S3150802935070027B68DB68274913430B627B681B68CC
S3150802936003F00803002B12D07B681A69214B1B6A8B
S315080293701B0903F070039A4209D21E4B1B6A23F497
S31508029380E0627B681B691B011A4913430B627B68FF
S315080293901B6803F01003002B12D07B685A69154B21
S315080293A01B6A1B0A03F070039A4209D2114B1B6A05
S315080293B023F4E0427B685B691B020E4913430B6286
S315080293C000F022F802460B4B1B6A03F00F030B4907
S315080293D0CB5C22FA03F30A4A13600A4B1B68184647
S315080293E0FBF7E0FE0346FB72FB7A18461037BD46CA
S315080293F080BD00BF000C024400200240F8B10308F9
S31508029400940500209805002080B489B000AF8C4BE3
S31508029410DB6903F01803082B02D18A4BFB6107E1CB
S31508029420874BDB6903F01803002B12D1844B1B68A8
S3150802943003F02003002B09D0814B1B68DB0803F0DD
S315080294400303814A22FA03F3FB61F1E07E4BFB61D7
S31508029450EEE07B4BDB6903F01803102B02D17B4B42
S31508029460FB61E5E0764BDB6903F01803182B40F045
S31508029470DD80734B9B6A03F003037B61704B9B6A27
S315080294801B0A03F03F033B616D4B9B6A1B0903F002
S315080294900103FB606A4B9B6BDB08C3F30C03FA6898
S315080294A002FB03F307EE903AF8EE677AC7ED027A03
S315080294B03B69002B00F0B7807B69012B03D07B69DF
S315080294C0032B56D077E05E4B1B6803F02003002B74
S315080294D02DD05B4B1B68DB0803F003035A4A22FABA
S315080294E003F37B607B6807EE903AF8EE676A3B699E
S315080294F007EE903AF8EE677A86EEA77A504B5B6BE0
S31508029500C3F3080307EE903AF8EE676A97ED026A24
S31508029510DFED4F5AC6EE257A76EEA77AF7EE006A9F
S3150802952077EEA67A67EE277AC7ED067A65E03B6993
S3150802953007EE903AF8EE677ADFED466A86EEA77A84
S315080295403F4B5B6BC3F3080307EE903AF8EE676A84
S3150802955097ED026ADFED3E5AC6EE257A76EEA77ACF
S31508029560F7EE006A77EEA67A67EE277AC7ED067AED
S3150802957043E03B6907EE903AF8EE677ADFED366A22
S3150802958086EEA77A2E4B5B6BC3F3080307EE903A77
S31508029590F8EE676A97ED026ADFED2D5AC6EE257A6E
S315080295A076EEA77AF7EE006A77EEA67A67EE277A5C
S315080295B0C7ED067A21E03B6907EE903AF8EE677A3C
S315080295C0DFED266A86EEA77A1D4B5B6BC3F30803AB
S315080295D007EE903AF8EE676A97ED026ADFED1C5AD3
S315080295E0C6EE257A76EEA77AF7EE006A77EEA67ABF
S315080295F067EE277AC7ED067A00BF114B5B6B5B0AEB
S3150802960003F07F0301333B603B6807EE903AB8EEFE
S31508029610677AD7ED066AC6EE877AFCEEE77A17EE20
S31508029620903AFB6104E00023FB6101E0064BFB6113
S31508029630FB6918462437BD465DF8047B704700BFB0
S31508029640000C024400093D000090D003001BB7003D
S31508029650000000460024744C001B374B0024744A51
S3150802966080B500AFFFF7D0FE0246084B1B6A03F02F
S315080296700F030749CB5C03F01F0322FA03F3054ADB
S315080296801360044B1B68184680BD00BF000C0244D9
S31508029690F8B103089405002080B500AFFFF7E0FF94
S315080296A00246064B1B6A1B0903F007030449CB5CF7
S315080296B003F01F0322FA03F3184680BD000C024486
S315080296C008B2030880B500AFFFF7CAFF0246064B89
S315080296D01B6A1B0A03F007030449CB5C03F01F034A
S315080296E022FA03F3184680BD000C024408B20308A6
S315080296F080B500AFFFF7B4FF0246064B1B6A1B0B89
S3150802970003F007030449CB5C03F01F0322FA03F3B1
S31508029710184680BD000C024408B2030880B485B01E
S3150802972000AF786039607B681F221A60154BDB69C7
S3150802973003F003027B685A60124B1B6AFB60FB68E4
S3150802974003F00F027B689A60FB6803F070027B687D
S31508029750DA60FB681B0903F070027B681A61FB6812
S315080297601B0A03F070027B685A61074B1B6803F0F9
S315080297700F023B681A6000BF1437BD465DF8047BCA
S31508029780704700BF000C0244002002402DE9B04F8A
S31508029790D8B000AFC7F84C01002387F85B31002325
S315080297A087F85A31D7F84C31D3E9002302F080748E
S315080297B0002554EA05030BD0CD4BD3F8E83023F045
S315080297C04041D7F84C319B6DC94A0B43C2F8E83081
S315080297D0D7F84C31D3E9002302F001084FF000090B
S315080297E058EA090342D0D7F84C31DB6D052B23D84A
S315080297F001A252F823F000BF419802081198020804
S3150802980025980208419802084198020841980208D8
S31508029810D7F84C310833184604F0DAFE034687F8BF
S315080298205B310EE0D7F84C313033184604F068FF46
S31508029830034687F85B3104E0012387F85B3100E0D1
S3150802984000BF97F85B31002B0CD1A94BD3F8D8305F
S3150802985023F00701D7F84C31DB6DA54A0B43C2F852
S31508029860D83003E097F85B3187F85A31D7F84C318C
S31508029870D3E9002302F0020A4FF0000B5AEA0B035F
S3150802988000F08880D7F84C311B6E282B68D801A2C5
S3150802989052F823F069990208619902086199020847
S315080298A06199020861990208619902086199020898
S315080298B061990208399902086199020861990208B0
S315080298C06199020861990208619902086199020878
S315080298D0619902084D99020861990208619902087C
S315080298E06199020861990208619902086199020858
S315080298F06199020869990208619902086199020840
S315080299006199020861990208619902086199020837
S31508029910619902086999020861990208619902081F
S315080299206199020861990208619902086199020817
S315080299306199020869990208D7F84C310833184622
S3150802994004F046FE034687F85B310EE0D7F84C3141
S315080299503033184604F0D4FE034687F85B3104E038
S31508029960012387F85B3100E000BF97F85B31002BD3
S315080299700CD15F4BD3F8D83023F03801D7F84C31E5
S315080299801B6E5B4A0B43C2F8D83003E097F85B318B
S3150802999087F85A31D7F84C31D3E9002302F0040389
S315080299A0C7F840310023C7F84431D7E950120B46AD
S315080299B013434ED0D7F84C315B6EB3F5A07F2CD04B
S315080299C0B3F5A07F25D8B3F5807F28D0B3F5807F7D
S315080299D01FD8C02B25D0C02B1BD8802B0FD0802B8D
S315080299E017D8002B1FD0402B13D1D7F84C31083388
S315080299F0184604F0EDFD034687F85B3114E0D7F804
S31508029A004C313033184604F07BFE034687F85B3147
S31508029A100AE0012387F85B3106E000BF04E000BFD5
S31508029A2002E000BF00E000BF97F85B31002B0CD1C3
S31508029A302F4BD3F8D83023F4E071D7F84C315B6E4C
S31508029A402B4A0B43C2F8D83003E097F85B3187F804
S31508029A505A31D7F84C31D3E9002302F00803C7F884
S31508029A6038310023C7F83C31D7E94E120B46134367
S31508029A7056D0D7F84C319B6EB3F5206F31D0B3F57B
S31508029A80206F2AD8B3F5006F2DD0B3F5006F24D80E
S31508029A90B3F5C06F29D0B3F5C06F1ED8B3F5806F82
S31508029AA011D0B3F5806F18D8002B23D0B3F5007FF9
S31508029AB013D1D7F84C310833184604F089FD03460A
S31508029AC087F85B3117E0D7F84C313033184604F083
S31508029AD017FE034687F85B310DE0012387F85B31F1
S31508029AE009E000BF07E000BF05E000BF03E000BFD2
S31508029AF0000C024400BF97F85B31002B0CD1BB4B1C
S31508029B00D3F8D83023F46061D7F84C319B6EB74A44
S31508029B100B43C2F8D83003E097F85B3187F85A311D
S31508029B20D7F84C31D3E9002302F01003C7F83031D5
S31508029B300023C7F83431D7E94C120B46134353D0E6
S31508029B40D7F84C31DB6EB3F5A04F31D0B3F5A04F41
S31508029B502AD8B3F5804F2DD0B3F5804F24D8B3F564
S31508029B60405F29D0B3F5405F1ED8B3F5005F11D028
S31508029B70B3F5005F18D8002B20D0B3F5805F13D158
S31508029B80D7F84C310833184604F022FD034687F805
S31508029B905B3114E0D7F84C313033184604F0B0FD87
S31508029BA0034687F85B310AE0012387F85B3106E052
S31508029BB000BF04E000BF02E000BF00E000BF97F864
S31508029BC05B31002B0CD1894BD3F8D83023F4E04112
S31508029BD0D7F84C31DB6E854A0B43C2F8D83003E01E
S31508029BE097F85B3187F85A31D7F84C31D3E9002315
S31508029BF002F02003C7F828310023C7F82C31D7E929
S31508029C004A120B46134353D0D7F84C311B6FB3F5A0
S31508029C10203F31D0B3F5203F2AD8B3F5003F2DD0E7
S31508029C20B3F5003F24D8B3F5C03F29D0B3F5C03FFA
S31508029C301ED8B3F5803F11D0B3F5803F18D8002B54
S31508029C4020D0B3F5004F13D1D7F84C310833184654
S31508029C5004F0BEFC034687F85B3114E0D7F84C31B2
S31508029C603033184604F04CFD034687F85B310AE0A8
S31508029C70012387F85B3106E000BF04E000BF02E07B
S31508029C8000BF00E000BF97F85B31002B0CD1574BA1
S31508029C90D3F8D83023F46031D7F84C311B6F534AC6
S31508029CA00B43C2F8D83003E097F85B3187F85A318C
S31508029CB0D7F84C31D3E9002302F04003C7F8203124
S31508029CC00023C7F82431D7E948120B46134353D069
S31508029CD0D7F84C315B6FB3F5A01F31D0B3F5A01F8F
S31508029CE02AD8B3F5801F2DD0B3F5801F24D8B3F533
S31508029CF0402F29D0B3F5402F1ED8B3F5002F11D027
S31508029D00B3F5002F18D8002B20D0B3F5802F13D126
S31508029D10D7F84C310833184604F05AFC034687F83C
S31508029D205B3114E0D7F84C313033184604F0E8FCBE
S31508029D30034687F85B310AE0012387F85B3106E0C0
S31508029D4000BF04E000BF02E000BF00E000BF97F8D2
S31508029D505B31002B0CD1254BD3F8D83023F4E01114
S31508029D60D7F84C315B6F214A0B43C2F8D83003E06F
S31508029D7097F85B3187F85A31D7F84C31D3E9002383
S31508029D8002F08003C7F818310023C7F81C31D7E957
S31508029D9046120B46134355D0D7F84C319B6FB3F591
S31508029DA0200F33D0B3F5200F2CD8B3F5000F2FD0E0
S31508029DB0B3F5000F26D8B3F5C00F2BD0B3F5C00FF5
S31508029DC020D8B3F5800F13D0B3F5800F1AD8002B1D
S31508029DD022D0B3F5001F15D1D7F84C3108331846EF
S31508029DE004F0F6FB034687F85B3116E0000C0244E2
S31508029DF0D7F84C313033184604F082FC034687F80C
S31508029E005B310AE0012387F85B3106E000BF04E014
S31508029E1000BF02E000BF00E000BF97F85B31002BED
S31508029E200CD1BB4BD3F8D83023F46001D7F84C31A8
S31508029E309B6FB74A0B43C2F8D83003E097F85B31F9
S31508029E4087F85A31D7F84C31D3E9002302F48073E4
S31508029E50C7F810310023C7F81431D7E944120B4664
S31508029E60134353D0D7F84C31DB6FB3F1A06F31D01F
S31508029E70B3F1A06F2AD8B3F1806F2DD0B3F1806FFA
S31508029E8024D8B3F1407F29D0B3F1407F1ED8B3F16D
S31508029E90007F11D0B3F1007F18D8002B20D0B3F180
S31508029EA0807F13D1D7F84C310833184604F090FB5B
S31508029EB0034687F85B3114E0D7F84C31303318463D
S31508029EC004F01EFC034687F85B310AE0012387F893
S31508029ED05B3106E000BF04E000BF02E000BF00E01D
S31508029EE000BF97F85B31002B0CD1894BD3F8D830D9
S31508029EF023F0E061D7F84C31DB6F854A0B43C2F891
S31508029F00D83003E097F85B3187F85A31D7F84C31E5
S31508029F10D3E9002302F40073C7F808310023C7F80F
S31508029F200C31D7E942120B46134355D0D7F84C31B8
S31508029F30D3F88030B3F1205F31D0B3F1205F2AD84D
S31508029F40B3F1005F2DD0B3F1005F24D8B3F1C05F3F
S31508029F5029D0B3F1C05F1ED8B3F1805F11D0B3F137
S31508029F60805F18D8002B20D0B3F1006F13D1D7F831
S31508029F704C310833184604F02BFB034687F85B314D
S31508029F8014E0D7F84C313033184604F0B9FB0346CF
S31508029F9087F85B310AE0012387F85B3106E000BFE8
S31508029FA004E000BF02E000BF00E000BF97F85B31A3
S31508029FB0002B0DD1564BD3F8D83023F06051D7F881
S31508029FC04C31D3F88030524A0B43C2F8D83003E0FA
S31508029FD097F85B3187F85A31D7F84C31D3E9002321
S31508029FE002F48063C7F800310023C7F80431D7E9C1
S31508029FF040120B46134344D0D7F84C31D3F8843079
S3150802A000052B23D801A252F823F000BF55A0020857
S3150802A01025A0020839A0020855A0020855A0020880
S3150802A02055A00208D7F84C310833184604F0D0FA7E
S3150802A030034687F85B310EE0D7F84C3130331846C1
S3150802A04004F05EFB034687F85B3104E0012387F8D8
S3150802A0505B3100E000BF97F85B31002B0DD12C4B2A
S3150802A060D3F8DC3023F00701D7F84C31D3F8843023
S3150802A070274A0B43C2F8DC3003E097F85B3187F8CE
S3150802A0805A31D7F84C31D3E9002302F40063C7F8F2
S3150802A090F8300023C7F8FC30D7E93E120B461343C3
S3150802A0A04FD0D7F84C31D3F88830502B29D0502BC3
S3150802A0B023D8402B27D0402B1FD8302B25D0302B26
S3150802A0C01BD8202B0FD0202B17D8002B22D0102BD1
S3150802A0D013D1D7F84C310833184604F079FA0346F7
S3150802A0E087F85B3117E0D7F84C313033184604F05D
S3150802A0F007FB034687F85B310DE0012387F85B31DE
S3150802A10009E000BF07E000BF05E000BF03E000BFAB
S3150802A110000C024400BF97F85B31002B0DD1AF4B00
S3150802A120D3F8DC3023F07001D7F84C31D3F88830F5
S3150802A130AA4A0B43C2F8DC3003E097F85B3187F88A
S3150802A1405A31D7F84C31D3E9002302F48053C7F8C1
S3150802A150F0300023C7F8F430D7E93C120B46134314
S3150802A16055D0D7F84C31D3F88C30B3F1A06F31D033
S3150802A170B3F1A06F2AD8B3F1806F2DD0B3F1806FF7
S3150802A18024D8B3F1407F29D0B3F1407F1ED8B3F16A
S3150802A190007F11D0B3F1007F18D8002B20D0B3F17D
S3150802A1A0807F13D1D7F84C310833184604F010FAD9
S3150802A1B0034687F85B3114E0D7F84C31303318463A
S3150802A1C004F09EFA034687F85B310AE0012387F812
S3150802A1D05B3106E000BF04E000BF02E000BF00E01A
S3150802A1E000BF97F85B31002B0DD17C4BD3F8E030DA
S3150802A1F023F0E061D7F84C31D3F88C30774A0B4319
S3150802A200C2F8E03003E097F85B3187F85A31D7F89D
S3150802A2104C31D3E9002302F40053C7F8E83000238F
S3150802A220C7F8EC30D7E93A120B4613433DD0D7F8B4
S3150802A2304C31D3F89030B3F5403F1BD0B3F5403FCD
S3150802A24014D8B3F5003F17D0B3F5003F0ED8002B4C
S3150802A25014D0B3F5803F09D1D7F84C3130331846BC
S3150802A26004F04EFA034687F85B3108E0012387F8C3
S3150802A2705B3104E000BF02E000BF00E000BF97F8D0
S3150802A2805B31002B0DD1554BD3F8E43023F4403122
S3150802A290D7F84C31D3F89030504A0B43C2F8E43021
S3150802A2A003E097F85B3187F85A31D7F84C31D3E98E
S3150802A2B0002302F48043C7F8E0300023C7F8E430ED
S3150802A2C0D7E938120B4613433DD0D7F84C31D3F8A9
S3150802A2D09430B3F5402F1BD0B3F5402F14D8B3F5FD
S3150802A2E0002F17D0B3F5002F0ED8002B14D0B3F5D4
S3150802A2F0802F09D1D7F84C313033184604F000FACA
S3150802A300034687F85B3108E0012387F85B3104E0EE
S3150802A31000BF02E000BF00E000BF97F85B31002BE8
S3150802A3200DD12E4BD3F8E43023F44021D7F84C3123
S3150802A330D3F89430294A0B43C2F8E43003E097F87D
S3150802A3405B3187F85A31D7F84C31D3E9002302F446
S3150802A3500043C7F8D8300023C7F8DC30D7E93612ED
S3150802A3600B46134340D0D7F84C31D3F89830B3F59F
S3150802A370401F1BD0B3F5401F14D8B3F5001F17D0E2
S3150802A380B3F5001F0ED8002B14D0B3F5801F09D1E0
S3150802A390D7F84C313033184604F0B2F9034687F839
S3150802A3A05B3108E0012387F85B3104E000BF02E075
S3150802A3B000BF00E000BF97F85B31002B10D1074BB6
S3150802A3C0D3F8E43023F44011D7F84C31D3F8983057
S3150802A3D0024A0B43C2F8E43006E000BF000C02440E
S3150802A3E097F85B3187F85A31D7F84C31D3E900230D
S3150802A3F00021C7F8D01003F48063C7F8D430D7E930
S3150802A40034120B4613433DD0D7F84C31D3F89C305F
S3150802A410B3F5400F1BD0B3F5400F14D8B3F5000FB0
S3150802A42017D0B3F5000F0ED8002B14D0B3F5800F52
S3150802A43009D1D7F84C313033184604F061F903468E
S3150802A44087F85B3108E0012387F85B3104E000BF37
S3150802A45002E000BF00E000BF97F85B31002B0DD188
S3150802A460BE4BD3F8E43023F44001D7F84C31D3F885
S3150802A4709C30BA4A0B43C2F8E43003E097F85B31E2
S3150802A48087F85A31D7F84C31D3E9002302F48033DE
S3150802A490C7F8C8300023C7F8CC30D7E932120B46C2
S3150802A4A0134335D0D7F84C31D3F8A030B3F1007F37
S3150802A4B015D0B3F1007F0ED8002B12D0B3F1807FEE
S3150802A4C009D1D7F84C313033184604F019F9034646
S3150802A4D087F85B3106E0012387F85B3102E000BFAB
S3150802A4E000E000BF97F85B31002B0DD19B4BD3F8E8
S3150802A4F0E43023F04071D7F84C31D3F8A030974AAC
S3150802A5000B43C2F8E43003E097F85B3187F85A3117
S3150802A510D7F84C31D3E900230021C7F8C01003F459
S3150802A5200063C7F8C430D7E930120B4613430ED07E
S3150802A5308A4BDB69894A23F40043D361874BD9697D
S3150802A540D7F84C31D3F80431844A0B43D361D7F890
S3150802A5504C31D3E9002302F40033C7F8B83000239C
S3150802A560C7F8BC30D7E92E120B46134355D0D7F895
S3150802A5704C31D3F8A430B3F5A06F31D0B3F5A06F40
S3150802A5802AD8B3F5806F2DD0B3F5806F24D8B3F5EA
S3150802A590407F29D0B3F5407F1ED8B3F5007F11D08E
S3150802A5A0B3F5007F18D8002B20D0B3F5807F13D1DE
S3150802A5B0D7F84C310833184604F00AF8034687F8E8
S3150802A5C05B3114E0D7F84C313033184604F098F86A
S3150802A5D0034687F85B310AE0012387F85B3106E018
S3150802A5E000BF04E000BF02E000BF00E000BF97F82A
S3150802A5F05B31002B0DD1594BD3F8DC3023F4E061E3
S3150802A600D7F84C31D3F8A430544A0B43C2F8DC309D
S3150802A61003E097F85B3187F85A31D7F84C31D3E91A
S3150802A620002302F48023C7F8B0300023C7F8B430F9
S3150802A630D7E92C120B46134355D0D7F84C31D3F829
S3150802A640A830B3F5A04F31D0B3F5A04F2AD8B3F549
S3150802A650804F2DD0B3F5804F24D8B3F5405F29D06B
S3150802A660B3F5405F1ED8B3F5005F11D0B3F5005FAE
S3150802A67018D8002B20D0B3F5805F13D1D7F84C3108
S3150802A6800833184603F0A4FF034687F85B3114E043
S3150802A690D7F84C313033184604F032F8034687F8B7
S3150802A6A05B310AE0012387F85B3106E000BF04E06C
S3150802A6B000BF02E000BF00E000BF97F85B31002B45
S3150802A6C00DD1264BD3F8DC3023F4E041D7F84C31D0
S3150802A6D0D3F8A830214A0B43C2F8DC3003E097F8D6
S3150802A6E05B3187F85A31D7F84C31D3E90023002178
S3150802A6F0C7F8A81003F02003C7F8AC30D7E92A1226
S3150802A7000B46134357D0D7F84C31D3F8AC30B3F5D0
S3150802A710A02F33D0B3F5A02F2CD8B3F5802F2FD086
S3150802A720B3F5802F26D8B3F5403F2BD0B3F5403F7B
S3150802A73020D8B3F5003F13D0B3F5003F1AD8002B43
S3150802A74022D0B3F5803F15D1D7F84C3108331846D5
S3150802A75003F03EFF034687F85B3116E0000C02441D
S3150802A760D7F84C313033184603F0CAFF034687F848
S3150802A7705B310AE0012387F85B3106E000BF04E09B
S3150802A78000BF02E000BF00E000BF97F85B31002B74
S3150802A7900DD1BB4BD3F8DC3023F4E021D7F84C318A
S3150802A7A0D3F8AC30B64A0B43C2F8DC3003E097F86C
S3150802A7B05B3187F85A31D7F84C31D3E900230021A7
S3150802A7C0C7F8A01003F04003C7F8A430D7E9281247
S3150802A7D00B46134355D0D7F84C31D3F8B030B3F5FE
S3150802A7E0A00F31D0B3F5A00F2AD8B3F5800F2DD01C
S3150802A7F0B3F5800F24D8B3F5401F29D0B3F5401F0F
S3150802A8001ED8B3F5001F11D0B3F5001F18D8002BB8
S3150802A81020D0B3F5801F13D1D7F84C310833184628
S3150802A82003F0D6FE034687F85B3114E0D7F84C31BD
S3150802A8303033184603F064FF034687F85B310AE0B3
S3150802A840012387F85B3106E000BF04E000BF02E09F
S3150802A85000BF00E000BF97F85B31002B0DD1884B93
S3150802A860D3F8DC3023F4E001D7F84C31D3F8B03012
S3150802A870834A0B43C2F8DC3003E097F85B3187F86A
S3150802A8805A31D7F84C31D3E900230021C7F898107A
S3150802A89003F08003C7F89C30D7E926120B46134308
S3150802A8A055D0D7F84C31D3F8B430B3F1A06F31D0C4
S3150802A8B0B3F1A06F2AD8B3F1806F2DD0B3F1806FB0
S3150802A8C024D8B3F1407F29D0B3F1407F1ED8B3F123
S3150802A8D0007F11D0B3F1007F18D8002B20D0B3F136
S3150802A8E0807F13D1D7F84C310833184603F070FE2F
S3150802A8F0034687F85B3114E0D7F84C3130331846F3
S3150802A90003F0FEFE034687F85B310AE0012387F867
S3150802A9105B3106E000BF04E000BF02E000BF00E0D2
S3150802A92000BF97F85B31002B0DD1554BD3F8DC30BD
S3150802A93023F0E061D7F84C31D3F8B430504A0B43D0
S3150802A940C2F8DC3003E097F85B3187F85A31D7F85A
S3150802A9504C31D3E900230021C7F8901003F4807321
S3150802A960C7F89430D7E924120B46134355D0D7F8C3
S3150802A9704C31D3F8B830B3F1A04F31D0B3F1A04F70
S3150802A9802AD8B3F1804F2DD0B3F1804F24D8B3F132
S3150802A990405F29D0B3F1405F1ED8B3F1005F11D0F2
S3150802A9A0B3F1005F18D8002B20D0B3F1805F13D122
S3150802A9B0D7F84C310833184603F00AFE034687F8DF
S3150802A9C05B3114E0D7F84C313033184603F098FE61
S3150802A9D0034687F85B310AE0012387F85B3106E014
S3150802A9E000BF04E000BF02E000BF00E000BF97F826
S3150802A9F05B31002B0DD1224BD3F8DC3023F0E0413A
S3150802AA00D7F84C31D3F8B8301D4A0B43C2F8DC30BC
S3150802AA1003E097F85B3187F85A31D7F84C31D3E916
S3150802AA20002302F40023C7F888300023C7F88C30C5
S3150802AA30D7E922120B46134355D0D7F84C31D3F82F
S3150802AA40C030B3F5802F35D0B3F5802F2ED8B3F5A5
S3150802AA50403F31D0B3F5403F28D8B3F5003F1BD06D
S3150802AA60B3F5003F22D8002B03D0B3F5803F09D0B7
S3150802AA701CE0034B9B6A024A43F4003393621CE0D0
S3150802AA80000C0244D7F84C310833184603F0A0FDEF
S3150802AA90034687F85B3110E0D7F84C313033184655
S3150802AAA003F02EFE034687F85B3106E0012387F89A
S3150802AAB05B3102E000BF00E000BF97F85B31002B74
S3150802AAC00DD1C34BD3F8E83023F4E021D7F84C3143
S3150802AAD0D3F8C030BE4A0B43C2F8E83003E097F811
S3150802AAE05B3187F85A31D7F84C31D3E9002302F49F
S3150802AAF08013C7F880300023C7F88430D7E92012BC
S3150802AB000B46134351D0D7F84C31D3F8C430B3F5BA
S3150802AB10001F33D0B3F5001F2CD8B3F5C01F2DD0B4
S3150802AB20B3F5C01F26D8B3F5801F19D0B3F5801F19
S3150802AB3020D8002B03D0B3F5002F07D01AE0A44B78
S3150802AB409B6AA34A43F40033936218E0D7F84C3160
S3150802AB500833184603F03CFD034687F85B310EE0DE
S3150802AB60D7F84C313033184603F0CAFD034687F846
S3150802AB705B3104E0012387F85B3100E000BF97F8F8
S3150802AB805B31002B0DD1924BD3F8E83023F46011D8
S3150802AB90D7F84C31D3F8C4308D4A0B43C2F8E830A3
S3150802ABA003E097F85B3187F85A31D7F84C31D3E985
S3150802ABB0002302F40013BB670023FB67D7E91E12C2
S3150802ABC00B46134332D0D7F84C31D3F8D430052B81
S3150802ABD00FD8032B11D2012B11D9022B09D1D7F881
S3150802ABE04C310833184603F0F3FC034687F85B3109
S3150802ABF006E0012387F85B3102E000BF00E000BFF0
S3150802AC0097F85B31002B0DD1714BD3F8E83023F05E
S3150802AC100701D7F84C31D3F8D4306D4A0B43C2F842
S3150802AC20E83003E097F85B3187F85A31D7F84C31A8
S3150802AC30D3E900230021396703F400737B67D7E958
S3150802AC401C120B46134324D0D7F84C31D3F8D8300C
S3150802AC50002B05D0082B05D0012387F85B3102E0CB
S3150802AC6000BF00E000BF97F85B31002B0DD1584BAF
S3150802AC70D3F8E83023F00801D7F84C31D3F8D830A6
S3150802AC80534A0B43C2F8E83003E097F85B3187F87A
S3150802AC905A31D7F84C31D3E9002302F00073BB6668
S3150802ACA00023FB66D7E91A120B46134300F0B98054
S3150802ACB0484B5B6A474A43F001035362FBF766FF58
S3150802ACC0C7F854010BE0FBF761FF0246D7F8543187
S3150802ACD0D31A022B03D9032387F85B3105E03D4BD0
S3150802ACE05B6A03F00103002BEDD097F85B31002B6A
S3150802ACF040F09380364BD3F8F03003F44073C7F82C
S3150802AD005C31D7F85C31002B23D0D7F84C31D3F815
S3150802AD10F820D7F85C3193421BD02D4BD3F8F0308C
S3150802AD2023F44073C7F85C31294BD3F8F030284A2C
S3150802AD3043F48033C2F8F030254BD3F8F030244A76
S3150802AD4023F48033C2F8F030214AD7F85C31C2F8CE
S3150802AD50F030D7F85C3103F00103002B19D0FBF76A
S3150802AD6015FFC7F854010DE0FBF710FF0246D7F8A6
S3150802AD705431D21A41F288339A4203D9032387F807
S3150802AD805B3106E0124BD3F8F03003F00203002BD6
S3150802AD90EAD097F85B31002B3AD1D7F84C31D3F881
S3150802ADA0F83003F44073B3F5407F15D1084BDB69DD
S3150802ADB023F47C51D7F84C31D3F8F8301B0923F029
S3150802ADC07F4323F03003024A0B43D3610AE000BFF4
S3150802ADD0000C0244000802449F4BDB699E4A23F496
S3150802ADE07C53D3619C4BD3F8F0309B4A23F44073CF
S3150802ADF0C2F8F030984BD3F8F010D7F84C31D3F8A4
S3150802AE00F830C3F30B03944A0B43C2F8F03008E058
S3150802AE1097F85B3187F85A3103E097F85B3187F880
S3150802AE205A31D7F84C31D3E9002302F080633B66E6
S3150802AE3000237B66D7E918120B46134335D0D7F899
S3150802AE404C31D3F8C830302B14D0302B0ED8202BE7
S3150802AE5012D0202B0AD8002B10D0102B06D17E4BED
S3150802AE609B6A7D4A43F40033936208E0012387F81C
S3150802AE705B3104E000BF02E000BF00E000BF97F8C4
S3150802AE805B31002B0DD1744BD3F8E83023F0300137
S3150802AE90D7F84C31D3F8C8306F4A0B43C2F8E830BA
S3150802AEA003E097F85B3187F85A31D7F84C31D3E982
S3150802AEB0002302F48003BB650023FB65D7E916125B
S3150802AEC00B46134333D0D7F84C31D3F8CC30002B8A
S3150802AED002D0402B07D010E05F4B9B6A5E4A43F4D0
S3150802AEE0003393620DE0D7F84C310833184603F065
S3150802AEF06FFB034687F85B3103E0012387F85B3172
S3150802AF0000BF97F85B31002B0DD1534BD3F8E430D1
S3150802AF1023F04001D7F84C31D3F8CC304E4A0B43D4
S3150802AF20C2F8E43003E097F85B3187F85A31D7F86C
S3150802AF304C31D3E9002302F400033B6500237B6509
S3150802AF40D7E914120B46134333D0D7F84C31D3F84A
S3150802AF50D030002B02D0802B07D010E03E4B9B6AE4
S3150802AF603D4A43F4003393620DE0D7F84C31083377
S3150802AF70184603F02DFB034687F85B3103E00123ED
S3150802AF8087F85B3100BF97F85B31002B0DD1324B46
S3150802AF90D3F8E43023F08001D7F84C31D3F8D03017
S3150802AFA02D4A0B43C2F8E43003E097F85B3187F881
S3150802AFB05A31D7F84C31D3E9002302F00063BB6457
S3150802AFC00023FB64D7E912120B4613434AD0D7F87B
S3150802AFD04C31D3F8E030042B27D801A252F823F0DB
S3150802AFE0F5AF020803B0020817B0020833B0020828
S3150802AFF033B00208184B9B6A174A43F4003393622C
S3150802B00018E0D7F84C310833184603F0E1FA03463C
S3150802B01087F85B310EE0D7F84C313033184603F027
S3150802B0206FFB034687F85B3104E0012387F85B313F
S3150802B03000E000BF97F85B31002B0FD1064BD3F81F
S3150802B040E03023F00701D7F84C31D3F8E030024A52
S3150802B0500B43C2F8E03005E0000C024497F85B3176
S3150802B06087F85A31D7F84C31D3E9002302F08053D6
S3150802B0703B6400237B64D7E910120B46134300F0A6
S3150802B0808180D7F84C31D3F8E430202B5FD801A25F
S3150802B09052F823F019B102084FB102084FB102085B
S3150802B0A04FB102084FB102084FB102084FB1020868
S3150802B0B04FB1020827B102084FB102084FB1020880
S3150802B0C04FB102084FB102084FB102084FB1020848
S3150802B0D04FB102083BB102084FB102084FB102084C
S3150802B0E04FB102084FB102084FB102084FB1020828
S3150802B0F04FB1020857B102084FB102084FB1020810
S3150802B1004FB102084FB102084FB102084FB1020807
S3150802B1104FB1020857B10208AB4B9B6AAA4A43F4DD
S3150802B1200033936218E0D7F84C310833184603F017
S3150802B1304FFA034687F85B310EE0D7F84C313033C5
S3150802B140184603F0DDFA034687F85B3104E001236B
S3150802B15087F85B3100E000BF97F85B31002B0DD111
S3150802B160994BD3F8E03023F03801D7F84C31D3F8AD
S3150802B170E430954A0B43C2F8E03003E097F85B31B6
S3150802B18087F85A31D7F84C31D3E9002302F0005335
S3150802B190BB630023FB63D7E90E120B4613434ED05B
S3150802B1A0D7F84C31D3F8E830B3F5807F2ED0B3F513
S3150802B1B0807F27D8C02B2BD0C02B23D8802B17D023
S3150802B1C0802B1FD8002B02D0402B07D01AE07E4BCB
S3150802B1D09B6A7D4A43F4003393621AE0D7F84C31EE
S3150802B1E00833184603F0F4F9034687F85B3110E092
S3150802B1F0D7F84C313033184603F082FA034687F8FB
S3150802B2005B3106E0012387F85B3102E000BF00E00C
S3150802B21000BF97F85B31002B0DD16B4BD3F8E030AA
S3150802B22023F4E071D7F84C31D3F8E830664A0B4379
S3150802B230C2F8E03003E097F85B3187F85A31D7F85D
S3150802B2404C31D3E9002302F080433B6300237B633E
S3150802B250D7E90C120B46134355D0D7F84C31D3F81D
S3150802B260EC30B3F5206F31D0B3F5206F2AD8B3F599
S3150802B270006F2DD0B3F5006F24D8B3F5C06F29D06F
S3150802B280B3F5C06F1ED8B3F5806F11D0B3F5806FD2
S3150802B29018D8002B20D0B3F5007F13D1D7F84C313C
S3150802B2A00833184603F094F9034687F85B3114E02D
S3150802B2B0D7F84C313033184603F022FA034687F89A
S3150802B2C05B310AE0012387F85B3106E000BF04E040
S3150802B2D000BF02E000BF00E000BF97F85B31002B19
S3150802B2E00DD1394BD3F8E03023F46061D7F84C31ED
S3150802B2F0D3F8EC30344A0B43C2F8E03003E097F84F
S3150802B3005B3187F85A31D7F84C31D3E9002302F07A
S3150802B3100043BB620023FB62D7E90A120B461343BA
S3150802B32058D0D7F84C31D3F8F030B3F5A04F31D016
S3150802B330B3F5A04F2AD8B3F5804F2DD0B3F5804F79
S3150802B34024D8B3F5405F29D0B3F5405F1ED8B3F5CC
S3150802B350005F11D0B3F5005F18D8002B20D0B3F5E3
S3150802B360805F13D1D7F84C310833184603F030F909
S3150802B370034687F85B3114E0D7F84C313033184668
S3150802B38003F0BEF9034687F85B310AE0012387F822
S3150802B3905B3106E000BF04E000BF02E000BF00E048
S3150802B3A000BF97F85B31002B10D1074BD3F8E0307A
S3150802B3B023F4E042D7F84C31D3F8F030024913436C
S3150802B3C0C1F8E03006E000BF000C024497F85B3192
S3150802B3D087F85A31D7F84C31D3E90023002139626C
S3150802B3E003F001037B62D7E908120B46134355D0D3
S3150802B3F0D7F84C31D3F8F430B3F5203F31D0B3F552
S3150802B400203F2AD8B3F5003F2DD0B3F5003F24D804
S3150802B410B3F5C03F29D0B3F5C03F1ED8B3F5803F78
S3150802B42011D0B3F5803F18D8002B20D0B3F5004FC2
S3150802B43013D1D7F84C310833184603F0C9F8034636
S3150802B44087F85B3114E0D7F84C313033184603F0ED
S3150802B45057F9034687F85B310AE0012387F85B311F
S3150802B46006E000BF04E000BF02E000BF00E000BF44
S3150802B47097F85B31002B0DD1884BD3F8E03023F4D3
S3150802B4806032D7F84C31D3F8F43084491343C1F803
S3150802B490E03003E097F85B3187F85A31D7F84C3138
S3150802B4A0D3E900230021B96103F00203FB61D7E95E
S3150802B4B006120B4613433DD0D7F84C31D3F8DC308D
S3150802B4C0032B1CD801A252F823F000BF07B50208C5
S3150802B4D0DDB40208EBB4020807B502086F4B9B6A93
S3150802B4E06E4A43F4003393620EE0D7F84C310833C0
S3150802B4F0184603F06DF8034687F85B3104E001232A
S3150802B50087F85B3100E000BF97F85B31002B0DD15D
S3150802B510624BD3F8E43023F00302D7F84C31D3F860
S3150802B520DC305E491343C1F8E43003E097F85B3137
S3150802B53087F85A31D7F84C31D3E90023002139610B
S3150802B54003F004037B61D7E904120B4613433AD08E
S3150802B550D7F84C31D3F8BC30B3F5007F0ED0B3F52B
S3150802B560007F15D8002B17D0B3F5807F10D14B4B2F
S3150802B5709B6A4A4A43F4003393620EE0D7F84C3189
S3150802B5800833184603F024F8034687F85B3104E0CB
S3150802B590012387F85B3100E000BF97F85B31002B87
S3150802B5A00DD13E4BD3F8E83023F44072D7F84C312C
S3150802B5B0D3F8BC3039491343C1F8E83003E097F8A9
S3150802B5C05B3187F85A31D7F84C31D3E90023002189
S3150802B5D0B96003F01003FB60D7E902120B46134366
S3150802B5E038D0D7F84C31D3F80031302B1BD0302B5A
S3150802B5F015D8102B02D0202B07D010E0274B9B6AB8
S3150802B600264A43F4003393620EE0D7F84C313033BE
S3150802B610184603F075F8034687F85B3104E0012300
S3150802B62087F85B3100E000BF97F85B31002B0DD13C
S3150802B6301A4BD3F8E43023F03002D7F84C31D3F85A
S3150802B640003116491343C1F8E43003E097F85B3139
S3150802B65087F85A31D7F84C31D3E9002300213960EB
S3150802B66003F008037B60D7E900120B4613430CD09C
S3150802B6700A4BD3F8E83023F0C002D7F84C31D3F896
S3150802B680FC3006491343C1F8E83097F85A31184690
S3150802B69007F5B077BD46BDE8B08F00BF000C02447F
S3150802B6A080B48BB000AF7860AD4B5B6BC3F3080315
S3150802B6B03B62AB4B9B6A03F00303FB61A84B9B6A95
S3150802B6C01B0A03F03F03BB61A54B9B6A03F01003F9
S3150802B6D07B61A34B9B6BDB08C3F30C037A6902FB02
S3150802B6E003F307EE903AF8EE677AC7ED047ABB6978
S3150802B6F0002B00F02681FB69032B53D0FB69032B31
S3150802B7006FD8FB69012B03D0FB69022B2BD068E0AB
S3150802B710934B1B68DB0803F00303924A22FA03F3EE
S3150802B720FB60FB6807EE903AF8EE676ABB6907EEBC
S3150802B730903AF8EE677A86EEA77A3B6A07EE903A6F
S3150802B740F8EE676A97ED046ADFED875AC6EE257A40
S3150802B75076EEA77AF7EE006A77EEA67A67EE277A8A
S3150802B760C7ED097A68E0BB6907EE903AF8EE677AA0
S3150802B770DFED7E6A86EEA77A3B6A07EE903AF8EE26
S3150802B780676A97ED046ADFED785AC6EE257A76EE91
S3150802B790A77AF7EE006A77EEA67A67EE277AC7EDFA
S3150802B7A0097A49E0BB6907EE903AF8EE677ADFED67
S3150802B7B0706A86EEA77A3B6A07EE903AF8EE676AEF
S3150802B7C097ED046ADFED685AC6EE257A76EEA77A11
S3150802B7D0F7EE006A77EEA67A67EE277AC7ED097A58
S3150802B7E02AE05F4B1B68DB0803F003035D4A22FA73
S3150802B7F003F3FB60FB6807EE903AF8EE676ABB69EB
S3150802B80007EE903AF8EE677A86EEA77A3B6A07EE73
S3150802B810903AF8EE676A97ED046ADFED535AC6EE78
S3150802B820257A76EEA77AF7EE006A77EEA67A67EEBB
S3150802B830277AC7ED097A00BF494B1B6803F00073E4
S3150802B840B3F1007F21D1464B9B6A03F48033002B68
S3150802B85017D0434B5B6B5B0A03F07F0307EE903A04
S3150802B860F8EE677AB7EE007A37EE877AD7ED096A85
S3150802B870C6EE877AFCEEE77A17EE902A7B681A609C
S3150802B88006E07B6800221A6002E07B6800221A60E2
S3150802B890334B1B6803F00073B3F1007F21D1304BA1
S3150802B8A09B6A03F40033002B17D02D4B5B6B1B0CE2
S3150802B8B003F07F0307EE903AF8EE677AB7EE007A5E
S3150802B8C037EE877AD7ED096AC6EE877AFCEEE77A0B
S3150802B8D017EE902A7B685A6006E07B6800225A6057
S3150802B8E002E07B6800225A601D4B1B6803F0007356
S3150802B8F0B3F1007F21D11A4B9B6A03F48023002BF4
S3150802B90017D0174B5B6B1B0E03F07F0307EE903ABB
S3150802B910F8EE677AB7EE007A37EE877AD7ED096AD4
S3150802B920C6EE877AFCEEE77A17EE902A7B689A606B
S3150802B93010E07B6800229A600CE07B6800229A601D
S3150802B94008E07B6800221A607B6800225A607B68DE
S3150802B95000229A6000BF2C37BD465DF8047B70470B
S3150802B960000C02440090D003000000460024744AEA
S3150802B970001B374B80B48BB000AF7860AD4BDB6BE6
S3150802B980C3F308033B62AB4BDB6A03F00303FB61B9
S3150802B990A84BDB6A1B0A03F03F03BB61A54BDB6AB4
S3150802B9A003F010037B61A34B1B6CDB08C3F30C0388
S3150802B9B07A6902FB03F307EE903AF8EE677AC7ED67
S3150802B9C0047ABB69002B00F02681FB69032B53D04E
S3150802B9D0FB69032B6FD8FB69012B03D0FB69022B8A
S3150802B9E02BD068E0934B1B68DB0803F00303924AEB
S3150802B9F022FA03F3FB60FB6807EE903AF8EE676AF1
S3150802BA00BB6907EE903AF8EE677A86EEA77A3B6A42
S3150802BA1007EE903AF8EE676A97ED046ADFED875A01
S3150802BA20C6EE257A76EEA77AF7EE006A77EEA67A5A
S3150802BA3067EE277AC7ED097A68E0BB6907EE903A9E
S3150802BA40F8EE677ADFED7E6A86EEA77A3B6A07EE3C
S3150802BA50903AF8EE676A97ED046ADFED785AC6EE11
S3150802BA60257A76EEA77AF7EE006A77EEA67A67EE79
S3150802BA70277AC7ED097A49E0BB6907EE903AF8EEEC
S3150802BA80677ADFED706A86EEA77A3B6A07EE903A26
S3150802BA90F8EE676A97ED046ADFED685AC6EE257A0C
S3150802BAA076EEA77AF7EE006A77EEA67A67EE277A37
S3150802BAB0C7ED097A2AE05F4B1B68DB0803F003032C
S3150802BAC05D4A22FA03F3FB60FB6807EE903AF8EE4A
S3150802BAD0676ABB6907EE903AF8EE677A86EEA77A46
S3150802BAE03B6A07EE903AF8EE676A97ED046ADFED6D
S3150802BAF0535AC6EE257A76EEA77AF7EE006A77EEFD
S3150802BB00A67A67EE277AC7ED097A00BF494B1B6802
S3150802BB1003F00063B3F1006F21D1464BDB6A03F4ED
S3150802BB208033002B17D0434BDB6B5B0A03F07F0392
S3150802BB3007EE903AF8EE677AB7EE007A37EE877A2A
S3150802BB40D7ED096AC6EE877AFCEEE77A17EE902AEF
S3150802BB507B681A6006E07B6800221A6002E07B684E
S3150802BB6000221A60334B1B6803F00063B3F1006FBF
S3150802BB7021D1304BDB6A03F40033002B17D02D4B4F
S3150802BB80DB6B1B0C03F07F0307EE903AF8EE677A3D
S3150802BB90B7EE007A37EE877AD7ED096AC6EE877A64
S3150802BBA0FCEEE77A17EE902A7B685A6006E07B6815
S3150802BBB000225A6002E07B6800225A601D4B1B680D
S3150802BBC003F00063B3F1006F21D11A4BDB6A03F469
S3150802BBD08023002B17D0174BDB6B1B0E03F07F035A
S3150802BBE007EE903AF8EE677AB7EE007A37EE877A7A
S3150802BBF0D7ED096AC6EE877AFCEEE77A17EE902A3F
S3150802BC007B689A6010E07B6800229A600CE07B6889
S3150802BC1000229A6008E07B6800221A607B6800228C
S3150802BC205A607B6800229A6000BF2C37BD465DF8D1
S3150802BC30047B7047000C02440090D00300000046C3
S3150802BC400024744A001B374B80B48BB000AF78606F
S3150802BC50AD4B5B6CC3F308033B62AB4B1B6B03F048
S3150802BC600303FB61A84B1B6B1B0A03F03F03BB6173
S3150802BC70A54B1B6B03F010037B61A34B9B6CDB0884
S3150802BC80C3F30C037A6902FB03F307EE903AF8EE64
S3150802BC90677AC7ED047ABB69002B00F02681FB6937
S3150802BCA0032B53D0FB69032B6FD8FB69012B03D0F7
S3150802BCB0FB69022B2BD068E0934B1B68DB0803F069
S3150802BCC00303924A22FA03F3FB60FB6807EE903AF3
S3150802BCD0F8EE676ABB6907EE903AF8EE677A86EE7F
S3150802BCE0A77A3B6A07EE903AF8EE676A97ED046A16
S3150802BCF0DFED875AC6EE257A76EEA77AF7EE006A60
S3150802BD0077EEA67A67EE277AC7ED097A68E0BB6905
S3150802BD1007EE903AF8EE677ADFED7E6A86EEA77A44
S3150802BD203B6A07EE903AF8EE676A97ED046ADFED2A
S3150802BD30785AC6EE257A76EEA77AF7EE006A77EE95
S3150802BD40A67A67EE277AC7ED097A49E0BB6907EE54
S3150802BD50903AF8EE677ADFED706A86EEA77A3B6A62
S3150802BD6007EE903AF8EE676A97ED046ADFED685ACD
S3150802BD70C6EE257A76EEA77AF7EE006A77EEA67A07
S3150802BD8067EE277AC7ED097A2AE05F4B1B68DB085C
S3150802BD9003F003035D4A22FA03F3FB60FB6807EE2E
S3150802BDA0903AF8EE676ABB6907EE903AF8EE677A58
S3150802BDB086EEA77A3B6A07EE903AF8EE676A97ED3F
S3150802BDC0046ADFED535AC6EE257A76EEA77AF7EEBF
S3150802BDD0006A77EEA67A67EE277AC7ED097A00BF78
S3150802BDE0494B1B6803F00053B3F1005F21D1464B60
S3150802BDF01B6B03F48033002B17D0434B5B6C5B0A37
S3150802BE0003F07F0307EE903AF8EE677AB7EE007A08
S3150802BE1037EE877AD7ED096AC6EE877AFCEEE77AB5
S3150802BE2017EE902A7B681A6006E07B6800221A6081
S3150802BE3002E07B6800221A60334B1B6803F000534A
S3150802BE40B3F1005F21D1304B1B6B03F40033002B97
S3150802BE5017D02D4B5B6C1B0C03F07F0307EE903A51
S3150802BE60F8EE677AB7EE007A37EE877AD7ED096A7F
S3150802BE70C6EE877AFCEEE77A17EE902A7B685A6056
S3150802BE8006E07B6800225A6002E07B6800225A605C
S3150802BE901D4B1B6803F00053B3F1005F21D11A4B07
S3150802BEA01B6B03F48023002B17D0174B5B6C1B0EFE
S3150802BEB003F07F0307EE903AF8EE677AB7EE007A58
S3150802BEC037EE877AD7ED096AC6EE877AFCEEE77A05
S3150802BED017EE902A7B689A6010E07B6800229A60C7
S3150802BEE00CE07B6800229A6008E07B6800221A60F0
S3150802BEF07B6800225A607B6800229A6000BF2C3752
S3150802BF00BD465DF8047B7047000C02440090D003DE
S3150802BF10000000460024744A001B374B90B58FB0C8
S3150802BF2000AFC7E90001D7E9000100F17E442143C9
S3150802BF3050D1264BD3F8F03003F440733B63234BBE
S3150802BF40D3F8F03003F00203022B08D13B6BB3F5AA
S3150802BF50807F04D14FF400437B6302F02ABB1B4B5C
S3150802BF60D3F8F03003F00063B3F1006F08D13B6BEE
S3150802BF70B3F5007F04D14FF4FA437B6302F019BB91
S3150802BF80124B1B6803F40033B3F5003F19D13B6B20
S3150802BF90B3F5407F15D10D4BDB6903F47C53B3F53A
S3150802BFA0007F0AD3094BDB691B0A03F03F03084AE1
S3150802BFB0B2FBF3F37B6302F0FCBA00237B6302F065
S3150802BFC0F8BA00237B6302F0F4BA00BF000C0244FD
S3150802BFD0001BB700D7E90001A1F5806450EA040105
S3150802BFE001F07582D7E90001012871F5806182F0B6
S3150802BFF0DD82D7E90001A1F5007450EA040101F0D7
S3150802C0006C81D7E90001012871F5007182F0CE82B0
S3150802C010D7E90001A1F5807450EA040101F002860D
S3150802C020D7E90001012871F5807182F0BF82D7E94C
S3150802C0300001A1F1800450EA040101F04C85D7E918
S3150802C0400001012871F1800182F0B082D7E900016E
S3150802C050A1F1400450EA040101F09E84D7E90001E7
S3150802C060012871F1400182F0A182D7E90001A1F10C
S3150802C070200450EA040101F0E883D7E90001012807
S3150802C08071F1200182F09282D7E90001A1F1100430
S3150802C09050EA040102F05682D7E90001012871F13B
S3150802C0A0100182F08382D7E90001A1F1080450EA5F
S3150802C0B0040102F0CC81D7E90001012871F10801D7
S3150802C0C082F07482D7E900010C1F50EA040101F0DC
S3150802C0D04886D7E90001012871F1040182F06682D7
S3150802C0E0D7E900018C1E50EA040102F04381D7E920
S3150802C0F00001012871F1020182F05882D7E9000194
S3150802C1004C1E50EA040102F0CE80D7E9000101284C
S3150802C11071F1010182F04A82D7E9000100F1004477
S3150802C120214302F05980D7E90001D94CA04271F1A6
S3150802C130000182F03B82D7E9000100F14044214325
S3150802C14001F0D987D7E90001D24CA04271F100016A
S3150802C15082F02C82D7E9000100F16044214301F004
S3150802C1605187D7E90001CC4CA04271F1000182F057
S3150802C1701D82D7E9000100F17044214301F09A8635
S3150802C180D7E90001C54CA04271F1000182F00E8286
S3150802C190D7E9000100F17844214301F01286D7E974
S3150802C1A00001BF4CA04271F1000182F0FF81D7E97C
S3150802C1B0000100F17C44214302F07E81D7E90001A7
S3150802C1C0B84CA04271F1000182F0F081D7E9000172
S3150802C1D0A0F50004214300F09E82D7E90001B24C83
S3150802C1E0A04271F1000182F0E181D7E90001A0F5D0
S3150802C1F08004214300F06D82D7E90001AB4CA042CE
S3150802C20071F1000182F0D281D7E90001A0F500148C
S3150802C210214301F00D80D7E90001A54CA04271F136
S3150802C220000182F0C381D7E90001A0F580142143F9
S3150802C23000F0D081D7E900019E4CA04271F10001BD
S3150802C24082F0B481D7E90001A0F50024214300F069
S3150802C2504281D7E90001984CA04271F1000182F0AF
S3150802C260A581D7E90001A0F58024214301F04E8279
S3150802C270D7E90001914CA04271F1000182F0968142
S3150802C280D7E90001A0F50034214301F09781D7E9E7
S3150802C29000018B4CA04271F1000182F08781D7E937
S3150802C2A00001A0F58034214301F05481D7E9000149
S3150802C2B0B0F1011F71F1000182F07881D7E900011E
S3150802C2C0A0F50044214301F0B780D7E9000148F2FE
S3150802C2D00104A04271F1000182F06881D7E90001E8
S3150802C2E0A0F58044214301F06480D7E9000144F2B5
S3150802C2F00104A04271F1000182F05881D7E90001D8
S3150802C300A0F50054214301F01180D7E9000142F259
S3150802C3100104A04271F1000182F04881D7E90001C7
S3150802C320A0F58054214300F01E87D7E9000141F2A7
S3150802C3300104A04271F1000182F03881D7E90001B7
S3150802C340A0F50064214300F0A886D7E9000140F66B
S3150802C3500104A04271F1000182F02881D7E90001A7
S3150802C360A0F58064214300F03286D7E9000140F245
S3150802C3700144A04271F1000182F01881D7E9000157
S3150802C380A0F50074214300F0B085D7E9000140F218
S3150802C3900124A04271F1000182F00881D7E9000167
S3150802C3A0A0F58074214300F03585D7E9000140F2F3
S3150802C3B00114A04271F1000182F0F880D7E9000168
S3150802C3C0A0F18004214300F0BA84D7E9000181284C
S3150802C3D071F1000182F0EA80D7E90001212871F1A2
S3150802C3E000016FD2D7E90001014302F0DF80D7E9E5
S3150802C3F00001421E41F1FF33202A73F1000182F047
S3150802C400D5801F2A02F2D28001A151F822F000BF7C
S3150802C41071C702083DC80208ADE50208FDC8020850
S3150802C420ADE50208ADE50208ADE50208CDC9020888
S3150802C430ADE50208ADE50208ADE50208ADE502087C
S3150802C440ADE50208ADE50208ADE50208AFCA020885
S3150802C450ADE50208ADE50208ADE50208ADE502085C
S3150802C460ADE50208ADE50208ADE50208ADE502084C
S3150802C470ADE50208ADE50208ADE50208ADE502083C
S3150802C480ADE50208ADE50208ADE5020885CB02086E
S3150802C4900100008001000040010000200100001098
S3150802C4A001000008010000040100800001004000AC
S3150802C4B0010020000100100001000800010004002C
S3150802C4C001000200D7E90023A2F140010B4300F064
S3150802C4D0C48302F06BB8A14BD3F8E83003F4E02327
S3150802C4E03B633B6BB3F5802F36D03B6BB3F5802F9E
S3150802C4F06BD83B6BB3F5403F2BD03B6BB3F5403F54
S3150802C50063D83B6BB3F5003F1BD03B6BB3F5003FDB
S3150802C5105BD83B6B002B04D03B6BB3F5803F08D04E
S3150802C52053E007F120031846FFF7BAF87B6A7B63E4
S3150802C5304EE007F114031846FFF71CFA7B697B6382
S3150802C54046E007F108031846FFF77EFBBB687B63E4
S3150802C5503EE0834B7B633BE0804BD3F8E83003F045
S3150802C5604043FB627D4B1B6803F00203022B0CD18E
S3150802C570FB6A002B09D1794B1B68DB0803F003031E
S3150802C580784A22FA03F37B631EE0744B1B6803F4B2
S3150802C5900073B3F5007F06D1FB6AB3F1804F02D16F
S3150802C5A0714B7B6310E06D4B1B6803F40033B3F5E4
S3150802C5B0003F06D1FB6AB3F1004F02D16B4B7B6396
S3150802C5C002E000237B6303E002E000237B6300BFF3
S3150802C5D001F0EFBF614BD3F8E83003F460133B6315
S3150802C5E03B6BB3F5001F36D03B6BB3F5001F6BD818
S3150802C5F03B6BB3F5C01F2BD03B6BB3F5C01F63D89B
S3150802C6003B6BB3F5801F1BD03B6BB3F5801F5BD822
S3150802C6103B6B002B04D03B6BB3F5002F08D053E0DD
S3150802C62007F120031846FFF73BF87B6A7B634EE067
S3150802C63007F114031846FFF79DF97B697B6346E009
S3150802C64007F108031846FFF7FFFABB687B633EE06B
S3150802C650434B7B633BE0414BD3F8E83003F040435E
S3150802C660FB623E4B1B6803F00203022B0CD1FB6AEA
S3150802C670002B09D1394B1B68DB0803F00303394A3F
S3150802C68022FA03F37B631EE0344B1B6803F4007340
S3150802C690B3F5007F06D1FB6AB3F1804F02D1324B64
S3150802C6A07B6310E02D4B1B6803F40033B3F5003FA0
S3150802C6B006D1FB6AB3F1004F02D12C4B7B6302E031
S3150802C6C000237B6303E002E000237B6300BF01F0E3
S3150802C6D070BF224BD3F8E43003F040033B633B6B55
S3150802C6E0002B08D107F120031846FEF7D9FF7B6A0B
S3150802C6F07B6301F05EBF3B6B402B08D107F1140345
S3150802C7001846FFF737F9FB697B6301F052BF00232E
S3150802C7107B6301F04EBF114BD3F8E43003F080037C
S3150802C7203B633B6B002B08D107F120031846FEF743
S3150802C730B7FF7B6A7B6301F03CBF3B6B802B08D15A
S3150802C74007F114031846FFF715F9FB697B6301F035
S3150802C75030BF00237B6301F02CBF00BF000C0244EC
S3150802C7600080BB000090D00300093D00001BB70003
S3150802C7709D4BD3F8D83003F007033B633B6B002B82
S3150802C78004D1FCF79FFF786301F013BF964B1B6831
S3150802C79003F00063B3F1006F0AD13B6B012B07D19B
S3150802C7A007F114031846FFF7E5F8BB697B6343E014
S3150802C7B08D4B1B6803F00053B3F1005F0AD13B6B44
S3150802C7C0022B07D107F108031846FFF73DFAFB6863
S3150802C7D07B6331E0844B1B6803F00203022B0CD106
S3150802C7E03B6B032B09D1804B1B68DB0803F0030361
S3150802C7F07E4A22FA03F37B631EE07B4B1B6803F433
S3150802C8000073B3F5007F05D13B6B042B02D1784B3D
S3150802C8107B6311E0744BD3F8F03003F00203022B6A
S3150802C82006D13B6B052B03D14FF400437B6303E030
S3150802C83000237B6301F0BDBE01F0BBBE6A4BD3F891
S3150802C840D83003F038033B633B6B002B04D1FCF76B
S3150802C85023FF786301F0ADBE634B1B6803F00063E8
S3150802C860B3F1006F0AD13B6B082B07D107F114030A
S3150802C8701846FFF77FF8BB697B633DE03B6B102BDD
S3150802C88008D107F108031846FFF7DEF9FB687B6350
S3150802C89001F08FBE544B1B6803F00203022B0CD126
S3150802C8A03B6B182B09D1504B1B68DB0803F00303BB
S3150802C8B04E4A22FA03F37B631EE04B4B1B6803F4D2
S3150802C8C00073B3F5007F05D13B6B202B02D1484B91
S3150802C8D07B6311E0444BD3F8F03003F00203022BDA
S3150802C8E006D13B6B282B03D14FF400437B6303E04D
S3150802C8F000237B6301F05DBE01F05BBE3A4BD3F8C1
S3150802C900D83003F4E0733B633B6B002B04D1FCF78E
S3150802C910C3FE786301F04DBE334B1B6803F0006318
S3150802C920B3F1006F0AD13B6B402B07D107F1140311
S3150802C9301846FFF71FF8BB697B6345E02A4B1B685D
S3150802C94003F00053B3F1005F0AD13B6B802B07D18A
S3150802C95007F108031846FFF777F9FB687B6333E0AC
S3150802C960214B1B6803F00203022B0CD13B6BC02B35
S3150802C97009D11D4B1B68DB0803F003031B4A22FA85
S3150802C98003F37B6320E0184B1B6803F40073B3F5CB
S3150802C990007F06D13B6BB3F5807F02D1144B7B63D4
S3150802C9A012E0114BD3F8F03003F00203022B07D141
S3150802C9B03B6BB3F5A07F03D14FF400437B6303E0DF
S3150802C9C000237B6301F0F5BD01F0F3BD064BD3F8F6
S3150802C9D0D83003F460633B633B6B002B0AD1FCF748
S3150802C9E05BFE786301F0E5BD000C02440090D003BB
S3150802C9F000093D00A04B1B6803F00063B3F1006F0A
S3150802CA000BD13B6BB3F5007F07D107F11403184628
S3150802CA10FEF7B0FFBB697B6347E0974B1B6803F0E1
S3150802CA200053B3F1005F0BD13B6BB3F5806F07D1AF
S3150802CA3007F108031846FFF707F9FB687B6334E03A
S3150802CA408D4B1B6803F00203022B0DD13B6BB3F52A
S3150802CA50C06F09D1884B1B68DB0803F00303874ABA
S3150802CA6022FA03F37B6320E0834B1B6803F400730B
S3150802CA70B3F5007F06D13B6BB3F5006F02D1804B4D
S3150802CA807B6312E07C4BD3F8F03003F00203022BEF
S3150802CA9007D13B6BB3F5206F03D14FF400437B6399
S3150802CAA003E000237B6301F084BD01F082BD724B73
S3150802CAB0D3F8D83003F4E0433B633B6B002B04D135
S3150802CAC0FCF7EAFD786301F074BD6B4B1B6803F053
S3150802CAD00063B3F1006F0BD13B6BB3F5805F07D1EF
S3150802CAE007F114031846FEF745FFBB697B6347E067
S3150802CAF0614B1B6803F00053B3F1005F0BD13B6B2C
S3150802CB00B3F5005F07D107F108031846FFF79CF84B
S3150802CB10FB687B6334E0584B1B6803F00203022B65
S3150802CB200DD13B6BB3F5405F09D1534B1B68DB084C
S3150802CB3003F00303514A22FA03F37B6320E04E4BC8
S3150802CB401B6803F40073B3F5007F06D13B6BB3F59C
S3150802CB50804F02D14A4B7B6312E0474BD3F8F03041
S3150802CB6003F00203022B07D13B6BB3F5A04F03D1A7
S3150802CB704FF400437B6303E000237B6301F019BD96
S3150802CB8001F017BD3C4BD3F8D83003F460333B634E
S3150802CB903B6B002B04D1FCF77FFD786301F009BDDE
S3150802CBA0354B1B6803F00063B3F1006F0BD13B6B87
S3150802CBB0B3F5004F07D107F114031846FEF7DAFE5C
S3150802CBC0BB697B6347E02C4B1B6803F00053B3F148
S3150802CBD0005F0BD13B6BB3F5803F07D107F1080322
S3150802CBE01846FFF731F8FB687B6334E0224B1B6873
S3150802CBF003F00203022B0DD13B6BB3F5C03F09D1FB
S3150802CC001D4B1B68DB0803F003031C4A22FA03F3D5
S3150802CC107B6320E0184B1B6803F40073B3F5007FAF
S3150802CC2006D13B6BB3F5003F02D1154B7B6312E08D
S3150802CC30114BD3F8F03003F00203022B07D13B6BFA
S3150802CC40B3F5203F03D14FF400437B6303E000238F
S3150802CC507B6301F0AEBC01F0ACBC074BD3F8D8300D
S3150802CC6003F4E0133B633B6B002B0BD1FCF714FD7B
S3150802CC70786301F09EBC00BF000C02440090D0030A
S3150802CC8000093D00A04B1B6803F00063B3F1006F77
S3150802CC900BD13B6BB3F5802F07D107F11403184666
S3150802CCA0FEF768FEBB697B6347E0974B1B6803F098
S3150802CCB00053B3F1005F0BD13B6BB3F5002F07D1DD
S3150802CCC007F108031846FEF7BFFFFB687B6334E0EB
S3150802CCD08D4B1B6803F00203022B0DD13B6BB3F598
S3150802CCE0402F09D1884B1B68DB0803F00303874AE8
S3150802CCF022FA03F37B6320E0834B1B6803F4007379
S3150802CD00B3F5007F06D13B6BB3F5801F02D1804B8A
S3150802CD107B6312E07C4BD3F8F03003F00203022B5C
S3150802CD2007D13B6BB3F5A01F03D14FF400437B63D6
S3150802CD3003E000237B6301F03CBC01F03ABC724B72
S3150802CD40D3F8D83003F460033B633B6B002B04D162
S3150802CD50FCF7A2FC786301F02CBC6B4B1B6803F052
S3150802CD600063B3F1006F0BD13B6BB3F5001F07D11C
S3150802CD7007F114031846FEF7FDFDBB697B6347E01E
S3150802CD80614B1B6803F00053B3F1005F0BD13B6B99
S3150802CD90B3F5800F07D107F108031846FEF754FFCB
S3150802CDA0FB687B6334E0584B1B6803F00203022BD3
S3150802CDB00DD13B6BB3F5C00F09D1534B1B68DB088A
S3150802CDC003F00303514A22FA03F37B6320E04E4B36
S3150802CDD01B6803F40073B3F5007F06D13B6BB3F50A
S3150802CDE0000F02D14A4B7B6312E0474BD3F8F0306F
S3150802CDF003F00203022B07D13B6BB3F5200F03D1D5
S3150802CE004FF400437B6303E000237B6301F0D1BB4D
S3150802CE1001F0CFBB3C4BD3F8D83003F0E0633B6359
S3150802CE203B6B002B04D1FCF737FC786301F0C1BBDE
S3150802CE30354B1B6803F00063B3F1006F0BD13B6BF4
S3150802CE40B3F1807F07D107F114031846FEF792FD66
S3150802CE50BB697B6347E02C4B1B6803F00053B3F1B5
S3150802CE60005F0BD13B6BB3F1007F07D107F10803D3
S3150802CE701846FEF7E9FEFB687B6334E0224B1B6823
S3150802CE8003F00203022B0DD13B6BB3F1407F09D1AC
S3150802CE901D4B1B68DB0803F003031C4A22FA03F343
S3150802CEA07B6320E0184B1B6803F40073B3F5007F1D
S3150802CEB006D13B6BB3F1806F02D1154B7B6312E04F
S3150802CEC0114BD3F8F03003F00203022B07D13B6B68
S3150802CED0B3F1A06F03D14FF400437B6303E0002351
S3150802CEE07B6301F066BB01F064BB074BD3F8D8300D
S3150802CEF003F060533B633B6B002B0BD1FCF7CCFB77
S3150802CF00786301F056BB00BF000C02440090D003C0
S3150802CF1000093D00A14B1B6803F00063B3F1006FE3
S3150802CF200BD13B6BB3F1006F07D107F11403184617
S3150802CF30FEF720FDBB697B6347E0984B1B6803F04D
S3150802CF400053B3F1005F0BD13B6BB3F1805F07D19E
S3150802CF5007F108031846FEF777FEFB687B6334E0A1
S3150802CF608E4B1B6803F00203022B0DD13B6BB3F108
S3150802CF70C05F09D1894B1B68DB0803F00303884AA3
S3150802CF8022FA03F37B6320E0844B1B6803F40073E5
S3150802CF90B3F5007F06D13B6BB3F1005F02D1814B3B
S3150802CFA07B6312E07D4BD3F8F03003F00203022BC9
S3150802CFB007D13B6BB3F1205F03D14FF400437B6388
S3150802CFC003E000237B6301F0F4BA01F0F2BA734B73
S3150802CFD0D3F8DC3003F007033B633B6B002B04D129
S3150802CFE0FCF75AFB786301F0E4BA6C4B1B6803F052
S3150802CFF00063B3F1006F0AD13B6B012B07D107F12E
S3150802D00014031846FEF7B6FCBB697B6343E0634B21
S3150802D0101B6803F00053B3F1005F0AD13B6B022B86
S3150802D02007D107F108031846FEF70EFEFB687B6375
S3150802D03031E05A4B1B6803F00203022B0CD13B6BFF
S3150802D040032B09D1554B1B68DB0803F00303544A2B
S3150802D05022FA03F37B631EE0504B1B6803F400734A
S3150802D060B3F5007F05D13B6B042B02D14D4B7B6395
S3150802D07011E04A4BD3F8F03003F00203022B06D133
S3150802D0803B6B052B03D14FF400437B6303E000237C
S3150802D0907B6301F08EBA01F08CBA404BD3F8DC30D0
S3150802D0A003F070033B633B6B002B04D1FCF7F4FAE5
S3150802D0B0786301F07EBA394B1B6803F00063B3F15B
S3150802D0C0006F0AD13B6B102B07D107F114031846E0
S3150802D0D0FEF750FCBB697B6343E0304B1B6803F0E9
S3150802D0E00053B3F1005F0AD13B6B202B07D107F13E
S3150802D0F008031846FEF7A8FDFB687B6331E0274B59
S3150802D1001B6803F00203022B0CD13B6B302B09D1AF
S3150802D110224B1B68DB0803F00303214A22FA03F3B6
S3150802D1207B631EE01D4B1B6803F40073B3F5007F97
S3150802D13005D13B6B402B02D11A4B7B6311E0174B8F
S3150802D140D3F8F03003F00203022B06D13B6B502BC7
S3150802D15003D14FF400437B6303E000237B6301F0B2
S3150802D16028BA01F026BA0D4BD3F8E03003F0E06393
S3150802D1703B633B6B002B04D1FCF7BAFA786301F0E8
S3150802D18018BA3B6BB3F1807F0ED107F11403184628
S3150802D190FEF7F0FBBB697B6301F00BBA000C024495
S3150802D1A00090D00300093D003B6BB3F1007F08D124
S3150802D1B007F108031846FEF747FDFB687B6301F093
S3150802D1C0F8B9A44B1B6803F00203022B0DD13B6B83
S3150802D1D0B3F1407F09D19F4B1B68DB0803F00303B9
S3150802D1E09D4A22FA03F37B6320E09A4B1B6803F4F9
S3150802D1F00073B3F5007F06D13B6BB3F1806F02D1A2
S3150802D200964B7B6312E0934BD3F8F03003F002039C
S3150802D210022B07D13B6BB3F1A06F03D14FF4004346
S3150802D2207B6303E000237B6301F0C3B901F0C1B954
S3150802D230884BD3F8E83003F007033B633B6B002BBC
S3150802D24004D1FCF70DFA786301F0B3B93B6B012BF5
S3150802D25004D1FCF7D9F8786301F0ABB93B6B022B22
S3150802D26008D107F114031846FEF784FBFB697B63B2
S3150802D27001F09FB9774B1B6803F40033B3F5003FFF
S3150802D28005D13B6B032B02D1754B7B6323E0714BB4
S3150802D2901B6803F00203022B0CD13B6B042B09D14A
S3150802D2A06C4B1B68DB0803F003036B4A22FA03F391
S3150802D2B07B6310E0674B1B6803F40073B3F5007FCA
S3150802D2C005D13B6B052B02D1644B7B6303E000233C
S3150802D2D07B6301F06EB901F06CB95E4BD3F8E830A6
S3150802D2E003F008033B635B4BD3F8F03003F0020309
S3150802D2F0022B06D13B6B002B03D14FF400437B6311
S3150802D30012E0544BD3F8F03003F00063B3F1006F28
S3150802D31006D13B6B082B03D14FF4FA437B6303E038
S3150802D32000237B6301F045B901F043B9494BD3F8B1
S3150802D330E43003F440333B633B6B002B04D1FCF728
S3150802D340ABF9786301F035B93B6BB3F5803F08D189
S3150802D35007F108031846FEF777FC3B697B6301F081
S3150802D36028B93C4B1B6803F00203022B0DD13B6B19
S3150802D370B3F5003F09D1374B1B68DB0803F00303FB
S3150802D380354A22FA03F37B6311E0324B1B6803F436
S3150802D3900073B3F5007F06D13B6BB3F5403F02D16C
S3150802D3A02E4B7B6303E000237B6301F002B901F095
S3150802D3B000B9284BD3F8E43003F440233B633B6BB4
S3150802D3C0002B04D1FCF768F9786301F0F2B83B6BDD
S3150802D3D0B3F5802F08D107F108031846FEF734FC87
S3150802D3E03B697B6301F0E5B81A4B1B6803F002033D
S3150802D3F0022B0DD13B6BB3F5002F09D1154B1B68D8
S3150802D400DB0803F00303144A22FA03F37B6311E0F1
S3150802D410104B1B6803F40073B3F5007F06D13B6B10
S3150802D420B3F5402F02D10D4B7B6303E000237B63E8
S3150802D43001F0BFB801F0BDB8064BD3F8E43003F4E7
S3150802D44040133B633B6B002B0CD1FCF751F9786315
S3150802D45001F0AFB8000C02440090D00300093D0069
S3150802D460001BB7003B6BB3F5801F08D107F1080311
S3150802D4701846FEF7E9FB3B697B6301F09AB89F4BB6
S3150802D4801B6803F00203022B0DD13B6BB3F5001F99
S3150802D49009D19A4B1B68DB0803F00303984A22FA60
S3150802D4A003F37B6311E0954B1B6803F40073B3F532
S3150802D4B0007F06D13B6BB3F5401F02D1914B7B63CC
S3150802D4C003E000237B6301F074B801F072B88B4B5A
S3150802D4D0D3F8E43003F440033B633B6B002B04D1DF
S3150802D4E0FCF706F9786301F064B83B6BB3F5800F75
S3150802D4F008D107F108031846FEF7A6FB3B697B63CA
S3150802D50001F057B87D4B1B6803F00203022B0DD1BD
S3150802D5103B6BB3F5000F09D1784B1B68DB0803F0A8
S3150802D5200303774A22FA03F37B6311E0734B1B6802
S3150802D53003F40073B3F5007F06D13B6BB3F5400FD6
S3150802D54002D1704B7B6303E000237B6301F031B8A1
S3150802D55001F02FB8694BD3F8E43003F040733B630C
S3150802D5603B6B002B04D1FCF797F8786301F021B8DE
S3150802D5703B6BB3F1807F08D107F108031846FEF723
S3150802D58063FB3B697B6301F014B85C4B1B6803F0D1
S3150802D5900203022B0ED13B6BB3F1007F0AD1574B24
S3150802D5A01B68DB0803F00303554A22FA03F37B637D
S3150802D5B000F0FFBF00237B6300F0FBBF4F4BD3F89D
S3150802D5C0DC3003F4E0633B633B6BB3F5A06F56D0E4
S3150802D5D03B6BB3F5A06F00F28B803B6BB3F5806FA4
S3150802D5E03ED03B6BB3F5806F00F282803B6BB3F59E
S3150802D5F0407F27D03B6BB3F5407F79D83B6BB3F5B9
S3150802D600007F17D03B6BB3F5007F71D83B6B002BBD
S3150802D61004D03B6BB3F5807F04D069E0FCF768F869
S3150802D620786368E007F114031846FEF7A3F97B69E5
S3150802D6307B6360E007F108031846FEF705FB3B69C2
S3150802D6407B6358E02D4BD3F8F03003F00203022B2C
S3150802D65003D14FF400437B634DE000237B634AE02A
S3150802D660264BD3F8F03003F00063B3F1006F03D111
S3150802D6704FF4FA437B633EE000237B633BE01F4B98
S3150802D680D3F8E83003F04043FB621C4B1B6803F0F7
S3150802D6900203022B0CD1FB6A002B09D1174B1B681C
S3150802D6A0DB0803F00303164A22FA03F37B631EE040
S3150802D6B0124B1B6803F40073B3F5007F06D1FB6AAD
S3150802D6C0B3F1804F02D10F4B7B6310E00B4B1B6803
S3150802D6D003F40033B3F5003F06D1FB6AB3F1004FFA
S3150802D6E002D1094B7B6302E000237B6303E002E07D
S3150802D6F000237B6300BF00F05CBF00BF000C02443E
S3150802D7000090D00300093D00001BB7009E4BD3F8DA
S3150802D710DC3003F4E0433B633B6BB3F5A04F56D0D2
S3150802D7203B6BB3F5A04F00F28B803B6BB3F5804F92
S3150802D7303ED03B6BB3F5804F00F282803B6BB3F56C
S3150802D740405F27D03B6BB3F5405F79D83B6BB3F5A7
S3150802D750005F17D03B6BB3F5005F71D83B6B002BAC
S3150802D76004D03B6BB3F5805F04D069E0FBF794FF06
S3150802D770786368E007F114031846FEF7FBF87B693D
S3150802D7807B6360E007F108031846FEF75DFA3B691A
S3150802D7907B6358E07C4BD3F8F03003F00203022B8C
S3150802D7A003D14FF400437B634DE000237B634AE0D9
S3150802D7B0754BD3F8F03003F00063B3F1006F03D171
S3150802D7C04FF4FA437B633EE000237B633BE06E4BF8
S3150802D7D0D3F8E83003F04043FB626B4B1B6803F057
S3150802D7E00203022B0CD1FB6A002B09D1664B1B687C
S3150802D7F0DB0803F00303654A22FA03F37B631EE0A0
S3150802D800614B1B6803F40073B3F5007F06D1FB6A0C
S3150802D810B3F1804F02D15E4B7B6310E05A4B1B6813
S3150802D82003F40033B3F5003F06D1FB6AB3F1004FA8
S3150802D83002D1584B7B6302E000237B6303E002E0DC
S3150802D84000237B6300BF00F0B4BE4F4BD3F8DC3035
S3150802D85003F4E0233B633B6BB3F5A02F56D03B6B37
S3150802D860B3F5A02F00F28B803B6BB3F5802F3ED029
S3150802D8703B6BB3F5802F00F282803B6BB3F5403FDA
S3150802D88027D03B6BB3F5403F79D83B6BB3F5003FE6
S3150802D89017D03B6BB3F5003F71D83B6B002B04D016
S3150802D8A03B6BB3F5803F04D069E0FBF721FF786351
S3150802D8B068E007F114031846FEF75CF87B697B6398
S3150802D8C060E007F108031846FEF7BEF93B697B6379
S3150802D8D058E02D4BD3F8F03003F00203022B03D1A4
S3150802D8E04FF400437B634DE000237B634AE0264BFB
S3150802D8F0D3F8F03003F00063B3F1006F03D14FF4AD
S3150802D900FA437B633EE000237B633BE01E4BD3F87E
S3150802D910E83003F04043FB621B4B1B6803F002032B
S3150802D920022B0CD1FB6A002B09D1174B1B68DB08AB
S3150802D93003F00303154A22FA03F37B631EE0124B34
S3150802D9401B6803F40073B3F5007F06D1FB6AB3F1D3
S3150802D950804F02D10E4B7B6310E00B4B1B6803F41E
S3150802D9600033B3F5003F06D1FB6AB3F1004F02D18B
S3150802D970084B7B6302E000237B6303E002E000239B
S3150802D9807B6300BF00F015BE000C02440090D00372
S3150802D99000093D00001BB7009E4BD3F8DC3003F4A8
S3150802D9A0E0033B633B6BB3F5A00F56D03B6BB3F575
S3150802D9B0A00F00F28B803B6BB3F5800F3ED03B6B1A
S3150802D9C0B3F5800F00F282803B6BB3F5401F27D078
S3150802D9D03B6BB3F5401F79D83B6BB3F5001F17D0E5
S3150802D9E03B6BB3F5001F71D83B6B002B04D03B6B26
S3150802D9F0B3F5801F04D069E0FBF77AFE786368E026
S3150802DA0007F114031846FDF7B5FF7B697B6360E0EF
S3150802DA1007F108031846FEF717F93B697B6358E0D6
S3150802DA207C4BD3F8F03003F00203022B03D14FF4F8
S3150802DA3000437B634DE000237B634AE0754BD3F8D2
S3150802DA40F03003F00063B3F1006F03D14FF4FA43E9
S3150802DA507B633EE000237B633BE06E4BD3F8E83002
S3150802DA6003F04043FB626B4B1B6803F00203022B75
S3150802DA700CD1FB6A002B09D1664B1B68DB0803F045
S3150802DA800303654A22FA03F37B631EE0614B1B68B4
S3150802DA9003F40073B3F5007F06D1FB6AB3F1804F36
S3150802DAA002D15E4B7B6310E05A4B1B6803F40033CA
S3150802DAB0B3F5003F06D1FB6AB3F1004F02D1584BCA
S3150802DAC07B6302E000237B6303E002E000237B63BF
S3150802DAD000BF00F06EBD4F4BD3F8DC3003F0E063B5
S3150802DAE03B633B6BB3F1A06F56D03B6BB3F1A06FB0
S3150802DAF000F28B803B6BB3F1806F3ED03B6BB3F188
S3150802DB00806F00F282803B6BB3F1407F27D03B6B7C
S3150802DB10B3F1407F79D83B6BB3F1007F17D03B6BEB
S3150802DB20B3F1007F71D83B6B002B04D03B6BB3F18A
S3150802DB30807F04D069E0FBF7DBFD786368E007F1D4
S3150802DB4014031846FDF716FF7B697B6360E007F14D
S3150802DB5008031846FEF778F83B697B6358E02D4BB5
S3150802DB60D3F8F03003F00203022B03D14FF400433B
S3150802DB707B634DE000237B634AE0264BD3F8F03003
S3150802DB8003F00063B3F1006F03D14FF4FA437B63EA
S3150802DB903EE000237B633BE01E4BD3F8E83003F0FC
S3150802DBA04043FB621B4B1B6803F00203022B0CD19A
S3150802DBB0FB6A002B09D1174B1B68DB0803F003032A
S3150802DBC0154A22FA03F37B631EE0124B1B6803F421
S3150802DBD00073B3F5007F06D1FB6AB3F1804F02D119
S3150802DBE00E4B7B6310E00B4B1B6803F40033B3F553
S3150802DBF0003F06D1FB6AB3F1004F02D1084B7B63A3
S3150802DC0002E000237B6303E002E000237B6300BF9C
S3150802DC1000F0CFBC000C02440090D00300093D007E
S3150802DC20001BB7009E4BD3F8DC3003F0E0433B639E
S3150802DC303B6BB3F1A04F56D03B6BB3F1A04F00F24A
S3150802DC408B803B6BB3F1804F3ED03B6BB3F1804F79
S3150802DC5000F282803B6BB3F1405F27D03B6BB3F196
S3150802DC60405F79D83B6BB3F1005F17D03B6BB3F1DA
S3150802DC70005F71D83B6B002B04D03B6BB3F1805F1E
S3150802DC8004D069E0FBF734FD786368E007F1140312
S3150802DC901846FDF76FFE7B697B6360E007F10803B0
S3150802DCA01846FDF7D1FF3B697B6358E07C4BD3F8F6
S3150802DCB0F03003F00203022B03D14FF400437B63D7
S3150802DCC04DE000237B634AE0754BD3F8F03003F04E
S3150802DCD00063B3F1006F03D14FF4FA437B633EE06E
S3150802DCE000237B633BE06E4BD3F8E83003F04043F6
S3150802DCF0FB626B4B1B6803F00203022B0CD1FB6A17
S3150802DD00002B09D1664B1B68DB0803F00303654A3F
S3150802DD1022FA03F37B631EE0614B1B6803F400736C
S3150802DD20B3F5007F06D1FB6AB3F1804F02D15E4B91
S3150802DD307B6310E05A4B1B6803F40033B3F5003FCC
S3150802DD4006D1FB6AB3F1004F02D1584B7B6302E05E
S3150802DD5000237B6303E002E000237B6300BF00F03D
S3150802DD6028BC4F4BD3F8E83003F440733B634C4B63
S3150802DD701B6803F40033B3F5003F06D13B6B002B57
S3150802DD8003D14A4B7B6300F014BC3B6BB3F5807F2F
S3150802DD9008D107F120031846FDF782FC7B6A7B63EC
S3150802DDA000F007BC3B6BB3F5007F07D107F11403FC
S3150802DDB01846FDF7DFFDBB697B63FAE300237B6345
S3150802DDC0F7E3374BD3F8E03003F007033B633B6BCB
S3150802DDD0042B61D801A252F823F000BFF1DD020834
S3150802DDE001DE020811DE020821DE020827DE020829
S3150802DDF007F120031846FDF753FC7B6A7B634EE066
S3150802DE0007F114031846FDF7B5FD7B697B6346E007
S3150802DE1007F108031846FDF717FFBB687B633EE068
S3150802DE20234B7B633BE01E4BD3F8E83003F04043B9
S3150802DE30FB621B4B1B6803F00203022B0CD1FB6A25
S3150802DE40002B09D1164B1B68DB0803F00303154A9E
S3150802DE5022FA03F37B631EE0114B1B6803F400737B
S3150802DE60B3F5007F06D1FB6AB3F1804F02D10E4BA0
S3150802DE707B6310E00A4B1B6803F40033B3F5003FDB
S3150802DE8006D1FB6AB3F1004F02D1084B7B6302E06D
S3150802DE9000237B6303E002E000237B6300BF88E381
S3150802DEA0000C02440090D00300093D00001BB70095
S3150802DEB00080BB00A94BD3F8E03003F038033B637C
S3150802DEC03B6B202B00F29A8001A252F823F000BF86
S3150802DED055DF0208FDDF0208FDDF0208FDDF020842
S3150802DEE0FDDF0208FDDF0208FDDF0208FDDF02088A
S3150802DEF065DF0208FDDF0208FDDF0208FDDF020812
S3150802DF00FDDF0208FDDF0208FDDF0208FDDF020869
S3150802DF1075DF0208FDDF0208FDDF0208FDDF0208E1
S3150802DF20FDDF0208FDDF0208FDDF0208FDDF020849
S3150802DF3085DF0208FDDF0208FDDF0208FDDF0208B1
S3150802DF40FDDF0208FDDF0208FDDF0208FDDF020829
S3150802DF508BDF020807F120031846FDF7A1FB7B6A4F
S3150802DF607B634EE007F114031846FDF703FD7B6950
S3150802DF707B6346E007F108031846FDF765FEBB68B2
S3150802DF807B633EE0764B7B633BE0744BD3F8E83029
S3150802DF9003F04043FB62714B1B6803F00203022B3A
S3150802DFA00CD1FB6A002B09D16C4B1B68DB0803F00A
S3150802DFB003036C4A22FA03F37B631EE0674B1B6872
S3150802DFC003F40073B3F5007F06D1FB6AB3F1804F01
S3150802DFD002D1654B7B6310E0604B1B6803F4003388
S3150802DFE0B3F5003F06D1FB6AB3F1004F02D15F4B8E
S3150802DFF07B6302E000237B6303E002E000237B638A
S3150802E00000BFD6E2554BD3F8E03003F4E0733B6326
S3150802E0103B6BB3F5807F31D03B6BB3F5807F66D817
S3150802E0203B6BC02B27D03B6BC02B60D83B6B802B3E
S3150802E03019D03B6B802B5AD83B6B002B03D03B6B1A
S3150802E040402B08D053E007F120031846FDF728FBBA
S3150802E0507B6A7B634EE007F114031846FDF78AFCD8
S3150802E0607B697B6346E007F108031846FDF7ECFD7A
S3150802E070BB687B633EE03A4B7B633BE0374BD3F8A6
S3150802E080E83003F04043FB62344B1B6803F002039B
S3150802E090022B0CD1FB6A002B09D1304B1B68DB081B
S3150802E0A003F003032F4A22FA03F37B631EE02B4B8A
S3150802E0B01B6803F40073B3F5007F06D1FB6AB3F15C
S3150802E0C0804F02D1284B7B6310E0244B1B6803F474
S3150802E0D00033B3F5003F06D1FB6AB3F1004F02D114
S3150802E0E0224B7B6302E000237B6303E002E000230A
S3150802E0F07B6300BF5DE2194BD3F8E03003F460633B
S3150802E1003B633B6B002B03D1FBF7DCFA786350E2E7
S3150802E110124B1B6803F00063B3F1006F0BD13B6B24
S3150802E120B3F5007F07D107F114031846FDF722FC61
S3150802E130BB697B634FE0094B1B6803F00053B3F1DD
S3150802E140005F15D13B6BB3F5806F11D107F1080358
S3150802E1501846FDF779FDFB687B633CE0000C024438
S3150802E1600080BB000090D00300093D00001BB700E9
S3150802E170944B1B6803F00203022B0DD13B6BB3F5DC
S3150802E180C06F09D18F4B1B68DB0803F003038E4A65
S3150802E19022FA03F37B631EE08A4B1B6803F40073BF
S3150802E1A0B3F5007F06D13B6BB3F5006F02D1874BFF
S3150802E1B07B6310E0834B1B6803F40033B3F5003F1F
S3150802E1C006D13B6BB3F5206F02D1814B7B6302E02C
S3150802E1D000237B63EDE1ECE17A4BD3F8E03003F4FC
S3150802E1E0E0433B633B6B002B03D1FBF781FA786371
S3150802E1F0DFE1744B1B6803F00063B3F1006F0BD1C8
S3150802E2003B6BB3F5805F07D107F114031846FDF798
S3150802E210B1FBBB697B6345E06A4B1B6803F000539D
S3150802E220B3F1005F0BD13B6BB3F5005F07D107F182
S3150802E23008031846FDF708FDFB687B6332E0614B6D
S3150802E2401B6803F00203022B0DD13B6BB3F5405F4B
S3150802E25009D15C4B1B68DB0803F003035A4A22FA0E
S3150802E26003F37B631EE0574B1B6803F40073B3F595
S3150802E270007F06D13B6BB3F5804F02D1534B7B63CC
S3150802E28010E0504B1B6803F40033B3F5003F06D188
S3150802E2903B6BB3F5A04F02D14D4B7B6302E00023E3
S3150802E2A07B6386E185E1474BD3F8E03003F46033BC
S3150802E2B03B633B6B002B03D1FBF704FA786378E1E7
S3150802E2C0404B1B6803F00063B3F1006F0BD13B6B45
S3150802E2D0B3F5004F07D107F114031846FDF74AFBB9
S3150802E2E0BB697B6345E0374B1B6803F00053B3F108
S3150802E2F0005F0BD13B6BB3F5803F07D107F10803EB
S3150802E3001846FDF7A1FCFB687B6332E02D4B1B68C0
S3150802E31003F00203022B0DD13B6BB3F5C03F09D1C3
S3150802E320284B1B68DB0803F00303274A22FA03F388
S3150802E3307B631EE0234B1B6803F40073B3F5007F6F
S3150802E34006D13B6BB3F5003F02D1204B7B6310E04D
S3150802E3501C4B1B6803F40033B3F5003F06D13B6B35
S3150802E360B3F5203F02D11A4B7B6302E000237B639D
S3150802E3701FE11EE1134BD3F8E43003F003033B63BA
S3150802E3803B6B032B5FD801A252F823F09DE30208E8
S3150802E390A5E30208B5E30208D5E30208FBF760F92C
S3150802E3A0786353E007F120031846FDF779F97B6A8B
S3150802E3B07B634BE007F114031846FDF7DBFAFB69AA
S3150802E3C07B6343E0000C02440090D00300093D0041
S3150802E3D0001BB700794BD3F8E83003F04043FB62E1
S3150802E3E0764B1B6803F00203022B0CD1FB6A002B47
S3150802E3F009D1724B1B68DB0803F00303704A22FA41
S3150802E40003F37B631EE06D4B1B6803F40073B3F5DD
S3150802E410007F06D1FB6AB3F1804F02D1694B7B6359
S3150802E42010E0664B1B6803F40033B3F5003F06D1D0
S3150802E430FB6AB3F1004F02D1634B7B6302E0002310
S3150802E4407B6303E002E000237B6300BFB1E05B4B22
S3150802E450D3F8E83003F0C0033B63584BD3F8F030E7
S3150802E46003F00203022B06D13B6B002B03D14FF4B8
S3150802E47000437B631FE0514BD3F8F03003F000638F
S3150802E480B3F1006F06D13B6B402B03D14FF4FA432D
S3150802E4907B6310E0494B1B6803F40073B3F5007FF6
S3150802E4A006D13B6B802B03D148F212037B6302E051
S3150802E4B000237B637DE07CE0404BD3F8E83003F031
S3150802E4C030033B633D4B1B6803F40053B3F5005F0F
S3150802E4D005D13B6B002B02D13C4B7B6331E0374BBA
S3150802E4E01B6803F00073B3F1007F0AD13B6B102B54
S3150802E4F007D107F120031846FDF7D2F87B6A7B633A
S3150802E5001FE02E4BD3F8F03003F00203022B06D19C
S3150802E5103B6B202B03D14FF400437B6311E0274B5F
S3150802E520D3F8F03003F00063B3F1006F06D13B6B0A
S3150802E530302B03D14FF4FA437B6302E000237B635B
S3150802E54037E036E01D4BD3F8E43003F030033B6383
S3150802E5503B6B102B07D107F120031846FDF7A0F8ED
S3150802E5607B6A7B6325E0154B1B6803F00053B3F106
S3150802E570005F0AD13B6B202B07D107F10803184627
S3150802E580FDF762FBFB687B630FE00C4B1B6803F429
S3150802E5900053B3F5005F05D13B6B302B02D10B4B11
S3150802E5A07B6302E000237B6303E002E000237B63D4
S3150802E5B000BF7B6B18463C37BD4690BD000C024433
S3150802E5C00090D00300093D00001BB700006CDC0276
S3150802E5D080B584B000AF7860484B1B68474A23F081
S3150802E5E080631360F8F7D2FAF86008E0F8F7CEFA13
S3150802E5F00246FB68D31A022B01D903237AE03F4B62
S3150802E6001B6803F00063002BF0D13C4BDB6A23F452
S3150802E6107C5323F003037A6811687A6852681202F7
S3150802E6200A4336491343CB627B689B68013BC3F3B3
S3150802E63008027B68DB68013B5B029BB21A437B6874
S3150802E6401B69013B1B0403F4FE031A437B685B69DF
S3150802E650013B1B0603F0FE4328491343CB63274BB2
S3150802E660DB6A23F00C027B689B6924491343CB625D
S3150802E670224BDB6A23F020027B68DB691F491343BE
S3150802E680CB621E4BDA6A7B685B6A1C491343CB6210
S3150802E6901A4BDB6A194A23F01003D362174B1B6C19
S3150802E6A023F47F4323F0F8037A68126AD2001349E7
S3150802E6B013430B64114BDB6A104A43F01003D3620F
S3150802E6C00E4B1B680D4A43F080631360F8F75EFA37
S3150802E6D0F86008E0F8F75AFA0246FB68D31A022BE2
S3150802E6E001D9032306E0054B1B6803F00063002BE0
S3150802E6F0F0D0002318461037BD4680BD000C0244F0
S3150802E70080B584B000AF7860484B1B68474A23F04F
S3150802E71080531360F8F73AFAF86008E0F8F736FA21
S3150802E7200246FB68D31A022B01D903237AE03F4B30
S3150802E7301B6803F00053002BF0D13C4B1B6B23F4F0
S3150802E7407C5323F003037A6811687A6852681202C6
S3150802E7500A43364913430B637B689B68013BC3F341
S3150802E76008027B68DB68013B5B029BB21A437B6843
S3150802E7701B69013B1B0403F4FE031A437B685B69AE
S3150802E780013B1B0603F0FE43284913434B64274B00
S3150802E7901B6B23F00C027B689B69244913430B63AA
S3150802E7A0224B1B6B23F020027B68DB691F4913434C
S3150802E7B00B631E4B1A6B7B685B6A1C4913430B631C
S3150802E7C01A4B1B6B194A23F010031363174B9B6CE6
S3150802E7D023F47F4323F0F8037A68126AD2001349B6
S3150802E7E013438B64114B1B6B104A43F010031363DC
S3150802E7F00E4B1B680D4A43F080531360F8F7C6F9AF
S3150802E800F86008E0F8F7C2F90246FB68D31A022B49
S3150802E81001D9032306E0054B1B6803F00053002BBE
S3150802E820F0D0002318461037BD4680BD000C0244BE
S3150802E83080B582B000AF78607B68002B01D10123D6
S3150802E84049E07B6893F83D30DBB2002B06D17B6842
S3150802E850002283F83C207868F6F7C4FB7B6802221C
S3150802E86083F83D207B681A687B680433194610468C
S3150802E87000F074FB7B68012283F848207B6801223A
S3150802E88083F83E207B68012283F83F207B680122B9
S3150802E89083F840207B68012283F841207B680122A5
S3150802E8A083F842207B68012283F843207B68012291
S3150802E8B083F844207B68012283F845207B6801227D
S3150802E8C083F846207B68012283F847207B68012269
S3150802E8D083F83D20002318460837BD4680BD000050
S3150802E8E080B485B000AF78607B6893F83D30DBB2C0
S3150802E8F0012B01D001237CE07B68022283F83D20AC
S3150802E9007B681B68DA687B681B6842F00102DA607A
S3150802E9107B681B683A4A93424AD07B681B68394A25
S3150802E920934245D07B681B68B3F1804F40D07B6821
S3150802E9301B68B3F1A04F3BD07B681B68324A9342EF
S3150802E94036D07B681B68314A934231D07B681B6894
S3150802E9502F4A93422CD07B681B682E4A934227D0B3
S3150802E9607B681B682C4A934222D07B681B682B4A19
S3150802E97093421DD07B681B68294A934218D07B684C
S3150802E9801B68284A934213D07B681B68264A93421F
S3150802E9900ED07B681B68254A934209D07B681B68A0
S3150802E9A0234A934204D07B681B68224A934215D1B4
S3150802E9B07B681B689A68204B1340FB60FB68062B32
S3150802E9C015D0FB68B3F5803F11D07B681B681A68BF
S3150802E9D07B681B6842F001021A6008E07B681B68C4
S3150802E9E01A687B681B6842F001021A6000E000BFE1
S3150802E9F0002318461437BD465DF8047B704700BFEE
S3150802EA00002C0140002C0150000400400004005074
S3150802EA100008004000080050000C0040000C00509E
S3150802EA20003401400034015000180040001800501C
S3150802EA3000400140004001500700010080B584B043
S3150802EA4000AF78607B681B68DB68FB607B681B68C5
S3150802EA501B69BB60BB6803F00203002B20D0FB686E
S3150802EA6003F00203002B1BD07B681B686FF00202BF
S3150802EA701A617B6801221A777B681B689B6903F017
S3150802EA800303002B03D0786800F04AFA05E0786899
S3150802EA9000F03CFA786800F04DFA7B6800221A7793
S3150802EAA0BB6803F00403002B20D0FB6803F00403C1
S3150802EAB0002B1BD07B681B686FF004021A617B6807
S3150802EAC002221A777B681B689B6903F44073002B42
S3150802EAD003D0786800F024FA05E0786800F016FAA0
S3150802EAE0786800F027FA7B6800221A77BB6803F079
S3150802EAF00803002B20D0FB6803F00803002B1BD069
S3150802EB007B681B686FF008021A617B6804221A7711
S3150802EB107B681B68DB6903F00303002B03D0786864
S3150802EB2000F0FEF905E0786800F0F0F9786800F080
S3150802EB3001FA7B6800221A77BB6803F01003002BE0
S3150802EB4020D0FB6803F01003002B1BD07B681B68E0
S3150802EB506FF010021A617B6808221A777B681B68B5
S3150802EB60DB6903F44073002B03D0786800F0D8F908
S3150802EB7005E0786800F0CAF9786800F0DBF97B6886
S3150802EB8000221A77BB6803F00103002B0CD0FB683E
S3150802EB9003F00103002B07D07B681B686FF00102A4
S3150802EBA01A617868F5F7BAFFBB6803F08003002B91
S3150802EBB00CD0FB6803F08003002B07D07B681B6828
S3150802EBC06FF080021A61786800F05CFCBB6803F497
S3150802EBD08073002B0CD0FB6803F08003002B07D050
S3150802EBE07B681B686FF480721A61786800F054FCBF
S3150802EBF0BB6803F04003002B0CD0FB6803F040030C
S3150802EC00002B07D07B681B686FF040021A61786890
S3150802EC1000F09AF9BB6803F02003002B0CD0FB68BE
S3150802EC2003F02003002B07D07B681B686FF02002D5
S3150802EC301A61786800F01CFCBB6803F48013002B89
S3150802EC400CD0FB6803F48013002B07D07B681B6883
S3150802EC506FF480121A61786800F028FCBB6803F426
S3150802EC600013002B0CD0FB6803F40013002B07D00B
S3150802EC707B681B686FF400121A61786800F020FC42
S3150802EC80BB6803F48003002B0CD0FB6803F48003F3
S3150802EC90002B07D07B681B686FF480021A617868BC
S3150802ECA000F018FCBB6803F40003002B0CD0FB68C9
S3150802ECB003F40003002B07D07B681B686FF400027D
S3150802ECC01A61786800F010FC00BF1037BD4680BD97
S3150802ECD080B584B000AF786039600023FB737B6827
S3150802ECE093F83C30012B01D10223FEE07B68012216
S3150802ECF083F83C207B68022283F83D207B681B68E8
S3150802ED009B68BB60BB6823F4441323F07703BB609C
S3150802ED10BB6823F47F43BB607B681B68BA689A604A
S3150802ED203B681B68B3F5001F00F0C980B3F5001FE6
S3150802ED3000F2CE806F4A934200F0C1806D4A934238
S3150802ED4000F2C6806C4A934200F0B9806A4A93423E
S3150802ED5000F2BE80694A934200F0B180674A934244
S3150802ED6000F2B680664A934200F0A980644A93424A
S3150802ED7000F2AE80634A934200F0A180614A934250
S3150802ED8000F2A680604A934200F099805E4A934256
S3150802ED9000F29E80B3F1101F00F09180B3F1101FAC
S3150802EDA000F29680B3F5801F00F08980B3F5801FC4
S3150802EDB000F28E80B3F5005F3ED0B3F5005F00F235
S3150802EDC08780B3F5805F00F08680B3F5805F7FD8D1
S3150802EDD0702B1AD0702B7BD8602B50D0602B77D82B
S3150802EDE0502B3CD0502B73D8402B58D0402B6FD881
S3150802EDF0302B64D0302B6BD8202B60D0202B67D8D1
S3150802EE00002B5CD0102B5AD062E07B6818683B68EE
S3150802EE1099683B685A683B68DB6800F039FA7B6890
S3150802EE201B689B68BB60BB6843F07703BB607B6863
S3150802EE301B68BA689A604FE07B6818683B689968ED
S3150802EE403B685A683B68DB6800F022FA7B681B68F5
S3150802EE509A687B681B6842F480429A603CE07B6849
S3150802EE6018683B6859683B68DB681A4600F094F9EB
S3150802EE707B681B685021184600F0EDF92CE07B6888
S3150802EE8018683B6859683B68DB681A4600F0B3F9AC
S3150802EE907B681B686021184600F0DDF91CE07B6878
S3150802EEA018683B6859683B68DB681A4600F074F9CB
S3150802EEB07B681B684021184600F0CDF90CE07B6898
S3150802EEC01A683B681B681946104600F0C4F903E045
S3150802EED00123FB7300E000BF7B68012283F83D2013
S3150802EEE07B68002283F83C20FB7B18461037BD4618
S3150802EEF080BD00BF700010006000100050001000B6
S3150802EF0040001000300010002000100080B483B0CA
S3150802EF1000AF786000BF0C37BD465DF8047B7047CA
S3150802EF2080B483B000AF786000BF0C37BD465DF889
S3150802EF30047B704780B483B000AF786000BF0C379B
S3150802EF40BD465DF8047B704780B483B000AF786035
S3150802EF5000BF0C37BD465DF8047B704780B485B0A8
S3150802EF6000AF786039607B681B68FB607B68744A0F
S3150802EF7093422BD07B68734A934227D07B68B3F1BE
S3150802EF80804F23D07B68B3F1A04F1FD07B686E4AAF
S3150802EF9093421BD07B686D4A934217D07B686C4AB2
S3150802EFA0934213D07B686B4A93420FD07B686A4AB6
S3150802EFB093420BD07B68694A934207D07B68684ABA
S3150802EFC0934203D07B68674A934208D1FB6823F0D1
S3150802EFD07003FB603B685B68FA681343FB607B68F7
S3150802EFE0574A93425BD07B68564A934257D07B680E
S3150802EFF0B3F1804F53D07B68B3F1A04F4FD07B68F3
S3150802F000514A93424BD07B68504A934247D07B6819
S3150802F0104F4A934243D07B684E4A93423FD07B681D
S3150802F0204D4A93423BD07B684C4A934237D07B6821
S3150802F0304B4A934233D07B684A4A93422FD07B6825
S3150802F040494A93422BD07B68484A934227D07B6829
S3150802F050474A934223D07B68464A93421FD07B682D
S3150802F060454A93421BD07B68444A934217D07B6831
S3150802F070434A934213D07B68424A93420FD07B6835
S3150802F080414A93420BD07B68404A934207D07B6839
S3150802F0903F4A934203D07B683E4A934208D1FB68B3
S3150802F0A023F44073FB603B68DB68FA681343FB6032
S3150802F0B0FB6823F080023B685B691343FB607B684D
S3150802F0C0FA681A603B689A687B68DA623B681A686B
S3150802F0D07B689A627B681A4A934223D07B68194AEC
S3150802F0E093421FD07B681E4A93421BD07B681D4AF7
S3150802F0F0934217D07B68224A934213D07B68214AEF
S3150802F10093420FD07B68204A93420BD07B681F4AF2
S3150802F110934207D07B681E4A934203D07B681D4AF6
S3150802F120934203D13B681A697B681A637B6801229A
S3150802F1305A6100BF1437BD465DF8047B704700BFAD
S3150802F140002C0140002C015000040040000400502D
S3150802F1500008004000080050000C0040000C005057
S3150802F16000340140003401500018004000180050D5
S3150802F170001C0040001C00500020004000200050E7
S3150802F1800040014000400150004401400044015043
S3150802F190004801400048015080B487B000AFF860CB
S3150802F1A0B9607A60FB681B6A7B61FB681B6A23F09D
S3150802F1B00102FB681A62FB689B693B613B6923F0A3
S3150802F1C0F0033B617B681B013A6913433B617B6928
S3150802F1D023F00A037B617A69BB6813437B61FB6888
S3150802F1E03A699A61FB687A691A6200BF1C37BD469A
S3150802F1F05DF8047B704780B487B000AFF860B960E9
S3150802F2007A60FB681B6A7B61FB681B6A23F0100243
S3150802F210FB681A62FB689B693B613B6923F470438E
S3150802F2203B617B681B033A6913433B617B6923F0A5
S3150802F230A0037B61BB681B017A6913437B61FB6888
S3150802F2403A699A61FB687A691A6200BF1C37BD4639
S3150802F2505DF8047B704780B485B000AF786039608A
S3150802F2607B689B68FB60FB6823F4401323F07003FA
S3150802F270FB603A68FB68134343F00703FB607B684D
S3150802F280FA689A6000BF1437BD465DF8047B70477A
S3150802F29080B487B000AFF860B9607A603B60FB68FB
S3150802F2A09B687B617B6923F47F437B613B681A0217
S3150802F2B07B681A43BB6813437A6913437B61FB680D
S3150802F2C07A699A6000BF1C37BD465DF8047B7047B1
S3150802F2D080B485B000AF786039607B6893F83C30BB
S3150802F2E0012B01D10223A1E07B68012283F83C208D
S3150802F2F07B68022283F83D207B681B685B68FB609B
S3150802F3007B681B689B68BB607B681B684A4A93429A
S3150802F3100ED07B681B68494A934209D07B681B68F2
S3150802F320474A934204D07B681B68464A934208D1EF
S3150802F330FB6823F47003FB603B685B68FA68134357
S3150802F340FB60FB6823F0007323F07003FB603B68E5
S3150802F3501B68FA681343FB607B681B68FA685A6085
S3150802F3607B681B68344A93424AD07B681B68334AD7
S3150802F370934245D07B681B68B3F1804F40D07B68C7
S3150802F3801B68B3F1A04F3BD07B681B682E4A934299
S3150802F39036D07B681B682D4A934231D07B681B683E
S3150802F3A02B4A93422CD07B681B682A4A934227D061
S3150802F3B07B681B68284A934222D07B681B68274AC7
S3150802F3C093421DD07B681B681D4A934218D07B68FE
S3150802F3D01B681C4A934213D07B681B68204A9342D7
S3150802F3E00ED07B681B681F4A934209D07B681B684C
S3150802F3F01D4A934204D07B681B681C4A93420CD16F
S3150802F400BB6823F08003BB603B689B68BA681343FA
S3150802F410BB607B681B68BA689A607B68012283F8BE
S3150802F4203D207B68002283F83C20002318461437C7
S3150802F430BD465DF8047B7047002C0140002C015044
S3150802F440003401400034015000040040000400501A
S3150802F4500008004000080050000C0040000C005054
S3150802F46000180040001800500040014000400150BA
S3150802F47080B483B000AF786000BF0C37BD465DF834
S3150802F480047B704780B483B000AF786000BF0C3746
S3150802F490BD465DF8047B704780B483B000AF7860E0
S3150802F4A000BF0C37BD465DF8047B704780B483B055
S3150802F4B000AF786000BF0C37BD465DF8047B704725
S3150802F4C080B483B000AF786000BF0C37BD465DF8E4
S3150802F4D0047B704780B483B000AF786000BF0C37F6
S3150802F4E0BD465DF8047B704780B483B000AF786090
S3150802F4F000BF0C37BD465DF8047B704780B582B005
S3150802F50000AF78607B68002B01D1012342E07B685B
S3150802F510D3F88830002B06D17B68002283F8842032
S3150802F5207868F5F785FD7B682422C3F888207B680E
S3150802F5301B681A687B681B6822F001021A607B68DE
S3150802F5409B6A002B02D0786800F020FF786800F0EA
S3150802F5502FFD0346012B01D101231BE07B681B68A3
S3150802F5605A687B681B6822F490425A607B681B685B
S3150802F5709A687B681B6822F02A029A607B681B6875
S3150802F5801A687B681B6842F001021A60786800F004
S3150802F5909FFF034618460837BD4680BD80B582B030
S3150802F5A000AF78607B68002B01D1012331E07B68CC
S3150802F5B02422C3F888207B681B681A687B681B6844
S3150802F5C022F001021A607B681B6800221A607B68B7
S3150802F5D01B6800225A607B681B6800229A6078685A
S3150802F5E0F5F7BCFD7B680022C3F890207B680022F1
S3150802F5F0C3F888207B680022C3F88C207B68002227
S3150802F600DA667B6800221A677B68002283F8842000
S3150802F610002318460837BD4680BD80B58AB002AFBA
S3150802F620F860B9603B601346FB80FB68D3F8883004
S3150802F630202B40F08B80BB68002B02D0FB88002B66
S3150802F64001D1012383E0FB681B689B6803F08003F2
S3150802F650802B07D1FB681B689A68FB681B6822F037
S3150802F66080029A60FB680022C3F89020FB68212278
S3150802F670C3F88820F7F78AFA7861FB68FA88A3F84C
S3150802F6805420FB68FA88A3F85620FB689B68B3F5F2
S3150802F690805F08D1FB681B69002B04D10023FB613C
S3150802F6A0BB68BB6103E0BB68FB610023BB6130E05A
S3150802F6B03B6800937B6900228021F86800F0B2FF5C
S3150802F6C00346002B05D0FB682022C3F888200323B3
S3150802F6D03DE0FB69002B0BD1BB691B881A46FB6808
S3150802F6E01B68C2F308029A62BB690233BB6107E070
S3150802F6F0FB691A78FB681B689A62FB690133FB612E
S3150802F700FB68B3F856309BB2013B9AB2FB68A3F882
S3150802F7105620FB68B3F856309BB2002BC8D13B681B
S3150802F72000937B6900224021F86800F07BFF0346BC
S3150802F730002B05D0FB682022C3F88820032306E0A5
S3150802F740FB682022C3F88820002300E0022318461B
S3150802F7502037BD4680BD000080B58AB000AFF8608C
S3150802F760B9601346FB80FB68D3F88C30202B4BD14B
S3150802F770BB68002B02D0FB88002B01D1012344E091
S3150802F780FB680022DA66FB681B689B6803F0400385
S3150802F790402B07D1FB681B689A68FB681B6822F036
S3150802F7A040029A60FB681B681A4A934224D0FB6897
S3150802F7B01B68194A93421FD0FB681B685B6803F4EF
S3150802F7C00003002B18D0FB681B687B617B6953E832
S3150802F7D0003F3B613B6943F080637B62FB681B68C1
S3150802F7E01A467B6A3B62FA61F9693A6A41E800237A
S3150802F7F0BB61BB69002BE6D1FB881A46B968F86873
S3150802F80000F078FF034600E0022318462837BD4673
S3150802F81080BD00BF002400440024005480B594B083
S3150802F82000AF78607B681B687B637B6B53E8003F9D
S3150802F8303B633B6B23F49073FB647B681B681A4635
S3150802F840FB6C3B64FA63F96B3A6C41E80023BB63D1
S3150802F850BB6B002BE6D17B681B6808333B623B6AAD
S3150802F86053E8003FFB61FB6923F0805323F0010351
S3150802F870BB647B681B680833BA6CFA62BB62B96AF6
S3150802F880FA6A41E800237B627B6A002BE3D17B6834
S3150802F890DB6E012B18D17B681B68FB60FB6853E89B
S3150802F8A0003FBB60BB6823F010037B647B681B6860
S3150802F8B01A467B6CBB617A617969BA6941E80023A9
S3150802F8C03B613B69002BE6D17B681B689B6803F0AA
S3150802F8D04003402B3AD17B68D3F88030002B17D0EF
S3150802F8E07B68D3F88030264ADA667B68D3F880309C
S3150802F8F01846F7F7E5FA0346002B3CD07B68D3F89F
S3150802F9008030DB6E7A68D2F880201046984732E05B
S3150802F9107B680022A3F85E207B6800229A657B68D2
S3150802F9201B680F221A627B681B689A697B681B68C8
S3150802F93042F008029A617B682022C3F88C207B6811
S3150802F9400022DA66786800F0FBFA14E07B68002287
S3150802F950A3F85E207B6800229A657B681B680F22E3
S3150802F9601A627B682022C3F88C207B680022DA663A
S3150802F970786800F0E5FA002318465037BD4680BD80
S3150802F980310A030880B5AEB000AF78607B681B68A1
S3150802F990DB69C7F8B4307B681B681B68C7F8B030E8
S3150802F9A07B681B689B68C7F8AC30D7F8B42040F66A
S3150802F9B00F031340C7F8A830D7F8A830002B1BD17D
S3150802F9C0D7F8B43003F02003002B15D0D7F8B0309F
S3150802F9D003F02003002B05D1D7F8AC3003F080538F
S3150802F9E0002B09D07B685B6F002B00F093827B6843
S3150802F9F05B6F786898478DE2D7F8A830002B00F03D
S3150802FA00FD80D7F8AC207A4B1340002B06D1D7F8E5
S3150802FA10B020784B1340002B00F0F080D7F8B430B2
S3150802FA2003F00103002B11D0D7F8B03003F480732A
S3150802FA30002B0BD07B681B6801221A627B68D3F8FD
S3150802FA40903043F001027B68C3F89020D7F8B430AF
S3150802FA5003F00203002B11D0D7F8AC3003F00103F0
S3150802FA60002B0BD07B681B6802221A627B68D3F8CC
S3150802FA70903043F004027B68C3F89020D7F8B4307C
S3150802FA8003F00403002B11D0D7F8AC3003F00103BE
S3150802FA90002B0BD07B681B6804221A627B68D3F89A
S3150802FAA0903043F002027B68C3F89020D7F8B4304E
S3150802FAB003F00803002B17D0D7F8B03003F0200361
S3150802FAC0002B05D1D7F8AC20494B1340002B0BD09D
S3150802FAD07B681B6808221A627B68D3F8903043F069
S3150802FAE008027B68C3F89020D7F8B43003F40063A1
S3150802FAF0002B12D0D7F8B03003F08063002B0CD05D
S3150802FB007B681B684FF400621A627B68D3F89030F0
S3150802FB1043F020027B68C3F890207B68D3F89030C4
S3150802FB20002B00F0F981D7F8B43003F02003002B3C
S3150802FB3013D0D7F8B03003F02003002B05D1D7F83D
S3150802FB40AC3003F08053002B07D07B685B6F002B29
S3150802FB5003D07B685B6F786898477B68D3F89030E8
S3150802FB60C7F8A4307B681B689B6803F04003402BE8
S3150802FB7005D0D7F8A43003F02803002B2ED07868D6
S3150802FB8000F0DAFE7B681B689B6803F04003402B93
S3150802FB9020D17B68D3F88030002B17D07B68D3F846
S3150802FBA08030154ADA667B68D3F880301846F7F74C
S3150802FBB087F90346002B19D07B68D3F88030DB6EB1
S3150802FBC07A68D2F88020104698470FE07868F6F7E8
S3150802FBD05DFF0BE07868F6F759FF07E07868F6F7F5
S3150802FBE055FF7B680022C3F8902095E100BF93E198
S3150802FBF00100001020010004050A03087B68DB6E79
S3150802FC00012B40F02981D7F8B43003F01003002BFA
S3150802FC1000F02281D7F8B03003F01003002B00F071
S3150802FC201B817B681B6810221A627B681B689B68AB
S3150802FC3003F04003402B40F091807B68D3F8803074
S3150802FC401B689B6CA7F89230B7F89230002B00F02D
S3150802FC5065817B68B3F85C30B7F892209A4280F0E7
S3150802FC605D817B68B7F89220A3F85E207B68D3F89B
S3150802FC7080301B6D812B60D07B681B687B677B6F2E
S3150802FC8053E8003F3B673B6F23F48073C7F88C3019
S3150802FC907B681B681A46D7F88C30C7F88030FA6733
S3150802FCA0F96FD7F8802041E80023BB67BB6F002BAA
S3150802FCB0E2D17B681B6808333B663B6E53E8003F1C
S3150802FCC0FB65FB6D23F00103C7F888307B681B6868
S3150802FCD00833D7F88820FA66BB66B96EFA6E41E829
S3150802FCE000237B667B6E002BE3D17B682022C3F858
S3150802FCF08C207B680022DA667B681B68FB64FB6CD7
S3150802FD0053E8003FBB64BB6C23F01003C7F884308A
S3150802FD107B681B681A46D7F88430BB657A65796DA5
S3150802FD20BA6D41E800233B653B6D002BE4D17B6845
S3150802FD30D3F880301846F7F747F87B6802221A6725
S3150802FD407B68B3F85C207B68B3F85E309BB2D31A43
S3150802FD509BB21946786800F0FDF8DFE07B68B3F8D5
S3150802FD605C207B68B3F85E309BB2D31AA7F8A23040
S3150802FD707B68B3F85E309BB2002B00F0D180B7F8EF
S3150802FD80A230002B00F0CC807B681B68BB63BB6B80
S3150802FD9053E8003F7B637B6B23F49073C7F89C3070
S3150802FDA07B681B681A46D7F89C307B643A64396CC0
S3150802FDB07A6C41E80023FB63FB6B002BE4D17B687A
S3150802FDC01B6808337B627B6A53E8003F3B623B6AE7
S3150802FDD023F0805323F00103C7F898307B681B6829
S3150802FDE00833D7F898203A63FB62F96A3A6B41E816
S3150802FDF00023BB62BB6A002BE1D17B682022C3F8D1
S3150802FE008C207B680022DA667B6800225A677B6848
S3150802FE101B683B613B6953E8003FFB60FB6823F0C4
S3150802FE201003C7F894307B681B681A46D7F89430D3
S3150802FE30FB61BA61B969FA6941E800237B617B69AA
S3150802FE40002BE4D17B6802221A67B7F8A23019465A
S3150802FE50786800F07FF863E0D7F8B43003F48013CB
S3150802FE60002B0ED0D7F8AC3003F48003002B08D051
S3150802FE707B681B684FF480121A62786801F060FB8F
S3150802FE8051E0D7F8B43003F08003002B14D0D7F82A
S3150802FE90B03003F08003002B05D1D7F8AC3003F459
S3150802FEA00003002B08D07B689B6F002B3AD07B6837
S3150802FEB09B6F7868984735E0D7F8B43003F040036B
S3150802FEC0002B09D0D7F8B03003F04003002B03D03B
S3150802FED0786800F0D2FD26E0D7F8B43003F40003C0
S3150802FEE0002B09D0D7F8B03003F08043002B03D09B
S3150802FEF0786801F039FB16E0D7F8B43003F080735E
S3150802FF00002B10D0D7F8B030002B0CDA786801F045
S3150802FF1021FB08E000BF06E000BF04E000BF02E0E4
S3150802FF2000BF00E000BFB837BD4680BD80B483B0CD
S3150802FF3000AF786000BF0C37BD465DF8047B70479A
S3150802FF4080B483B000AF786000BF0C37BD465DF859
S3150802FF50047B704780B483B000AF78600B467B8021
S3150802FF6000BF0C37BD465DF8047B704780B485B088
S3150802FF7000AF78607B68D3F88830FB607B68D3F87B
S3150802FF808C30BB60FA68BB68134318461437BD4603
S3150802FF905DF8047B704780B483B000AF78607B68F5
S3150802FFA0D3F8903018460C37BD465DF8047B704787
S3150802FFB02DE9B04F94B000AFF862002387F84730B6
S3150802FFC0FB6A1A68784B9A42FB6A9A68FB6A1B694B
S3150802FFD01A43FB6A5B691A43FB6ADB691343FB64D0
S3150802FFE0FB6A1B681B6871491940FB6A1A68FB6C35
S3150802FFF00B431360FB6A1B685B6823F44050FB6A79
S31508030000D968FB6A1A6840EA01035360FB6A9B696D
S31508030010FB64FB6A1A68644B9A4209D0FB6A1A683E
S31508030020634B9A4204D0FB6A1A6AFB6C1343FB645C
S31508030030FB6A1B689B6823F06E4121F43061FB6AF7
S315080300401A68FB6C0B439360FB6A1B68DB6A23F035
S315080300500F00FB6A596AFB6A1A6840EA0103D3620E
S31508030060FB6A1A68534B9A4202D10123BB6466E0C2
S31508030070FB6A1A68504B9A4202D10223BB645EE0BC
S31508030080FB6A1A684D4B9A4202D10423BB6456E0B5
S31508030090FB6A1A684A4B9A4202D10823BB644EE0AC
S315080300A0FB6A1A68474B9A4202D11023BB6446E09F
S315080300B0FB6A1A68444B9A4202D12023BB643EE08A
S315080300C0FB6A1A68414B9A4202D14023BB6436E065
S315080300D0FB6A1A683E4B9A4202D18023BB642EE020
S315080300E0FB6A1A683B4B9A4203D14FF48073BB648D
S315080300F025E0FB6A1A68384B9A4203D14FF400731A
S31508030100BB641CE0FB6A1A68344B9A4203D14FF46A
S315080301108063BB6413E0FB6A1A68314B9A4203D1C6
S315080301204FF40063BB640AE0FB6A1A681E4B9A42E3
S3150803013003D14FF48053BB6401E00023BB64FB6A1D
S315080301401A68194B9A4205D0FB6A1A68184B9A42E1
S3150803015040F09480BB6C00223B627A62D7E90801BF
S31508030160FBF7DCFE38643B6C002B00F0F780FB6A78
S315080301705B6A1C4A32F813301A463B6CB3FBF2F33C
S315080301807B63FB6A5A6813465B0013447A6B9A428D
S3150803019005D3FB6A5B681B037A6B9A4224D901234E
S315080301A087F8473069E000BF00240044F369FFCFAE
S315080301B00024005400380140004400400048004031
S315080301C0004C0040005000400064004000780040A6
S315080301D0007C00400080004000680040006C00403E
S315080301E00084004020B203083B6C0022BB61FA611D
S315080301F0FB6A5B6A644A32F813309BB200223B619E
S315080302007A61D7E90423D7E90601F0F74DFD0246DB
S315080302100B46104619464FF000024FF000030B0237
S3150803022043EA10630202F96A4968490800200C4642
S31508030230054612EB040843EB0509FB6A5B680022D3
S31508030240BB60FA60D7E9022340464946F0F72CFD1E
S3150803025002460B461346FB63FB6BB3F5407F08D395
S31508030260FB6BB3F5801F04D2FB6A1B68FA6BDA6073
S3150803027003E0012387F8473070E06FE0FB6ADB6928
S31508030280B3F5004F3CD1BB6C00223B607A60D7E9DB
S315080302900001FBF743FE38643B6C002B5ED0FB6A18
S315080302A05B6A394A32F813301A463B6CB3FBF2F3EE
S315080302B05A00FB6A5B685B081A44FB6A5B68B2FB15
S315080302C0F3F3FB63FB6B0F2B16D9FB6BB3F5803F7D
S315080302D012D2FB6B9BB223F00F037B87FB6B5B0886
S315080302E09BB203F007039AB27B8F13437B87FB6AA0
S315080302F01B687A8FDA6031E0012387F847302DE0EF
S31508030300BB6C00229A46934650465946FBF706FEAF
S3150803031038643B6C002B21D0FB6A5B6A1A4A32F8B5
S3150803032013301A463B6CB3FBF2F2FB6A5B685B0855
S315080303301A44FB6A5B68B2FBF3F3FB63FB6B0F2B95
S3150803034009D9FB6BB3F5803F05D2FB6B9AB2FB6AFF
S315080303501B68DA6002E0012387F84730FB6A01224B
S31508030360A3F86A20FB6A0122A3F86820FB6A002225
S315080303705A67FB6A00229A6797F847301846503738
S31508030380BD46BDE8B08F00BF20B2030880B483B072
S3150803039000AF78607B689B6A03F00803002B0AD0DA
S315080303A07B681B685B6823F400417B689A6B7B68F0
S315080303B01B680A435A607B689B6A03F00103002B98
S315080303C00AD07B681B685B6823F400317B68DA6AAA
S315080303D07B681B680A435A607B689B6A03F00203BF
S315080303E0002B0AD07B681B685B6823F480317B6823
S315080303F01A6B7B681B680A435A607B689B6A03F01F
S315080304000403002B0AD07B681B685B6823F48021EE
S315080304107B685A6B7B681B680A435A607B689B6ACE
S3150803042003F01003002B0AD07B681B689B6823F430
S3150803043080517B68DA6B7B681B680A439A607B6822
S315080304409B6A03F02003002B0AD07B681B689B6812
S3150803045023F400517B681A6C7B681B680A439A600D
S315080304607B689B6A03F04003002B1AD07B681B68E2
S315080304705B6823F480117B685A6C7B681B680A43A4
S315080304805A607B685B6CB3F5801F0AD17B681B686F
S315080304905B6823F4C0017B689A6C7B681B680A4314
S315080304A05A607B689B6A03F08003002B0AD07B683B
S315080304B01B685B6823F400217B68DA6C7B681B681E
S315080304C00A435A6000BF0C37BD465DF8047B704784
S315080304D080B598B002AF78607B680022C3F8902095
S315080304E0F6F754FB78657B681B681B6803F00803FB
S315080304F0082B2FD16FF07E4300937B6D00224FF4B8
S315080305000011786800F08EF80346002B22D07B682A
S315080305101B68BB63BB6B53E8003F7B637B6B23F0B2
S3150803052080033B657B681B681A463B6D7B643A64AC
S31508030530396C7A6C41E80023FB63FB6B002BE6D12D
S315080305407B682022C3F888207B68002283F88420EE
S31508030550032363E07B681B681B6803F00403042B0F
S3150803056049D16FF07E4300937B6D00224FF48001DF
S31508030570786800F057F80346002B3CD07B681B6865
S315080305807B627B6A53E8003F3B623B6A23F49073C2
S31508030590FB647B681B681A46FB6C3B63FA62F96A61
S315080305A03A6B41E80023BB62BB6A002BE6D17B6842
S315080305B01B6808333B613B6953E8003FFB60FB68F4
S315080305C023F00103BB647B681B680833BA6CFA61C2
S315080305D0BB61B969FA6941E800237B617B69002B32
S315080305E0E5D17B682022C3F88C207B68002283F838
S315080305F08420032312E07B682022C3F888207B68C3
S315080306002022C3F88C207B680022DA667B680022E6
S315080306101A677B68002283F8842000231846583714
S31508030620BD4680BD80B584B000AFF860B9603B6055
S315080306301346FB7149E0BB69B3F1FF3F45D0F6F7B3
S31508030640A5FA02463B68D31ABA699A4202D3BB692A
S31508030650002B01D1032348E0FB681B681B6803F0E2
S315080306600403002B31D0FB681B68DB6903F008031E
S31508030670082B10D1FB681B6808221A62F86800F079
S315080306805BF9FB680822C3F89020FB68002283F80D
S315080306908420012329E0FB681B68DB6903F40063F4
S315080306A0B3F5006F11D1FB681B684FF400621A6239
S315080306B0F86800F041F9FB682022C3F89020FB682C
S315080306C0002283F8842003230FE0FB681B68DA699A
S315080306D0BB681340BA689A420CBF01230023DBB2F6
S315080306E01A46FB799A42A6D0002318461037BD4608
S315080306F080BD000080B4A3B000AFF860B9601346AC
S31508030700FB80FB68BA689A65FB68FA88A3F85C20DD
S31508030710FB68FA88A3F85E20FB6800225A67FB6821
S315080307209B68B3F5805F0ED1FB681B69002B05D167
S31508030730FB6840F2FF12A3F860202DE0FB68FF2256
S31508030740A3F8602028E0FB689B68002B0DD1FB68A3
S315080307501B69002B04D1FB68FF22A3F860201BE06A
S31508030760FB687F22A3F8602016E0FB689B68B3F159
S31508030770805F0DD1FB681B69002B04D1FB687F22C0
S31508030780A3F8602008E0FB683F22A3F8602003E093
S31508030790FB680022A3F86020FB680022C3F89020B8
S315080307A0FB682222C3F88C20FB681B6808337B6628
S315080307B07B6E53E8003F3B663B6E43F00103C7F885
S315080307C08430FB681B680833D7F884203A67FB66CE
S315080307D0F96E3A6F41E80023BB66BB6E002BE3D183
S315080307E0FB685B6EB3F1005F4FD1FB68B3F8683003
S315080307F0FA889A4249D3FB689B68B3F5805F07D1A9
S31508030800FB681B69002B03D1FB68474A5A6702E05A
S31508030810FB68464A5A67FB681B69002B1AD0FB68B4
S315080308201B683B653B6D53E8003FFB64FB6C43F475
S315080308308073C7F88030FB681B681A46D7F8803080
S31508030840FB65BA65B96DFA6D41E800237B657B6D77
S31508030850002BE4D1FB681B680833FB63FB6B53E887
S31508030860003FBB63BB6B43F08053FB67FB681B68A6
S315080308700833FA6FBA647B64796CBA6C41E800236F
S315080308803B643B6C002BE5D146E0FB689B68B3F5FC
S31508030890805F07D1FB681B69002B03D1FB68244AD9
S315080308A05A6702E0FB68234A5A67FB681B69002BF1
S315080308B019D0FB681B68BB62BB6A53E8003F7B62BF
S315080308C07B6A43F490737B67FB681B681A467B6FE6
S315080308D07B633A63396B7A6B41E80023FB62FB6AF5
S315080308E0002BE6D118E0FB681B687B617B6953E83C
S315080308F0003F3B613B6943F02003BB67FB681B680A
S315080309001A46BB6F3B62FA61F9693A6A41E8002302
S31508030910BB61BB69002BE6D1002318468C37BD465D
S315080309205DF8047B704700BFC9110308590E030815
S31508030930950C0308D10A030880B495B000AF786014
S315080309407B681B687B637B6B53E8003F3B633B6BAE
S3150803095023F49073FB647B681B681A46FB6C3B6441
S31508030960FA63F96B3A6C41E80023BB63BB6B002B54
S31508030970E6D17B681B6808333B623B6A53E8003F52
S31508030980FB61FB6923F0805323F00103BB647B6897
S315080309901B680833BA6CFA62BB62B96AFA6A41E839
S315080309A000237B627B6A002BE3D17B68DB6E012B1A
S315080309B018D17B681B68FB60FB6853E8003FBB6084
S315080309C0BB6823F010037B647B681B681A467B6C41
S315080309D0BB617A617969BA6941E800233B613B697E
